:020000040800F2
:1000000000000220B9000C083D010C08F5B30608F9
:100010003D010C083D010C083D010C0800000000EA
:100020000000000000000000000000003D010C087E
:100030003D010C08000000003D010C08E5410508E9
:100040003D010C083D010C083D010C083D010C0868
:100050003D010C083D010C084D040508510405083C
:1000600055040508590405085D040508D93F04082E
:10007000ED3F040801400408154004082940040825
:100080003D400408514004083D010C083D010C08A6
:100090003D010C083D010C083D010C0861040508F8
:1000A0003D010C083D010C083D010C08794A04088B
:1000B0008D4A0408A14A0408B54A04080933040813
:1000C000FD3204083D330408313304083D010C08B7
:1000D0003D010C084D5404085954040865540408A3
:1000E000650405083D010C0800000000F14A040801
:1000F000414B0408694B0408DD4A040865400408C4
:100100003D010C08C1640408C94A04083D010C08FB
:10011000715404083D010C083D010C0819990408AC
:10012000794004088D400408A1400408B540040843
:10013000C94004083D010C083D010C083D010C08B4
:1001400000000000000000000000000000000000AF
:10015000DD400408F1400408054104087D5404080A
:1001600071330408653304083D010C083D010C0897
:100170003D010C083D010C083D010C080000000089
:100180003D010C083D010C088954040895540408ED
:100190003D010C083D010C083D010C083D010C0817
:1001A0003D010C083D010C083D010C083D010C0807
:1001B0003D010C083D010C083D010C083D010C08F7
:1001C0003D010C083D010C083D010C083D010C08E7
:1001D0003D010C08298504083D010C083D010C086F
:1001E0003D010C083D010C083D010C083D010C08C7
:1001F0003D010C083D010C083D010C083D010C08B7
:100200003D010C083D010C083D010C083D010C08A6
:10021000054B0408194B04082D4B04083D010C083C
:100220003D010C083D010C083D010C0800000000D8
:10023000C56404083D010C08000000003D010C08E5
:100240003D010C083D010C083D010C083D010C0866
:100250003D010C083D010C083D010C083D010C0856
:100260003D010C083D010C083D010C083D010C0846
:100270003D010C083D010C083D010C080000000088
:100280003D010C08000000003D010C0800000000CA
:08029000000000003D010C0814
:0802980064F00B0001000000FE
:1002A000F8AD01240207000006003F0018AE01244B
:1002B0000207000106003F0038AE012402070000DB
:1002C00006035B0058AE0124010C0000000176001B
:1002D00078AE0124011000000001760098AE0124E0
:1002E000010D010000017700B8AE012401120000E9
:1002F00000017600D8AE01240117000000010C00B7
:10030000F8AE01240118000000010E0018AF01240E
:10031000021E00000002520038AF01240129010032
:100320000000180058AF012401210000000048001F
:1003300078AF0124012200000000490098AF012499
:100340000123000000004A00B8AF0124012400008E
:1003500000004B00D8AF01240125000000004C0034
:10036000F8AF01240126000000004D0018B0012460
:100370000127000000004E0038B0012401280000D1
:1003800000004F0058B00124012C0000000029009B
:1003900078B00124012D01000000290098B001244B
:1003A000012E010000007000B8B0012401300000EF
:1003B00000003100D8B00124012F010000005200DC
:1003C000F8B00124013101000000280018B1012417
:1003D000013201000000280038B10124022A050082
:1003E00000012C0058B101240135000000013C003F
:0C03F00078B1012401380000000020005A
:020000040804EE
:10000000836B5A6D12F0500F5A6D1AD1196842F471
:1000100000725A650A6812F0080FCA6816D012F406
:10002000406F15D1CA68920412D45A6D22F48072BE
:100030005A655A6DD1040BD45A6D42F001025A65CB
:100040007047D20604D4DB6CDB6C18479007ECD009
:10005000704700BF704700BF836B5A6D42F040028B
:100060005A659A6D42F004029A65704702685549D4
:1000700038B5554B554D564CAA4218BF9A420CBF45
:10008000012300238A4208BF43F001033031A2421A
:1000900008BF43F0010330348A4208BF43F0010334
:1000A0003031A24208BF43F0010330348A4208BF16
:1000B00043F0010301F55C71A24208BF43F0010364
:1000C00004F55C748A4208BF43F001033031A24258
:1000D00008BF43F0010330348A4208BF43F00103F4
:1000E0003031A24208BF43F0010330348A4208BFD6
:1000F00043F001033031A24208BF43F001038A42BA
:1001000008BF43F0010313B9324B9A4208D10423CC
:1001100080F83530136823F001031360002038BDE8
:100120002D4B2E4D1168AA4218BF9A422C4C21F03B
:100130000E0105F13C050CBF012300231160A24212
:1001400008BF43F0010311682834AA4208BF43F0F6
:10015000010321F00101A24208BF43F0010314345E
:100160001160A24208BF43F001031E498A4208BF42
:1001700043F0010313B91C4B9A4217D10123856D3B
:10018000D0E91714226801F01F0122F480728B401D
:1001900022606B60C36ED0E91921516033B11A68D7
:1001A000D0E91C1422F480721A604C6001210022F4
:1001B000036D80F8351080F83420002BAED09847BE
:1001C000ACE700BF4000024010000240280002409F
:1001D00058000240B80402401C5402580854025807
:1001E0003054025880540258945402580168002236
:1001F0000B6880F842205A0410B40ED50B6823F423
:1002000080430B6090F84130292B10D090F841309A
:100210002A2B24D05DF8044B70471B04F2D50B68E1
:1002200023F400430B6090F84130292BEED12822B3
:10023000212380F841200022036390F841300C68AC
:1002400003F02803282B14BF6FF0F2036FF0420372
:1002500023405DF8044B0B6080F840207047282253
:10026000222380F841200022036390F841300C687B
:1002700003F02803282B14BF6FF0F4036FF044033E
:1002800023405DF8044B0B6080F84020704700BFAE
:100290000023202210B4174C4363C462036380F828
:1002A000412080F842304B07026811D5526A436AF8
:1002B0001A70436A028D013343624AB1438D013A99
:1002C000013B02859BB24385436C43F004034364C6
:1002D0000368102490F84120002190F841201A680A
:1002E00022F0FE021A60DC615DF8044B80F84010D9
:1002F000704700BF0000FFFF70B5574B002590F816
:100300004120044680F84250283AC3624585436C38
:10031000022A41EA0301036841642FD890F8411092
:1003200090F84120282001F0280102F02802282915
:1003300014BFF6214621282A1A680CBFC9436FF062
:10034000F6010A4045491A6084F84100A06B226B0F
:10035000616318B1112A42D0212A40D0E06B18B154
:10036000122A51D0222A4FD094F84130602B4FF0FE
:1003700000032DD0236384F8403070BD90F84120F5
:1003800090F841201A6822F0FE021A609A699207DA
:1003900000D59D629A69D60703D49A6942F001029A
:1003A0009A6194F84120602A10D0202284F84120DC
:1003B0009A6995060AD59A69D00605D51022DA61A0
:1003C000626C42F0040262642022DA610021BDE71F
:1003D000202284F8403084F84120236370BD1A68DD
:1003E00051042CD490F83530012BBDD000221C4B89
:1003F000036584F8402090F83520022A24D080221A
:100400004265BDE8704018471A68120403D51A689F
:1004100022F400421A6090F83530012BA4D000225B
:100420000F4B036584F8402090F83520022AE6D16E
:10043000FFF71CFE0028A0D0E06B036DE1E71A680F
:1004400022F480421A60CDE7FFF710FE002894D016
:10045000A06B036DD5E700BF0000FFFFDD040408BB
:100460002D08040803689A69196810B4D40528D5C2
:100470000C0606D4416C11F00B0F1FD15DF8044B34
:100480007047416C4FF4807441F0010141645105A3
:10049000DC6120D5416C4FF48064920541F0080185
:1004A0004164DC61E6D5426C4FF4007142F0020217
:1004B0004264D961416C11F00B0FDFD05DF8044B41
:1004C0001AE7540502D50906E4D4D3E79405D1D53B
:1004D0000906E8D4CEE79205E5D4CBE7F8B590F865
:1004E00040300D46C16A012B00F008810123AE06A1
:1004F000044680F8403001D5900656D4EB0619D555
:10050000D70617D5638D9BB2002B40F0F98094F885
:100510004130B1F1007FDBB240F0D580282B40F0B4
:10052000D28029462046FFF7B3FE0023184684F800
:100530004030F8BD68071AD42F0701D516074AD4F2
:10054000A807F2D59307F0D5638D9BB2002B00F07E
:10055000FA80616A236811F8010B228D9862638D1D
:10056000013A6162013B22859BB26385DDE7530757
:10057000E2D5638D9BB26BB12268636A526A1A70CE
:10058000638D606A228D013B0130013A9BB260624B
:1005900022856385638D9BB2002BC6D111F5803F08
:1005A000C3D02046FFF722FEBFE72368202118684A
:1005B000E66A94F84120D961213A092A1ED8DFE879
:1005C00012F0C70015001D001D001D001D001D00BC
:1005D000F000C700150094F84130226803F02803AA
:1005E000282B00F0C5800823D3619EE794F84120B2
:1005F0001A6822F0FC021A60222222635A68894992
:1006000042F400425A605A680A405A609A69910757
:1006100001D500229A629A69D20703D49A6942F0FE
:1006200001029A6147047BD51A6822F480421A605D
:10063000A26B1AB111684A6892B262856A070BD53B
:100640005A6A25F00405636A1A70636A01336362AB
:10065000238D002B40F08580638D9BB21BB1636CB2
:1006600043F004036364EB061AD5C70618D5638DFF
:100670009BB2002B40F0AA8094F84130282B03D184
:10068000B6F1007F00F0C98094F8413016F5803F44
:100690002268DBB202D0292B00F0AD801023D36199
:1006A000002384F84230666C6363002E40F084803F
:1006B000E36A5D4DAB423DD194F84130202384F88C
:1006C0004130266331E794F841202368292A4FF00E
:1006D0001002DA617FF429AF11F5803F3FF425AFB6
:1006E0009A69960701D500229A629A69D5073FF563
:1006F00058AF9A6942F001029A6152E70220F8BDB0
:1007000023681022DA61636C43F00403636431F000
:1007100080737FF40AAF616C2046FFF7EDFD04E7BC
:1007200001048BD51A6822F400421A60E26B002A99
:1007300080D183E72046FFF759FD2023E56284F846
:1007400041302663F1E631F080737FF4EEAE28E7A6
:1007500094F841201A6822F0FA021A6021222263DA
:100760004CE7013B2385638D013B9BB2638573E7B7
:10077000E1689369022990699368D56836D1C3F31B
:10078000C21383EA104313F006032FD1A16C013189
:10079000A164A16C02297FF4C8AE0821A364D161D1
:1007A000C3E694F8412094F841201A6822F0FE0232
:1007B0001A600022226321E7616C2046FFF79CFD4E
:1007C00094F84130282B7FF4B0AEAAE623681022BB
:1007D000DA61636C43F00403636436F080737FF482
:1007E0005FAF616C2046FFF787FD59E7136823F080
:1007F000B803136099E61023D3619369980701D574
:10080000002393629369D90703D4936943F00103EA
:1008100093612046FFF7EAFC42E729462046FFF7AE
:1008200037FD3DE700E800FE0000FFFF836B9A6B99
:100830000AB100211165DA6B0AB10021116593F844
:100840004120602A05D000221A63002283F840204C
:1008500070470022202183F841101A63002283F898
:1008600040207047016870B4CC072DD5914A1369B8
:10087000926A03F03803102B00F0E180182B00F08F
:10088000D9804368B3F5803F00F00581002B00F06C
:100890005A81B3F5A02F874B1A6800F0678222F4C3
:1008A00080321A601A6822F480221A60824B41F268
:1008B000883C804C1D6804E01A68521B624500F2B7
:1008C0003F8122689603F7D58A0768D4CD0631D5D3
:1008D000784A1369926A03F03803082B00F0C0804D
:1008E000182B00F0B880C369724C002B00F05F81B8
:1008F0002268714B42F0800222601D6804E01A6891
:10090000521B022A00F21C812268D205F7D56B4BDC
:10091000026A1D6841F20303B3EB154FC0F0448235
:100920006368202A23F0F8430CBF43F0804343EA76
:10093000826363600D0713D543695E4C002B00F0A2
:100940001881626F5C4B42F0010262671D6804E02F
:100950001A68521B022A00F2F380626F9207F7D5E1
:100960008C0613D58369534C002B00F0118122684B
:10097000514B42F4805222601D6804E01A68521BF9
:10098000022A00F2DD8022689204F7D5490700F1BF
:100990008880436A002B40F0BC80002059E0454A23
:1009A0001369926A13F038032BD1424AC368126864
:1009B000520701D5002B4BD03E4C226822F0190281
:1009C0001A433D4B22601D6804E01A68521B022A3C
:1009D00000F2B68022685607F7D5384B02691D68C9
:1009E00041F20303B3EB154F6368C0F0028123F4B7
:1009F0007C33402A0CBF43F4003343EA0233636084
:100A000064E7182B00F0F180C3682A4C002B00F03B
:100A1000DD80226822F019021A43274B22601D68EC
:100A200004E01A68521B022A00F28A8022685207E8
:100A3000F7D5D2E702F00302022A7FF422AF1D4B62
:100A40001B689B037FF540AF4368002B7FF43CAFEE
:100A5000012070BC704702F00302012A7FF443AF0B
:100A6000144B1B68DC0502D5C369802BF0D1134CF5
:100A700041F20303026A2468B3EB144FC0F0BF8055
:100A8000202A00F09E810B4C636823F0F84343EA70
:100A9000826363604EE7074A136843F48033136050
:100AA00004E70749044B0A6842F480720A601C6834
:100AB0000CE000BF00440258802E00240010005CAF
:100AC000004802581A68121B642A39D80A68D505EA
:100AD000F8D58268012A00F06E81002A00F04E816C
:100AE000052A9F4A116F00F0748121F001011167FE
:100AF000116F21F0040111671D6841F28834984993
:100B000003E01A68521BA2421AD80A6F9207F8D55E
:100B10003FE793490A6902F03802182A00F0D580AD
:100B20000A68022B8F4B22F080720A606FD018681F
:100B30000A6892017FF531AF1A68121A022AF7D9B2
:100B4000032070BC7047864C41F28835854B226883
:100B500022F480322260226822F4802222601E6801
:100B600003E01A68921BAA42EAD822689203F8D4DA
:100B7000AAE6626F7B4B22F0010262671D6803E008
:100B80001A68521B022ADBD8626F9607F8D4E7E690
:100B90002268744B22F4805222601D6803E01A68B8
:100BA000521B022ACCD822689604F8D4EEE62268BA
:100BB0006C4B22F0800222601D6803E01A68521B11
:100BC000022ABDD82268D605F8D4B3E62268654B60
:100BD00022F0010222601D6803E01A68521B022AFB
:100BE000AED822685607F8D470E694077FF40CAFAD
:100BF000DBE623F0FE4343EA0263636066E6584C9B
:100C0000E36823F07C5343EA0263E36092E61C68E6
:100C100003E01A68121B022A92D80A689501F8D4D8
:100C20008C6A514A2240846A2243C46A42EA04120E
:100C30008A62D0E90D24013A013C5202240492B2A6
:100C400004F4FE042243046B013CC4F30804224371
:100C5000C46B013C240604F0FE4422430A63CA6AC2
:100C600022F00102CA624A6B846C6FF3CF0242EA3F
:100C7000C4024A63CA6A046C22F00C022243384C54
:100C8000CA62CA6A406C22F002020243CA62CA6A9D
:100C900042F48032CA62CA6A42F40032CA62CA6A44
:100CA00042F48022CA62CA6A42F00102CA620A6839
:100CB00042F080720A601968226890013FF56DAEBB
:100CC0001A68521A022AF7D93AE7012B8A6A0D6B81
:100CD0003FF4BEAE02F00303846AA3427FF4B8AED1
:100CE000C2F30512C36A9A427FF4B2AE036BC5F336
:100CF0000802013B9A427FF4ABAE436BC5F3462238
:100D0000013B9A427FF4A4AE836BC5F30642013BDC
:100D10009A427FF49DAEC36BC5F30665013B9D42CD
:100D20007FF496AE4B6B816CC3F3CC0399423FF4D6
:100D300034AE0B480B4BC26A22F00102C2621A6841
:100D400018688242FCD0064A536B6FF3CF0343EA24
:100D5000C1035363D36A43F00103D3621DE600BFAE
:100D600000440258802E00240CFCFFFF42F4802235
:100D70001A601A6842F480321A6097E5194941F204
:100D800088350A6F22F001020A670A6F22F0040216
:100D90000A671C6804E01A68121BAA423FF6D0AE2C
:100DA0000A6F9607F7D4F4E5E36823F07C5343EA2F
:100DB0000263E360BEE50B490A6F42F001020A6775
:100DC0009AE6084A536823F0F84343F0804353609F
:100DD000B0E541F004011167116F41F001011167A5
:100DE0008AE600BF00440258334B30B4996A9C6ACB
:100DF000DD6A14F47C7F5A6BC4F3051036D0C2F35D
:100E0000CC0205F0010501F0030107EE900A05FB95
:100E100002F20129B8EEE77A06EE902AFAEEE96AC4
:100E200002D0022942D019B3DFED247A87EE876A17
:100E30001B6BC3F3080307EE903AF7EE005AF8EE87
:100E4000E77A77EEA67A77EEA57A67EE867A1A4B7E
:100E50001B6BC3F34623013307EE103AF8EEC76A63
:100E600087EEA67AFCEEC77A17EE900A30BC704780
:100E70001A6892061DD51968F7EE005A104A1B6BC6
:100E8000C1F3C101C3F30803CA4007EE903A06EE6E
:100E9000102AF8EEE77AB8EEC66A77EEA66AC6EED2
:100EA000077A36EEA57A67EE877AD0E7DFED057A26
:100EB000BCE7DFED057AB9E7004402580024744A24
:100EC0000090D0030024F44A0024744C836A1A076B
:100ED00010B406D50168846B4A6822F400422243AC
:100EE0004A60DC0706D50168C46A4A6822F4003209
:100EF00022434A60990706D50168046B4A6822F4C8
:100F0000803222434A605A0706D50168446B4A681A
:100F100022F4802222434A60DC0606D50168C46BB5
:100F20008A6822F4805222438A60990606D50168B5
:100F3000046C8A6822F4005222438A605A060AD559
:100F40000168446C4A68B4F5801F22F4801242EABA
:100F500004024A600BD01B0606D50268C16C5368B8
:100F600023F400230B4353605DF8044B70474A6839
:100F7000846C22F4C00222434A60ECE70022836BB7
:100F8000A3F85E20704700BF124B41F2883C124A22
:100F900001461B68A2FB03235B0A0CFB03F33BB176
:100FA0004A6B12F0450F01D0920404D5013BF7D1F2
:100FB0004FF0004070474B6B5B0707D4486B10F055
:100FC000010014BF0123054B8B63704704231846AF
:100FD0008B63704700000024D34D6210C5002000D1
:100FE000036942681F2B70B430D9A3F1200520217A
:100FF0005468A940214227D08169087C022835D055
:1010000048681F2BC9681B4D4E680169C1F3032452
:10101000194951F8244015F804C0056856F80C40E9
:1010200024F0010446F80C40407901EB4001088CA3
:10103000E96800F4F05021EA0001E96010D9A3F159
:10104000200120238B40D36070BC7047202114689E
:1010500099402142F8D08169087C0228D0D105E06E
:10106000202101FA03F370BC9360704700200874DC
:10107000C6E700BF888D0C08188C0C08D0E9072340
:101080009A423CBFC1685218D01A7047D0E9092370
:1010900000699A4238BF12180138D31AC01A704733
:1010A000D0E90902101AB0FA80F04009704700BF79
:1010B000016A034640694A1C405CD9688A4228BFDD
:1010C00000221A62704700BF436A826910B4D1548B
:1010D000436A416B046901330A68A34228BF0023B5
:1010E0005DF8044B42F0800243620A60704700BF23
:1010F000436BD86910F0100002D0102201201A6250
:10110000704700BF704700BF704700BF704700BF07
:1011100001207047014B5868704700BF802E0024A3
:10112000074B93F8A422012A01D10020704793F8BD
:10113000A402A0F10300B0FA80F04009704700BF9C
:10114000802E0024012380F849307047EFF311828C
:10115000702383F312880849D2B2D1E9B93182F3FE
:101160001188581E8B42A0EB01008CBF0023012385
:1011700000EB0330704700BF802E002470B5D0F81C
:10118000D442D0F8C86200EB840EDEF8C05245B3FA
:1011900001F00F040A4604EB840C00EB8C0CDCF825
:1011A00018306BB9DEF8C43200211B69C5F814127F
:1011B00023B105F50471D5F808029847002070BDE9
:1011C00004EBC40406EB8406F469B3FBF4F604FBF9
:1011D0001633002BE6D11A46CCF818307CF034FDDB
:1011E000ECE7032070BD00BFD0F8D42200EB8202F0
:1011F00010B5D2F8C042ACB101F00F03D0F8C8026C
:10120000D2F8C42204F5037103EBC303D26800EBE8
:101210008303D4F80402D3F86832C4F80C32904740
:10122000002010BD032010BDD0F8D43200EB8300A5
:1012300010B5D0F8C04284B1D0F8C4325BB194F894
:101240000002FF2807D09B68214694F801229847A6
:10125000FF2384F80032002010BD032010BD00BF22
:1012600030B52B4C86462379E5889D4242D91846F5
:10127000043419461A4602E0954246D921780C44B6
:101280000A44617892B20529F6D1A1788229F3D176
:101290009C461A461F4903E0AA4234D291F800C086
:1012A0006144624491F801C092B2BCF1050FF3D1E0
:1012B00091F802C0BCF1010FEED1164A02E0A8423B
:1012C0001DD213781A44034492F801C098B2BCF1BD
:1012D000050FF4D19378812BF1D10CB11023A371B8
:1012E00019B10020022308714B711AB100210223A9
:1012F0001171537143230748AEF8003030BD00220E
:10130000002CEBD1ECE70021D7E70024C0E700BFB9
:10131000000000240400002430B52B4C86462379BD
:10132000E5889D4242D91846043419461A4602E01F
:10133000954246D921780C440A44617892B2052935
:10134000F6D1A1788229F3D19C461A461F4903E0C1
:10135000AA4234D291F800C06144624491F801C0BD
:1013600092B2BCF1050FF3D191F802C0BCF1010FAC
:10137000EED1164A02E0A8421DD213781A44034463
:1013800092F801C098B2BCF1050FF4D19378812B8B
:10139000F1D10CB11023A37119B100204023487181
:1013A0000B711AB100214023517113714323074877
:1013B000AEF8003030BD0022002CEBD1ECE700216C
:1013C000D7E70024C0E700BF000000240400002489
:1013D000A2E700BF03460A2201481A80704700BFF7
:1013E00048000024064B4FF0120C064AA3F11400EB
:1013F000526DA1F800C0022A18BF1846704700BFFE
:101400006800002400400058042301480B80704706
:101410007C0000242DE9F047046982B0C3681C40B9
:1014200046D0814688464FF0004501F1500701F152
:101430003806B4FA84F325FA03F21B3BD243144076
:10144000C9F81020B8F1000F5FD0042B2ED8DFE8C8
:1014500003F052483D320300D8F81030D9F82CA0E0
:1014600033B19B6823B11FFA8AF108F1080098474D
:10147000D8F8283033B19B6823B11FFA8AF108F1FC
:1014800020009847D8F8403033B19B6823B11FFA49
:101490008AF108F138009847D8F8583033B19B6882
:1014A00023B11FFA8AF108F150009847002CC0D1EF
:1014B00002B0BDE8F087D8F8103008F10800D9F87C
:1014C00034105B689847002CB3D1F1E7D8F8283086
:1014D00008F12000D9F838105B689847002CA8D193
:1014E000E6E7D8F840303046D9F83C105B689847BA
:1014F000002C9ED1DCE7D8F858303846D9F8401097
:101500005B689847002C94D1D2E7042B07D8DFE81A
:1015100003F01903140F0A00D9F83C300193019B22
:10152000002C86D1C4E7D9F82C300193019BF7E752
:10153000D9F834300193019BF2E7D9F838300193A0
:10154000019BEDE7D9F840300193019BE8E700BF2C
:101550000A49D1F8EC324A685BB1002AFCD0013A62
:1015600010B513F8014B4A60C1F8EC3212B12046B5
:1015700010BDFEE774F02EFF204610BD802E002423
:10158000F8B50E4E96F8A432012B00D1F8BD96F8AE
:10159000A432032BFAD10D461446D6F8F07208E0B7
:1015A00008F060FAD6F8F032241A0544DB1B322B1F
:1015B000ECD8002C21462846F2DCF8BD802E002411
:1015C000F8B590F848305D1C0344EDB280F84850FF
:1015D00083F8341090F8493053B1132D07D9002304
:1015E00080F84830104F97F8A432012B05D1F8BD90
:1015F00080F84830002DF5D1F8BD97F8A432032BC0
:10160000F5D1D7F8F06200F134042946204608F0FD
:1016100029FAD7F8F0322D1A04449B1B322BE6D856
:10162000002DF2D1F8BD00BF802E0024F8B50023B4
:1016300090F84850A0F8483005B9F8BD0D4F97F81C
:10164000A432012BF9D097F8A432032BF5D1D7F8A7
:10165000F06200F134042946204608F003FAD7F876
:10166000F0322D1A04449B1B322BE6D8002DF2D108
:10167000F8BD00BF802E00242DE9F0410121044671
:101680004FF4077087F064F8054600286CD0D4F852
:10169000D46204EB8606C6F8C002237CC4F8BC0200
:1016A000002B40D040230222812120467CF03EF8CE
:1016B000012140230222204621877CF037F84FF099
:1016C00001080823032282212046A4F878817CF0B7
:1016D0002DF8294B0027E364D6F8C432C5F804720C
:1016E0001B689847D5F80402C5F81472C5F818723B
:1016F00000283ED0227CD4F8C83222BBC3F88C220A
:101700004FF400749A7903F51E71C3F88402012A1C
:10171000A3F87882C3F8884223D018687CF084F953
:101720000020BDE8F08120464FF4007302228121A1
:101730007BF0FCFF01214FF4007302222046218739
:101740007BF0F4FFBBE79A79402403F51E71C3F8E0
:101750008C72012AC3F88402A3F87882C3F8884205
:10176000DBD1C3F89402D8E7D4F8D432B03344F8CC
:1017700023000220BDE8F08101001000F8B5D0F888
:10178000C85240F20112044695F894342A87012B7E
:101790003ED00126002728683246314685F89464F9
:1017A0007CF0D2FA27873A4631462868A5F8786255
:1017B00085F894647CF0C8FA4FF48173A4F87871CA
:1017C00032460221286885F89464A5F85C307CF0E4
:1017D000BBFA85F89474D4F8D432002504EB830363
:1017E000E564D3F8C0228AB1D3F8C4325B68984765
:1017F000D4F8D432B03354F8230086F007FCD4F880
:10180000D432B03344F82350C4F8BC520020F8BDA1
:1018100000224FF481710287A5F87832A0F8782170
:10182000A5F85C10D7E700BFD0F8D43200EB8303F3
:10183000F0B5002683B0D3F8C0728DF80560ADF81E
:1018400006605FB191F800C004460D461CF06002CE
:101850002FD0202A05D020467CF0ACF8032003B01E
:10186000F0BDCA884878002A42D01CF0800F00F0F2
:101870008380D3F8C43239469B689847EA880223AC
:101880004FF48071072AC4F8943228BF0722D4F895
:10189000C832C4E906225A629A79998203F1140186
:1018A000012A1F629E6200D11F6318687CF0BCF899
:1018B00022E04B780B2BCED801A252F823F000BFC8
:1018C000FD180408F91804085718040857180408E4
:1018D000571804085718040857180408571804081C
:1018E00057180408571804083D1904083319040848
:1018F000D3F8C4329B6898470020B0E790F89C3238
:10190000032BA8D10222D0F8C8320020C4F89422B8
:1019100003F11401C4E906220DF106049862C3E93B
:1019200008424FF480729A829A79012ABDD11C63D1
:10193000BBE790F89C32032BDED08CE790F89C320A
:10194000032B88D101220221D0F8C832C0F89412AA
:1019500003F11401C0E906220DF10500C3E90802F4
:101960004FF4807200209A829A799862012A9CD161
:101970000DF10500186398E7402A4FF0030387F83C
:10198000000228BF402287F80122C4F89432D4F81C
:10199000C832C4F85821C4F85C2103F51571C3F8A6
:1019A00064229A79C3F86072012AC3F86862A3F8C6
:1019B000546208BFC3F8707277E700BF70B5124D6C
:1019C000124A2B68A2FB03239B09013BB3F1807FE2
:1019D00001D3012070BD4FF0E0220D4900240F28F3
:1019E00053614FF0F003064681F823304FF00703B0
:1019F00094611361EDD801464FF0FF3074F024F983
:101A00002046C5F8806070BD00000024D34D6210F0
:101A100000ED00E03749024603688B4233D01831AD
:101A2000591AB1FA81F1490969BB3348834240D060
:101A30001830834240D01830834236D01830834269
:101A40003DD01830834240D0183083422CD000F56E
:101A50005670834237D029498B4233D018318B429C
:101A600036D018318B4236D018318B4236D01831EF
:101A70008B4236D018318B4236D018318B4236D05B
:101A800023F0FF0013E0DBB21D491E48103B10B4E9
:101A90001D4CA4FB03435DF8044B01EB131393F8B7
:101AA0002810C2E91601704716211848D1659065C3
:101AB000704710211348F9E716211248F6E706216E
:101AC0001248F3E706211248F0E710210F48EDE72E
:101AD00010210F48EAE716210D48E7E700210D48DD
:101AE000E4E706210B48E1E710210A48DEE716216A
:101AF0000848DBE710000240400002402804024092
:101B0000188C0C0800000240ABAAAAAA04000240EC
:101B10000004024004040240F0B50C46114602687D
:101B20008646936913F0100C72D04FF0000C10230E
:101B300038486546D36193699E065FD445B903680A
:101B40005B1AA3423DD893699F06F8D52023D36141
:101B50004CF0040C01209369D90552D54FF48071E3
:101B60005F054CF0010CD16104D54FF480614CF05D
:101B7000080CD1619D0504D54FF400734CF0020CA4
:101B8000D3619369990701D5002393629369DB07B9
:101B900003D4936943F001039361536820241E49E1
:101BA00001200B4000215360DEF844308EF84010D5
:101BB00043EA0C03CEF844308EF841408EF84210D0
:101BC000F0BD57689EF842309669DBB2360408D5FE
:101BD0007E0406D4202B04D0536843F48043536022
:101BE000016893699F06A6D403685B1A192BF8D97C
:101BF00093694FF0200C01259E069FD5002DA5D09E
:101C0000A6E75E05B1D49C05B6D40028B9D1F0BDD5
:101C10006046A0E7802E002400E800FE2DE9F04792
:101C200007689A46089EBB6931EA03030CBF01238B
:101C30000023934220D180460C461546DFF85C9085
:101C4000324651464046FFF767FF20BBD9F80030C7
:101C5000A3EB060CD44507D9BB6934EA03030CBFD8
:101C600001230023AB420AD0BB6934EA03030CBF53
:101C700001230023AB42E3D00020BDE8F087D8F871
:101C80004430202288F840001343C8F8443088F8D4
:101C9000412088F842000120BDE8F087802E002412
:101CA0000C4A136903F03803102B0DD0182B09D000
:101CB00063B913689B060BD513680748C3F3C103C8
:101CC000D8407047FFF790B8044870470448704701
:101CD00001487047004402580090D00300127A0077
:101CE00000093D00184A136903F03803102B10B5A2
:101CF00024D0182B09D01BBB13689B0622D5136870
:101D00001248C3F3C103D84001E0FFF76DF80E4954
:101D10000F4A8B698969C3F303230E4C01F00F014D
:101D200013440A4493F8301092F8303001F01F0247
:101D300003F01F03D0402060D84010BD0648E6E7FE
:101D40000648E4E70148E2E7004402580090D00367
:101D5000188C0C080000002400127A0000093D00D5
:101D6000474A70B4946A956AD66A15F47C3FC5F305
:101D70000533D16B5BD0C1F3CC01C6F3001604F080
:101D8000030407EE903A06FB01F1012CB8EEE77A66
:101D900006EE901AFAEEE96A03D0022C6AD0002C03
:101DA0004AD0DFED387A87EE876A936BC3F3080376
:101DB00007EE903AF7EE005AF8EEE77A77EEA67A59
:101DC00077EEA57A67EE867A2D4AB7EE006A936BB6
:101DD000C3F3462307EE103AB8EEC77A70BC37EE6D
:101DE000067AC7EE876AFCEEE66AC0ED006A936B7E
:101DF000C3F3064307EE103AB8EEC77A37EE067A19
:101E0000C7EE876AFCEEE66AC0ED016A936BC3F326
:101E1000066306EE903AF8EEE66A76EE866A87EE9C
:101E2000A67AFCEEC77A17EE903A8360704770BCD2
:101E3000C0E900338360704713689B061DD51468A2
:101E4000F7EE005A936B1049C4F3C102C3F30803C1
:101E5000D14007EE903A06EE101AF8EEE77AB8EEA7
:101E6000C66A77EEA66AC6EE077A36EEA57A67EE00
:101E7000877AA9E7DFED057A95E7DFED057A92E746
:101E8000004402580024744A0090D0030024F44A0D
:101E90000024744C474A70B4946A956AD66A15F067
:101EA0007C7FC5F30553516C5BD0C1F3CC01C6F305
:101EB000002604F0030407EE903A06FB01F1012C22
:101EC000B8EEE77A06EE901AFAEEE96A03D0022C31
:101ED0006AD0002C4AD0DFED387A87EE876A136C1F
:101EE000C3F3080307EE903AF7EE005AF8EEE77AEC
:101EF00077EEA67A77EEA57A67EE867A2D4AB7EE68
:101F0000006A136CC3F3462307EE103AB8EEC77AA3
:101F100070BC37EE067AC7EE876AFCEEE66AC0ED63
:101F2000006A136CC3F3064307EE103AB8EEC77AA3
:101F300037EE067AC7EE876AFCEEE66AC0ED016A04
:101F4000136CC3F3066306EE903AF8EEE66A76EE9B
:101F5000866A87EEA67AFCEEC77A17EE903A83601F
:101F6000704770BCC0E900338360704713689B06FC
:101F70001DD51468F7EE005A136C1049C4F3C10262
:101F8000C3F30803D14007EE903A06EE101AF8EEBC
:101F9000E77AB8EEC66A77EEA66AC6EE077A36EE3C
:101FA000A57A67EE877AA9E7DFED057A95E7DFED99
:101FB000057A92E7004402580024744A0090D00346
:101FC0000024F44A0024744C0269836870B5044606
:101FD00005681343C069626986B029681343AC4A37
:101FE00003430A40616A1343E2682B606B6823F481
:101FF00040531343A2696B60A64B9D4200F066817B
:10200000236AAE681A43A44B33401A43AA60EB6AB2
:1020100023F00F030B43EB62A04B9D4228D0A04B53
:102020009D421AD09F4B9D4217D09F4B9D4214D08A
:102030009E4B9D4211D09E4B9D4219D09D4B9D427F
:102040000BD09D4B9D4208D0012000234FF0011280
:102050006367A266A36706B070BD984B5B6D03F023
:102060000703052BF0D8DFE803F09F7F8A925F79A2
:10207000924B5B6D03F03803282BE5D801A252F890
:1020800023F000BF31220408492004084920040835
:10209000492004084920040849200408492004086C
:1020A000492004086921040849200408492004083B
:1020B000492004084920040849200408492004084C
:1020C000492004087F210408492004084920040805
:1020D000492004084920040849200408492004082C
:1020E000492004088F2104084920040849200408D5
:1020F000492004084920040849200408492004080C
:10210000492004082921040849200408492004081A
:1021100049200408492004084920040849200408EB
:10212000492004085D210408B0F5004F644853D0ED
:10213000644B626803EB4103B3F84030B0FBF3F04B
:1021400000EB52004FF6EF73B0FBF2F0A0F110027B
:102150009A423FF679AFE860002076E7B0F5004F8D
:102160003AD04FF40040E3E7B0F5004F2DD003A87C
:10217000FFF7F6FD04980028EED0616AD8E7B0F5C5
:10218000004F71D06846FFF785FE0198F3E7B0F580
:10219000004F5ED0494B1A68920639D51B684A48F1
:1021A000C3F3C103D840C3E7B0F5004F32D0FFF707
:1021B00099FD424A434BD269C2F30212134493F889
:1021C000303003F01F03D840D5E703A8FFF7C8FD60
:1021D00004980028C0D0616A3A4B626803EB41035F
:1021E0004FF6EF71B3F84030B0FBF3F0530803EB58
:1021F0004003B3FBF2F3A3F110028A423FF624AF8F
:1022000023F00F02C3F3420392B21343EB60A3E740
:102210002D488DE7FFF766FD284A2A4BD269C2F3A5
:102220000212134493F8303003F01F03D840D0E774
:10223000B0F5004F1DD0FFF755FD204A214BD26964
:10224000C2F30222134493F8303003F01F03D84046
:1022500091E71A4B1A68900640F1A5801B681A484E
:10226000C3F3C103D840B7E76846FFF713FE0198F0
:10227000AFE7FFF737FD114A124BD269C2F30222D2
:10228000134493F8303003F01F03D840A1E700BF98
:10229000F369FFCF000C0058FFF4FF11001001405C
:1022A0000044004000480040004C00400050004006
:1022B0000014014000780040007C004000440258B7
:1022C00000093D00188C0C080090D003A868374B1B
:1022D00003401343364AAB60EB6A23F00F030B4312
:1022E000EB62936D03F00703052B3FF6ADAEDFE81D
:1022F00003F0413C3303524F2D4B1A6895064CD4E2
:102300002C482D4B656803EB410305EB4501B3F801
:102310004020B0FBF2F399423FF696AEB3EB053F97
:102320003FF692AE002319467DF0ACFE2A46090224
:10233000030241EA1061680818184FF0000341F1E8
:1023400000017DF09FFE1D4BA0F540729A423FF6C2
:102350007BAE1B4BD860FFE66846FFF79BFD0198FC
:1023600000283FF4F9AE616ACBE703A8FFF7F8FC59
:102370000498F5E7FFF7B6FC0D4A0F4B126AC2F35B
:102380000212134493F8303003F01F03D840E7E7FC
:102390004FF40040B5E70B48B3E71B680548C3F3AB
:1023A000C103D840ADE7034816E700BFFFF4FF11B3
:1023B000004402580090D003188C0C08FFFC0F005A
:1023C000000C005800093D00474A70B4946A956AB1
:1023D000D66A15F47C7FC5F30513516B5BD0C1F34E
:1023E000CC0106F0010604F0030407EE903A06FB68
:1023F00001F1012CB8EEE77A06EE901AFAEEE96ADE
:102400004ED0022C6DD0002C4DD0DFED387A87EE07
:10241000876A136BC3F3080307EE903AF7EE005A8E
:10242000F8EEE77A77EEA67A77EEA57A67EE867A07
:102430002D4AB7EE006A136BC3F3462307EE103A3A
:10244000B8EEC77A70BC37EE067AC7EE876AFCEE44
:10245000E66AC0ED006A136BC3F3064307EE103A59
:10246000B8EEC77A37EE067AC7EE876AFCEEE66A00
:10247000C0ED016A136BC3F3066306EE903AF8EE03
:10248000E66A76EE866A87EEA67AFCEEC77A17EEE3
:10249000903A8360704770BCC0E900338360704736
:1024A000DFED137AB3E713689B06AED51468F7EE39
:1024B000005A136B0F49C4F3C102C3F30803D140A0
:1024C00007EE903A06EE101AF8EEE77AB8EEC66A12
:1024D00077EEA66AC6EE077A36EEA57A67EE877AB9
:1024E000A6E7DFED057A92E7004402580024744C19
:1024F0000024744A0090D0030024F44A344A13683C
:1025000030B423F08063334C1360256803E0236804
:102510005B1B022B54D813681B01F8D4936A05681F
:1025200023F47C3343EA053393628368C568013B37
:10253000013D5B022D049BB205F4FE052B4345686B
:10254000013DC5F308052B430569013D2D0605F046
:10255000FE452B439363D36A456923F0C0032B43A5
:10256000D362D36A856923F020032B43D362D36AF5
:1025700023F01003D362D36BC0696FF3CF0343EA38
:10258000C003D363D36A43F01003D362D36AD1B1DB
:1025900001290CBF43F4801343F40013D3620C4AA7
:1025A000136843F080631360216803E023685B1ABB
:1025B000022B05D813681B01F8D5002030BC7047EA
:1025C000032030BC704743F40023D362E7E700BF29
:1025D00000440258802E0024344A136830B423F09B
:1025E0008053334C1360256803E023685B1B022B88
:1025F00054D813689B00F8D4936A056823F07C7361
:1026000043EA055393628368C568013B013D5B0261
:102610002D049BB205F4FE052B434568013DC5F32F
:1026200008052B430569013D2D0605F0FE452B43AA
:102630001364D36A456923F440632B43D362D36A9E
:10264000856923F400732B43D362D36A23F4807328
:10265000D362536CC0696FF3CF0343EAC003536482
:10266000D36A43F48073D362D36AD1B101290CBF1A
:1026700043F4000343F08073D3620C4A136843F0C1
:1026800080531360216803E023685B1A022B05D88E
:1026900013689B00F8D5002030BC7047032030BC85
:1026A000704743F48003D362E7E700BF0044025859
:1026B000802E0024F0B5354AB0F1804F344DA0EBA8
:1026C00002020368A0EB050E4C69B2FA82F28F6831
:1026D000BEFA8EFE0E684FEA52124FEA5E1E1FD0FF
:1026E000F2B9DFF8B8C0604537D00CF5806C6045B2
:1026F00033D00CF5806C604512D0BEF1000F0FD1C5
:10270000244D254A904218BFA8422AD002F5806283
:10271000904226D023F08003C76286621C4314E0F7
:102720004D6823F07003D1F80CC02B43C76286625A
:1027300023F4407343EA0C0323F080031C4312B9D3
:10274000BEF1000F16D00B6903630368012243F04A
:102750000403036042610460F0BD23F070034A6823
:102760001343CA6823F44073C7621343866223F09D
:1027700080031C43074A084B984218BF9042E2D09E
:1027800003F580639842DED0DFE700BF0000014020
:1027900000040140004001400044014000040040AA
:1027A000026810B452E8003F23F4907342E800310D
:1027B0000029F7D1144C02F1080353E8003F2340ED
:1027C00002F1080C4CE800310029F4D1C36E012B52
:1027D00008D0002320225DF8044BC0F88C2043670A
:1027E000C366704752E8003F23F0100342E800310F
:1027F0000029EED052E8003F23F0100342E80031F8
:102800000029EFD1E5E700BFFEFFFFEF436BDA6978
:10281000F0B5970683B0044642D5586AE36AC0B261
:10282000002B00F09580216B9847636B1A681D465A
:1028300022F480721A609A6822F001029A609A6902
:1028400042F008029A61DA69D6072DD4DA69900756
:1028500001D502221A62DA69510701D504221A62EF
:10286000DA69120701D508221A62DA69170612D549
:10287000D4F8BC20212A0ED0D4E909128A4273D0A0
:10288000A169895C0132C9B299622169B2FBF1F098
:1028900001FB1022A262DA69560608D403B0F0BD2B
:1028A000DA691D46D607D1D501221A62CEE7DA6968
:1028B00040F60F0C1E6804F1340012EA0C0F996800
:1028C00036D0B24F0F4040F0BB80DFF8CCC216EAE2
:1028D0000C0F40F06381D4F8A050012D4CD0D502EC
:1028E00002D54F0200F16781150606D501F40001FB
:1028F00006F080050D4340F043815106CED57206A7
:10290000CCD553E8002F22F0400243E8002141B12A
:10291000626B52E8003F23F0400342E80031002997
:10292000F7D120220023C4F8BC20C4F8AC30B5E7AE
:102930009506D0D506F0200501F080573D43CAD05A
:10294000D4F8A830002BA9D003B0BDE8F040184758
:10295000E3696269D054E369E2680133B3FBF2F1E1
:1029600002FB1133E36160E70022A4F88A201A68B1
:1029700022F080021A608EE7D706B0D5F506AED5F4
:102980001022B4F890501A629A68570640F11D81DF
:10299000D4F8B40001684A6892B2002A00F050816D
:1029A000AA4280F04D81C169A4F89220B1F5807FE0
:1029B00040D053E8002F22F4807243E8002141B157
:1029C000626B52E8001F21F4807142E80015002D6F
:1029D000F7D103F1080252E8002F22F0010203F1BF
:1029E000080545E800210029F3D103F1080252E867
:1029F000002F22F0400203F1080545E800210029DC
:102A0000F3D12022C4F8C020C4F8A01053E8002F4E
:102A100022F0100243E80026002EF7D15C490D6831
:102A200040B190F83530022B00F01381802380F8FC
:102A3000346043650223C4F8A430B4F892302DE723
:102A400012F0010F0CD016F4807F09D04FF0010C6A
:102A5000C3F820C0D4F8C4C04CF0010CC4F8C4C002
:102A600012F0020F7BD112F0040F0CD011F0010F05
:102A700009D04FF0040CC3F820C0D4F8C4C04CF007
:102A8000020CC4F8C4C012F0080F0CD006F0200CE1
:102A90005CEA070C07D008271F62D4F8C47047F01F
:102AA0000807C4F8C47017050AD5770108D54FF494
:102AB00000671F62D4F8C43043F02003C4F8C43068
:102AC000D4F8C430002B3FF4E9AE92060CD506F0E2
:102AD000200601F080510E4306D0D4F8A8301BB177
:102AE00001909847656B0198D4F8C420AB6802F058
:102AF000280203F04003134361D0FFF751FEAB6897
:102B00005B067FF5CBAE05F1080353E8003F23F0E9
:102B1000400305F1080141E8003262B1626B02F145
:102B2000080353E8003F23F0400302F1080040E8A7
:102B300000310029F3D1D4F8B40000283FF4AEAE40
:102B400090F83520134B022A03653BD1FDF78EFA2E
:102B500000283FF4A3AED4F8B400036DF4E611F0FE
:102B6000010F90D04FF0020C12F0040FC3F820C0F8
:102B7000D4F8C4C04CF0040CC4F8C4C083D078E7C7
:102B8000D4F8AC30002B7FF4DFAE87E601000010F4
:102B9000802E00247D0F04082001000412F0010F94
:102BA0003FF471AF16F4807F7FF450AF12F0020F44
:102BB0007FF469AF57E74FF480121A626EE6C4F8EB
:102BC000C4306BE680224265BEE6B4F89220B4F8C9
:102BD000921092B289B2AA423FF460AE00293FF44B
:102BE0005DAE53E8002F22F4907243E8002141B11A
:102BF000626B52E8001F21F4907142E80010002837
:102C0000F7D1954803F1080252E8002F024003F182
:102C1000080545E800210029F4D12022C4F8A810B5
:102C2000C4F8C020C4F8A01053E8002F22F010020E
:102C300043E800210029F7D10223C4F8A4302DE68F
:102C4000AA427FF42BAEC369B3F5807F7FF426AE32
:102C5000F2E70368814A824E824FB34218BF934223
:102C600006F118060CBF01220022B34208BF42F051
:102C700001021836B34208BF42F001021836B342CF
:102C800008BF42F001021836B34208BF42F0010209
:102C900006F55676B34208BF42F001021836B34239
:102CA00008BF42F001021836B34208BF42F00102E9
:102CB0001836B34208BF42F001021836B34208BFCB
:102CC00042F001021836B34208BF42F00102183642
:102CD000B34208BF42F00102A6F59266BB4218BF9C
:102CE000B34207F592670CBF01260026BB4208BF1E
:102CF00042F0010256EA020779D0D3F800C02CF066
:102D00001E0CC3F800C0D3F814C02CF0800CC3F81C
:102D100014C0D0F860C076BBD0F860C0DCF80060AA
:102D200026F48076CCF800601A6822F001021A605E
:102D300003E00A68521B052A24D81A68D607F8D47B
:102D4000D0E9165101F01F012FB33F238B40AB6038
:102D5000C36ED0E91921516033B11A68016F22F4B2
:102D600080721A60436F4B600122002380F8352087
:102D700080F834305EE6DCF8002022F48072CCF873
:102D80000020D1E7202103220023416580F8343060
:102D900080F835204EE6344A344EB34218BF934291
:102DA00006F114060CBF01220022B34208BF42F014
:102DB00001021436B34208BF42F001021436B34296
:102DC00008BF42F001021436B34208BF42F00102CC
:102DD000012606FA01F1696025498B4208BF42F0DD
:102DE0000102002AB4D1234A9342B1D0BCE71E4E5F
:102DF000DFF878C0634518BFB3420CF1140C0CBF68
:102E000001260026634508BF46F001060CF1140CAC
:102E1000634508BF46F001060CF1140C634508BF7A
:102E200046F001060CF1140C634508BF46F001069C
:102E3000D3F800C02CF00E0CC3F800C0DFF830C08F
:102E4000634508BF46F00106002E7FF465AF094ECA
:102E5000B3423FF461AF67E7FEFFFFEF400002407F
:102E60005800024028000240085402581C540258DE
:102E700080540258945402584B4B10B41B684B4C6E
:102E8000A4FB03435B0A03FB02F25AB18446531EC0
:102E90004748DCF83420013B024201D0920406D5B9
:102EA0005C1CF6D14FF000405DF8044B7047DCF835
:102EB00034305C0741D4DCF83430D80709D43D4BBA
:102EC000CCF83830DCF81030DBB2994205D0012064
:102ED000EAE70123CCF83830F9E7DCF8143036485B
:102EE00018400028E0D0002B2CDB5A002DD49C0089
:102EF0002DD4D9002DD41A012ED45C012FD4D901A0
:102F000030D41A0231D45C0232D499023CD4DA02B1
:102F100037D45C0332D499032DD4DA0340D41C0493
:102F20003BD4590436D49A0431D413F0080F0CBFA3
:102F30004FF480304FF40000B6E704231846CCF875
:102F40003830B1E74FF00070AEE74020ACE78020AA
:102F5000AAE74FF48070A7E74FF40070A4E74FF49E
:102F60008060A1E74FF400609EE74FF480509BE73C
:102F70004FF4005098E74FF4802095E74FF400306D
:102F800092E74FF400408FE74FF480408CE74FF416
:102F9000800089E74FF4001086E74FF4801083E744
:102FA0004FF4002080E700BF00000024D34D6210E2
:102FB00045002000C500200008E0FFFD82B000238E
:102FC000019302E00369002B09DB019B01330193AC
:102FD000019BB3F1706FF5D9032002B070478901EE
:102FE000002341F020010193016103E0036913F024
:102FF000200307D0019B01330193019BB3F1706F54
:10300000F4D9E9E7184602B0704700BF82B0002348
:10301000019302E00369002B09DB019B013301935B
:10302000019BB3F1706FF5D9032002B07047002205
:1030300010230192036103E0036913F0100307D02A
:10304000019B01330193019BB3F1706FF4D9EBE75E
:10305000184602B0704700BF82B00023019302E01F
:103060000369002B09DB019B01330193019BB3F141
:10307000706FF5D9032002B07047002301930369F4
:1030800043F00103036103E0036913F0010307D078
:10309000019B01330193019BB3F1706FF4D9E9E710
:1030A0001846E8E72DE9F843056807460C46C5F3DE
:1030B0001009B9F1000F39D18A4B4FF6FF72B3F8FE
:1030C0008030934256D0002B54D0874A02EA4328DE
:1030D00008F10068454534BF4FF001084FF0020881
:1030E000824B9D4206D903F500339D4200F2CF800A
:1030F0004FF001097E4E96F80833012B12D00123C0
:10310000B8F1010F86F808334FF00003C6F80C330E
:1031100036D0022072F044FD002800F09980002390
:1031200086F808334FF0FF30BDE8F883704E96F80C
:103130000833012B4CD0012386F8083305F178437E
:10314000B3F5801F48D3A5F10163B3F5801F3FD2CB
:1031500000230220C6F80C3372F022FD002870D143
:10316000644A4FF00208D2F80C3143EA0803C2F86F
:103170000C313FE0B5F1016F67D3052011F0E0F8A5
:10318000404672F00DFD0028C9D14046DFF8648149
:10319000D8F80C3023F4E663C8F80C30D8F80C30BB
:1031A00043EA092343F0A403C8F80C3072F0F8FC9A
:1031B000D8F80C20504B1340C8F80C300028AED182
:1031C00005F178430122B3F5801F86F8082303D365
:1031D0006FF00100BDE8F88300230120C6F80C332E
:1031E00072F0DEFC68BB434A4FF00108D36843F03D
:1031F0000203D360BFF36F8FBFF34F8F04F1200240
:1032000054F8043B944245F8043BF9D1BFF36F8F67
:10321000BFF34F8F404672F0C3FCB8F1010F354A3F
:1032200030D0D2F80C3123F00203C2F80C31002365
:1032300086F808330028CBD13B6820333B60BDE8DB
:10324000F883002386F80833C2E74FF0010847E708
:10325000DFF8A0800220D8F80C3123F4E663C8F828
:103260000C31D8F80C3143EA092343F0A403C8F821
:103270000C3172F095FCD8F80C211F4B1340C8F8A4
:103280000C319BE7D36823F00203D360CFE703F54B
:1032900000339D4211D903F500339D4210D903F547
:1032A00000339D4206D903F500339D420BD84FF001
:1032B00005091FE74FF004091CE74FF0020919E761
:1032C0004FF0030916E703F500339D4206D9B5F127
:1032D000016FBFF452AF4FF007090BE74FF006093B
:1032E00008E700BF00E8F11F00FE1F00FFFF010814
:1032F000802E002400200052FBF8FFFF0148FDF75C
:10330000B1B800BF94310024084810B4D0F8143389
:10331000D0F8484399691A682CB1234600F54570E6
:103320005DF8044B18475DF8044B7047802E00246D
:103330000148FDF797B800BFEC310024084810B4ED
:10334000D0F86C33D0F8A04399691A682CB12346A1
:1033500000F55B705DF8044B18475DF8044B70474F
:10336000802E00240148FDF77DB800BF44320024C0
:10337000084810B4D0F8C433D0F8F84399691A68F3
:103380002CB1234600F571705DF8044B18475DF8C9
:10339000044B7047802E00242DE9F04FDFF85C933A
:1033A00000EB400583B0430009EB85050093D5F899
:1033B00084300193002B00F05E818046B5F88A00CE
:1033C00071F0D6FE95F8880008F0C4FA044695F826
:1033D000890008F0BFFA08F101030746DBB2002CB0
:1033E00000F06E8140F60C12A1882372E280226800
:1033F000002800F05981037240F60C23C3809161CC
:103400003B68BA889A6111212046092608F0CAFA59
:103410001121384608F0C6FA6525002C00F02E81EF
:103420002268A38811690B4200F028811B04936174
:1034300010F02AFF05468B4610F026FF401B61EB7B
:103440000B01052871F10001F6D314B12368A2889D
:103450009A6110F019FF05468B4610F015FF401BCE
:1034600061EB0B01052871F10001F6D3013ED3D1C8
:103470001CB1A38822681B04936110F005FF054668
:103480000E4610F001FF401B61EB0601052871F1AB
:103490000001F6D31FB1BB883A681B04936110F09A
:1034A000F3FE05460E4610F0EFFE401B61EB0601F1
:1034B000052871F10001F6D314B12368A2889A613E
:1034C00010F0E2FE05460E4610F0DEFE401B61EBFA
:1034D0000601052871F10001F6D317B13B68BA88DF
:1034E0009A61009B20463E21434409EB830393F8F5
:1034F0008F4022460DF022F8224638463E210DF03C
:103500001DF8784C5823019A03FB0843C3F8142391
:10351000754B9A4200F0C380FEF7E4FB734BDA6907
:10352000C2F30212724B134493F8303003F01F03BE
:10353000D840009B434409EB830393F88C30022B63
:1035400000F0B980032B00F0B180012B14BF4FF4C1
:10355000C8714FF4487171F03DFF034658220021B5
:1035600002FB0842C2F81C13C2F81833C2E9C911A1
:10357000C2E9CC110121C2F8201392F8551301F0D1
:10358000FF00002900F0A480582123F07062242657
:103590004FF4004701FB08415648D1F8143381F835
:1035A00055631D6825F001051D601A619A6822F4B3
:1035B00000429A609F605A6822F400625A605A681A
:1035C0001043D1F82C2358601202D86820F4004030
:1035D000D860DA6000221A60186840F001001860B4
:1035E0002020C1F8582381F85503C1F8442381F8FD
:1035F000562391F855032028C5B217D191F85403EA
:10360000012813D081F85563186820F00100186074
:10361000186820F48050186018681860186840F026
:103620000100186081F8555381F85423009B022152
:103630000126314F434409EB830999F88E502846FF
:1036400072F002FB05F01F036A0999F88D5006FA23
:1036500003F30221284647F8223072F0F5FA582386
:1036600003FB084405F01F036D0906FA03F347F84E
:10367000253084F8106303B0BDE8F08F013D2AD0F7
:1036800010F002FE83468A4610F0FEFDB0EB0B0000
:1036900061EB0A01052871F10001F5D3BDE6FEF7E3
:1036A00021FB124B1A6A3BE79161ACE6C82171F02D
:1036B00091FE034652E7642171F08CFE03464DE70C
:1036C00000283FF4A0AE037240F60C23C38097E6B7
:1036D00082F8540358E7002C3FF4AAAEA38822686E
:1036E000A4E600BF802E0024001C005800440258AD
:1036F000188C0C080080000200E100E000000024AB
:103700002DE9F04F441C85B017469DF83C202DD084
:103710005824DFF8A8831E46054600FB04F408EB96
:10372000040393F81093B9F1000F1FD044444900EB
:10373000FF2F04F54574039100D0EEB9002A40F044
:10374000C680582303FB058393F85523202A04D110
:10375000B6B94FF40072C3F85823B8F818342846A5
:1037600001339BB2A8F81834FFF716FE4FF000099A
:10377000484605B0BDE8F08F93F85533202BECD1C7
:103780004FF0580A0AFB058A9AF85433012BE4D00B
:103790000122D8F800B019234FF400418AF85423CD
:1037A0002046CDF800B0FEF739FA0028D5D10E9B9F
:1037B000DAF81413CAF838332123BA4A8AF8553391
:1037C0004023CAF848038AF85633CAF858032046FB
:1037D000AAF83E634B681340039A1343B24A1A4354
:1037E0004A60594672F0AEF90246002840F0FB806C
:1037F000DAF81433802120469F620A23CDF800B006
:10380000FEF70CFA002840F0EE80BAF83E339BB287
:10381000FF2B40F21681DAF81413FF23A348AAF80D
:103820003C334B68A24A0340039803431A434A605F
:103830005826DDF80CA05F46039506FB058605E0DB
:10384000B6F83E339BB2002B00F01081394620467B
:1038500072F078F9002840F0F280D6F83813D6F8E4
:10386000145311F8012BB6F83C33AA62C6F838138A
:10387000013BB6F83E139BB20139A6F83C3389B23E
:10388000A6F83E13B6F83E1389B2002BD8D1002912
:10389000D6D002460A23802120460097FEF7BEF9C3
:1038A000FF22002840F0CB80B6F83E339BB2934213
:1038B00040F2A080D6F81413A6F83C234B687B4A4C
:1038C00013407B4A43EA0A031A434A60B8E74FF0C1
:1038D000580A0AFB058A9AF85533202B7FF43DAF2E
:1038E0009AF85433012B3FF438AF0122D8F8007016
:1038F00019234FF400418AF8542320460097FEF71D
:103900008DF900287FF429AF0E9BCAF84803CAF846
:10391000383321238AF8553310238AF85633CAF8EE
:103920005803AAF83E63BAF83E339BB2FF2B00F26D
:10393000C780BAF83E339BB2AAF83C33002B40F064
:10394000F180DAF8141357484B685A4A0340039839
:1039500003431A434A605826AA4606FB0586B6F872
:103960003E3339469BB2002B00F0D480204672F0E3
:10397000E9F8002878D1D6F83813D6F8145311F89E
:10398000012BB6F83C33AA62C6F83813013BB6F8EF
:103990003E139BB20139A6F83C3389B2A6F83E1318
:1039A000B6F83E1389B2002BD9D10029D7D00246F0
:1039B0000A23802120460097FEF730F9FF220028D5
:1039C00052D1B6F83E339BB2934225D9D6F81413A0
:1039D000A6F83C234B68354A1340039A1343344AF4
:1039E0001A434A60BBE75823002203FB058383F890
:1039F0005423B2E6B6F83E33D6F814239BB22B48D4
:103A00005168A6F83C33DBB201404AEA03430B435A
:103A100043F00073536013E7B6F83E33D6F814133F
:103A20009BB2039A2148A6F83C33DBB242EA034337
:103A30004A680240134343F000734B608FE7039DD5
:103A40008BE6BAF83E33DAF814139BB2039A1748A0
:103A5000AAF83C33DBB242EA03434A68024013430C
:103A600043F000734B60E3E6554676E63946204660
:103A7000039D72F039F800287FF46FAED6F8143346
:103A800020210D4CD9615A6822405A6058230022E7
:103A900086F8551303FB058386F8560383F85423F1
:103AA00066E600BF009800FC00200101009C00FCBD
:103AB0000000FF010020000200E800FE802E00242C
:103AC000FF234FF47F00FE224FF08076AAF83C33AC
:103AD000039BDDF838E01E4358231EF801AB03FBBF
:103AE0000583DFF850C0D3F81413C1F828A0A3F859
:103AF0003C23B3F83E23C3F838E3013A92B2A3F86B
:103B00003E234B6803EA0C033343034343F400535F
:103B10004B6020E72046554671F0E6FF00287FF411
:103B20001CAEABE7013B4FF000769AB2501CC0B21E
:103B30000004CDE7009800FC2DE9F04F441C85B04F
:103B400099469DF83C3000F096805825C34C0646B7
:103B500000FB05F504EB050B9BF810A3BAF1000F71
:103B600000F089802544FF2A90464FEA410705F579
:103B7000457540F08680002B00F083809BF855331C
:103B8000202B6FD19BF85433012B6BD00122D4F83A
:103B9000008019234FF400418BF854232846CDF8B8
:103BA0000080FEF73BF800285CD10E9BCBF8480361
:103BB000CBF8383322238BF8553310238BF8563348
:103BC000CBF85803ABF83E93BBF83E339BB2FF2BC8
:103BD00000F21081BBF83E33DBF814139BB2A0480F
:103BE0004A68ABF83C33DBB2024047EA0343134375
:103BF0009C4A1A434A604FF0580909FB0649B9F834
:103C00003E339BB2002B00F08481D9F814339A69BB
:103C1000520700F1318142460A212846FDF77CFF18
:103C2000002840F0F480D9F814339A69910640F1E5
:103C3000F9809A699A6912F0100200F0F18010225E
:103C40002021894DDA610422C9F85823D9615A68C4
:103C50002A405A6089F8551389F8540389F85603A5
:103C600022689B69B4F81834304601339BB2A4F83B
:103C70001834FFF791FB4FF0000A504605B0BDE83D
:103C8000F08F4FF0580B0BFB064B9BF85533202B56
:103C9000E8D10E9B002B00F0A8809BF85433012B39
:103CA000E0D0236801224FF4004128468BF85423CA
:103CB000039300931923FDF7B1FF0028D2D12223EB
:103CC000DBF814130E9A8BF855334023CBF83823C6
:103CD0008BF85633CBF85803ABF83E93DFF880915E
:103CE0004A68CBF84803284602EA09023A4342F4FC
:103CF00090324A60039971F025FF0246002840F097
:103D00003481402328461946DBF81433C3F8288051
:103D1000039B00930A23FDF781FF002840F02581D3
:103D2000BBF83E339BB2FF2B40F22681DBF8141325
:103D3000FF234E4AABF83C334B6803EA09033B438D
:103D40001A434A604FF05808B946039F08FB0648DB
:103D500005E0B8F83E339BB2002B00F01F810A2328
:103D60000022042128460097FDF758FF00287FF421
:103D700079AFD8F81433596AD8F838331970B8F8CD
:103D80003E13D8F838330139013389B2C8F83833D3
:103D9000B8F83C33A8F83E13013BB8F83E139BB289
:103DA00089B2A8F83C330029D3D0002BD1D10246E8
:103DB0000A23802128460097FDF730FFFF220028C4
:103DC0007FF450AFB8F83E339BB2934240F2BB80D1
:103DD000D8F81413A8F83C234B68254A1340254A09
:103DE00043EA09031A434A60B3E74FF40073CBF880
:103DF000583337E7DBF81413FF231948ABF83C338B
:103E00004B681A4A03403B431A434A60F3E658237F
:103E100003FB0643D3F814339A6922689B6921E7B0
:103E2000C9F858232268A2EB08020A2A7FF6EFAEEF
:103E30009A6912F004027FF4EAAE582101FB0641B0
:103E4000D1F8580381F85423202240F02000C1F813
:103E5000580381F855239B6904E700BF802E002496
:103E6000009800FC0024000200E800FE0024FF018E
:103E7000009C00FC0000FF015A6AD9F838331A7020
:103E8000B9F83E33D9F83823013B01329BB2C9F867
:103E90003823A9F83E33B9F83C33B9F83E23013B47
:103EA00092B29BB2A9F83C33002A3FF4A8AE002B93
:103EB0007FF4A5AE0A23002280212846CDF8008099
:103EC000FDF7ACFE00287FF4CDAEB9F83E339BB2CF
:103ED000FF2B0CD9D9F81413FF233B48A9F83C3326
:103EE0004B683A4A03403B431A434A6087E6B9F8B5
:103EF0003E33D9F814139BB233484A68A9F83C33CF
:103F0000DBB2024047EA0343134343F000734B60C4
:103F100075E64146284671F0E7FD00287FF4A2AE21
:103F2000D9F8143320212A4DD9615A682A405A60A1
:103F300089F8551389F856035822002302FB0644DA
:103F400084F8543399E6B8F83E33D8F814239BB27A
:103F50001D485168A8F83C33DBB2014049EA0343ED
:103F60000B4343F000735360F3E65823002203FB36
:103F7000064383F8542375E6BBF83E33DBF814138D
:103F80009BB24A68ABF83C33DBB202EA090247EA6B
:103F9000034313430F4A1A434A60D3E60399284662
:103FA00071F0A2FD034600287FF45CAED8F814231C
:103FB0002020074DD06151682940516088F8550391
:103FC00088F85633B8E700BF009C00FC0000FF01F2
:103FD00000E800FE002400020348D0F8B4300BB122
:103FE000A8301847704700BF000000240348D0F8ED
:103FF000D4300BB1C8301847704700BF0000002410
:104000000348D0F8F4300BB1E8301847704700BFD0
:10401000000000240348D0F8143113B100F5847077
:1040200018477047000000240348D0F8343113B11A
:1040300000F5947018477047000000240348D0F83A
:10404000543113B100F5A4701847704700000024E4
:104050000348D0F8743113B100F5B47018477047B5
:10406000000000240348D0F8943113B100F5C47067
:1040700018477047000000240348D0F8B43113B14A
:1040800000F5D47018477047000000240348D0F8AA
:10409000D43113B100F5E4701847704700000024D4
:1040A0000348D0F8F43113B100F5F47018477047A5
:1040B000000000240348D0F8143213B100F5027058
:1040C00018477047000000240348D0F8343213B179
:1040D00000F50A7018477047000000240348D0F824
:1040E000543213B100F512701847704700000024D5
:1040F0000348D0F8743213B100F51A7018477047AE
:10410000000000240348D0F8943213B100F5227067
:10411000184770470000002410B41C4643688446CA
:104120006FF30F0323434360036843F0010303600D
:10413000036843F400730360002C3AD040F2E93086
:10414000DCF814309B0748D5002A49D012F8013B0F
:1041500040F2E9308CF82030DCF81430DB0720D452
:104160000138F9D1214B9C450CD0A3F578439C45EF
:1041700038D003F580639C4536D003F578439C45E1
:104180000BD103201A4A00EB400002EBC002B2F848
:10419000BC3201339BB2A2F8BC3200205DF8044B64
:1041A00070479CF83000C0B209B101F8010B013C26
:1041B000C4D1DCF814301B07FBD5DCF81830012023
:1041C0005DF8044B43F01003CCF81830DCF80030F5
:1041D00023F00103CCF8003070470138B0D1C1E7BB
:1041E000FF23B5E70120CDE70220CBE700300140F7
:1041F000000000242DE9F84300242C4E804603687B
:1042000056F83450AB4209D001340E2CF8D1284A6C
:104210000021052009F02EFA002019E0254B03EBC0
:104220008409D9F81C74AFB198F8051000204B1C14
:1042300001EB410203EB430307EBC202DB00C2F8D0
:104240000C80C2E90400F854182303FB0170083005
:10425000BDE8F8830721682009F092FA0146C9F801
:104260001C04F0B13946682283F0A8FAD9F81C146E
:1042700006EBC4043B4689600C60096289630965EA
:1042800056F83320954205D001330E2BF8D14F60FC
:104290000F46C9E7084F4C2202FB03774F600F46D9
:1042A000C2E7064A052009F0E5F9B5E7708C0C086D
:1042B000E0350D08802E0024D432002408360D0885
:1042C000B0B1022330B4D0E900428D6864685279FD
:1042D00003FA02F223684C685CB1DC6885B12243C2
:1042E0008160DA60DA6842F00102DA6030BC70475F
:1042F0007047DC6824EA0202DA604DB18160F1E7C0
:1043000024F00104DC60DC6881602243DA60EDE7C0
:10431000DA6822F00102DA608160E7E7F0B544680C
:10432000A37913F002025FD002224FF0080C036859
:1043300064795B689B48204493F83C40012C90F8DA
:10434000C80050D0012483F83C40142848D8DFE846
:1043500010F0150047004700470084004700470061
:1043600047003B01470047004700BB0047004700AC
:104370004700F2004700470047004D0018688A4C8C
:10438000056A8A4E25F00205B04242EA0502056A36
:1043900025F0010505624768856904EA050444F0D3
:1043A000600407D0824DA84204D005F57055A8429C
:1043B00040F04D8122F0080247F440774CEA0202B7
:1043C00022F004024760846141630262826942F024
:1043D00008028261826922F004028261826982613C
:1043E000002283F83C20F0BD9446A0E718686F4E89
:1043F000046AB04224F4001444EA0252046A24F429
:10440000801404626B4C4568476D04EA070444F469
:10441000C0440ED006F58066B0420AD0664F06F55D
:104420008046B04218BFB84203D006F58066B0425D
:1044300001D145F4802545604465C1650262426D45
:1044400042F400624265426D22F480624265426D30
:104450004265002283F83C20C5E71868574C056A7E
:10446000524E25F02005B04245EA0215026A22F0BC
:10447000100202624768826904EA020444F4C044FC
:1044800000F0DE804A4A904200F0DA804A4E4C4A00
:10449000904218BFB04203D002F58062904201D131
:1044A00047F440674760846181630562826942F432
:1044B00000628261826922F4806282618269826123
:1044C000002283F83C208EE71868384E046AB04218
:1044D00024F4005444EA0232046A24F4805404624E
:1044E000364C4568C76904EA070444F4C0440ED05A
:1044F00006F58066B0420AD02F4F06F58046B042DE
:1045000018BFB84203D006F58066B04201D145F429
:1045100080454560C46101640262C26942F4006280
:10452000C261C26922F48062C261C269C2610022B2
:1045300083F83C2057E718681C4E046AB04224F404
:10454000003444EA0242046A24F4803404621D4CBC
:104550004568476D04EA070444F060040ED006F590
:104560008066B0420AD0144F06F58046B04218BFAC
:10457000B84203D006F58066B04201D145F48035DB
:104580004560446581650262426D42F00802426501
:10459000426D22F004024265426D4265002283F8BA
:1045A0003C2020E7188C0C088CFFFEFF0000014027
:1045B00000040140FF8FFFFE00400140FF8CFFFE22
:1045C000004401408FFFFEFF1868264C056A264E06
:1045D00025F4007EB0424EEA0225026A22F480727F
:1045E00002624768C26904EA020444F0600420D011
:1045F0001E4A90421DD01E4E1E4A904218BFB04225
:1046000003D002F58062904201D147F440574760E1
:10461000C461C1630562C26942F00802C261C26935
:1046200022F00402C261C269C261002283F83C2008
:10463000D9E625F4006E4EEA0C2E2EF48065E4E7F0
:1046400025F0800545EA0C1525F0400528E705F51D
:104650008065A8423FF4AEAE05F58065A8427FF4C0
:10466000B1AEA7E68CFFFEFF000001400004014050
:10467000004001400044014042685379032B0FD8A9
:10468000DFE803F00B08050210684030704710683F
:104690003C307047106838307047106834307047CD
:1046A00000207047D0E90002064B517992790B4403
:1046B000406893F8C810530701D579F003BC79F02E
:1046C0007DBC00BF188C0C08F0B54468374A2469DB
:1046D000C368C4F303245B6852F82460EFF31184C9
:1046E000102585F312884568314F95F805E0D0F81C
:1046F0000CC002EB4E02D5F800E0158CDEF80C2061
:1047000005F4F05522EA0502CEF80C2017F806E071
:10471000DCF8102053F80E501F2A25F0010543F84D
:104720000E5039D9203A2025DCF804C005FA02F2EF
:10473000CCF80C20E2B282F31188BA5DDFF874C0C5
:1047400003EB020E46684569DEF8044004EA0C0CEF
:104750004CEA0101CEF804107179032924D8DFE86E
:1047600001F01815120231684031CEF80C500124C6
:10477000CEF80810995841F01001995099582143EA
:1047800099500474F0BD31683C31EEE7316838313E
:10479000EBE731683431E8E72025DCF804C005FA9E
:1047A00002F2CCF80820C5E70021DEE7188C0C08DF
:1047B000888D0C080000FFFF03681A7E012A2ED0A6
:1047C000002293F83010012909D093F848100129EC
:1047D0000ED093F8601001291BD02ABB704702212C
:1047E00042F4806283F8301093F84810012904D114
:1047F000022142F4006283F8481093F86010012906
:1048000007D01B6800211B685962D9680A43DA6027
:104810007047022142F4805283F86010F1E70221D0
:104820004FF400721976CCE74FF40072E9E700BF4D
:1048300008B5204B98420ED003F5806398420AD009
:104840001D4A03F58043984218BF904203D003F5F8
:10485000806398421BD1FDF745FA1849184BCA6985
:10486000C969C2F30222C1F302211A4492F830202E
:1048700002F01F02D040114A1269C2F3C03241EA6D
:10488000C202134493F8CC3003FB00F008BDFDF7DF
:1048900029FA0A490A4BCA69C969C2F3021CC1F361
:1048A000021103EB0C0292F8302002F01F02D040FC
:1048B000E1E700BF00000140004001400044025811
:1048C000188C0C0870B50E4605EE102AD0E90031A0
:1048D000013E1A680868B6B25C681568FFF7A8FF61
:1048E00007EE900AB8EE455A9FED5D7AF8EE677ACA
:1048F00087EE850A30EE070A7EF04CFA236801380D
:10490000AB4280B268D0C4E9005000238022E66048
:10491000A360A261C4E9043394F83D3003F0FF02C0
:10492000002B78D00223211D284684F83D30FDF766
:10493000C1FE4C4A0123B5F1804FA5EB020284F879
:104940004830B2FA82F284F83E3084F83F304FEAC1
:10495000521284F8403084F8413084F8423084F8B0
:10496000433084F8443084F8453084F8463084F885
:10497000473084F83D3034D09ABB3B4B9D420CD03D
:1049800003F580639D4208D003F580639D4245D0C6
:1049900003F578439D4241D070BD94F83C30012B23
:1049A000FAD00222314B012184F83D20A86803404F
:1049B000AB6084F83D1084F83D206B68A96823F053
:1049C000700321F0800101226B600023A96084F84C
:1049D0003D2084F83C3070BD636883423AD060600B
:1049E00093E794F83C30012BD6D002211F4B0020D6
:1049F00084F83D10A9680B400121AB6084F83D109C
:104A0000022384F83D306B68A9680AB90028D6D023
:104A100023F47003D3E784F83C2083E794F83C3018
:104A2000012BB9D00221114B114884F83D10A9681F
:104A3000281A0B40B0FA80F00121AB600023400936
:104A400084F83D1084F83C300A4B9D42D8D00028B1
:104A5000D6D170BDE368B3427FF457AF70BD00BFDD
:104A60000AD7233C00000140000400408800CEFF2C
:104A700000040140000C0040024B0348D3F81C1412
:104A8000FCF7C8BC802E002400000140034B4FF00F
:104A90008040D3F82014FCF7BDBC00BF802E00245A
:104AA000024B0348D3F82414FCF7B4BC802E002436
:104AB00000040040024B0348D3F82814FCF7AABCBA
:104AC000802E002400080040024B0348D3F82C1429
:104AD000FCF7A0BC802E0024000C0040024B0348D1
:104AE000D3F83814FCF796BC802E00240004014053
:104AF000024B0348D3F84814FCF78CBC802E0024EA
:104B000000180040024B0348D3F85414FCF782BC51
:104B1000802E002400400140024B0348D3F8581473
:104B2000FCF778BC802E002400440140024B03486F
:104B3000D3F85C14FCF76EBC802E002400480140C2
:104B400010B5064C0648D4F83814FCF763FCD4F8CA
:104B50004C140448BDE81040FCF75CBC802E0024D7
:104B600000040140001C004010B5064C0648D4F873
:104B70003814FCF74FFCD4F850140448BDE810403A
:104B8000FCF748BC802E00240004014000200040B7
:104B9000BFF34F8F0549064BCA6802F4E062134326
:104BA000CB60BFF34F8F00BFFDE700BF00ED00E01B
:104BB0000400FA050021012008B50DF061FF72B66E
:104BC000FFF7E6FF2DE9F043BFB0BFF35F8FA14CC5
:104BD0000023626A22F480326262C4F894309DF845
:104BE00043109DF844C009069DF842200F9841EA01
:104BF0000C7141EAC2419DF8452041EA82419DF88D
:104C0000462041EA42419DF8472041EA02419DF891
:104C1000412041EA02219DF8402041EA4201C4F8C6
:104C200098300133D4F8A020112B22F00102C4F8EF
:104C3000A020C4F89C00C4F8A010F0D10523C4F84B
:104C40009430636A43F480336362BFF34F8FBFF3E2
:104C50006F8F8148814A8249121A80F031FD814B61
:104C60005A6D012A00F0DF80D4F8881000227E4BB4
:104C7000012041F47001C4F8881018601A611968A5
:104C800041F080011960196801431960196841F405
:104C900080311960196841F4805119609A61DA61B4
:104CA0001A629A62DA621A635A639A63DA631A645E
:104CB0005A64196821F4802119601A664FF0006364
:104CC0006A49C1F80801A3607AF090FA684AD3688B
:104CD00013F0040FD36840F09480664B0021644ABF
:104CE0000591D96A21F00101D962DB6A03F0010361
:104CF0000593936943F440439361936903F44043FC
:104D00000593059B93699E04FCD54C2200210EA8B7
:104D1000594C82F053FD594A42F20303A4F11001A9
:104D20001268B3EB124F4FF000024FF0040308BFBC
:104D30000C460892E268A370002A4FD04D4BD96A06
:104D400021F00101D962DB6A494903F001030893AC
:104D50008B6923F4404313438B618B6903F4404315
:104D60000893089B424A93699D04FCD53E4B4FF43F
:104D7000403543480321D3F8E02042F08002C3F8D5
:104D8000E0200122D3F8E03003F080030793079B73
:104D900085610D9BCDE9001300237AF0D5F802233D
:104DA00001204FF48031A288CDE9173304231993F1
:104DB000A379CDE90E01E079217A1C900EA81D910E
:104DC000CDE91A2308220023CDE91E23FBF74AFD73
:104DD000032800F06082002858D0FEE7244A254BC3
:104DE000916941F440419161926902F44042089214
:104DF000DA6A42F00102DA62DB6A03F00103089327
:104E0000AFE723F007031F4C43F00203D360216890
:104E100005E023685B1AB3F57A7F3FF65EAF53680F
:104E20009F04F6D559E7104A002017495865D2F873
:104E3000F43043F00203C2F8F430D2F8F43003F057
:104E400002030E930E9B0B6883F308884B68984708
:104E5000FEE700BF00ED00E000000000D0370000DA
:104E600038B60D0800400058004402580080005138
:104E70000048025800040058180300240010005C89
:104E8000001C0258802E00240098F01F754B1A68F1
:104E900012F00E0F0BD11A6822F00F0242F002023C
:104EA0001A601B6803F00F03022B40F0F6816E4A74
:104EB000936903F070033F2B05D8936923F07003C7
:104EC00043F040039361684AD36903F070033F2BBA
:104ED00005D8D36923F0700343F04003D361624ADD
:104EE000D36903F4E063B3F5806F05D2D36923F48B
:104EF000E06343F48063D3615B4A136A03F0700399
:104F00003F2B05D8136A23F0700343F0400313626C
:104F1000554B9A69140705D49A6922F00F0242F0A2
:104F200008029A61504A936923F47063936113688D
:104F3000980130D5136941F288314C4C23F00703B6
:104F400043F003031361206804E023681B1A8B42BB
:104F500000F2AC81136903F03803182BF5D1936983
:104F600003F00F03082B05D9936923F00F0343F0D7
:104F7000080393613B4A136803F00F03022B0BD91C
:104F8000136823F00F0343F002031360136803F068
:104F90000F03022B00D0FEE7334A936903F070033E
:104FA000402B05D9936923F0700343F040039361CC
:104FB0002D4AD36903F07003402B05D9D36923F040
:104FC000700343F04003D361274AD36903F4E063DD
:104FD000B3F5806F05D9D36923F4E06343F48063AC
:104FE000D361214A136A03F07003402B00F256810B
:104FF0001D4EFCF755FE1E4DB269B369C2F3032284
:105000001C4B134493F8303003F01F0320FA03F3D2
:10501000D5F880002B60FCF7D1FC002840F08D8192
:105020001023159017900EA80E93FBF71BFC002879
:1050300040F030813368104A43F080033360D6F883
:10504000F43043F00203C6F8F430D6F8F43003F03D
:1050500002030493049B136A43F001031362074B9A
:10506000216810E00020005200440258802E0024E5
:1050700000000024188C0C0800040058803801003F
:10508000013B00F0088122689142F9D02268236830
:105090009B1A0A2BFBD900214FF48020A74C4FF418
:1050A00040130026002730934FF00208CDE90E018F
:1050B0000EA879F06FF8D4F8EC30A14941F2030260
:1050C00043F002030EA8C4F8EC30D4F8EC3003F03F
:1050D00002030393039BD4F8943043F00203C4F813
:1050E0009430D4F8943023F00203C4F894300B6861
:1050F0009449B2EB134F944B944A28BF0A465A6026
:105100001A6822F47C5242F400521A601A6842F083
:1051100060021A6003220023CDE92C67CDE90E233B
:1051200079F038F84FF4E04200230EA8CDE9266765
:1051300000270326CDE90E233A9779F02BF81822A1
:1051400000230EA82F973497CDE90E2379F022F88B
:105150004FF4803200230EA81797CDE90E230522C5
:105160004FF4FA73CDE91023042314934FF48033E2
:10517000CDE915772293CDE9128679F00BF8D4F8B2
:10518000E03042464FF4807143F001037048C4F8A8
:10519000E030D4F8E03003F001030993099B3B466B
:1051A000CDE9006779F0D0FE23694246694823F0D3
:1051B000FE7343F088732361D4F8E03043F00403B6
:1051C000C4F8E030D4F8E03003F0040306933B4623
:1051D00006994FF40071CDE9006779F0B5FE2369B7
:1051E00023F07E4343F0FC432361FCF759FD286024
:1051F000BFF35F8F584C3E46584D4FF00108636A2D
:1052000023F480336362C4F8947028E0002A4CD001
:105210002F686B7A103515F8061C1B0643EA0173DC
:1052200043EA420315F8052C43EA824315F8042C9F
:1052300043EA424315F8032CC4F89860013643EA68
:105240000243D4F8A020032E43F0010322F0010210
:10525000C4F8A020C4F89C70C4F8A03027D06B68B4
:105260002A7A002BD2D02F68002AD2D127F01F0231
:10527000A3EB0209B9F1200F38BF4FF020094846CF
:1052800080F000FC421E08FA02F1894508BF024680
:10529000D2B2BEE7FEE7FFF78DFC7CE6136A23F08F
:1052A000700343F040031362A2E6FEE773E60523B2
:1052B000C4F89430636A43F480336362BFF34F8F62
:1052C000BFF36F8FBFF34F8FBFF36F8F0022C4F810
:1052D0005022BFF34F8FBFF36F8F636943F40033E6
:1052E0006361BFF34F8FBFF36F8FC4F88420BFF3A8
:1052F0004F8FD4F8805043F6E0761749C5F34E340B
:10530000C5F3C905640104EA06002B4640EA83722E
:10531000013BC1F86022F9D2203C14F1200FF2D1F8
:10532000BFF34F8F4B6943F480334B61BFF34F8F13
:10533000BFF36F8F3FB0BDE8F0832CE60044025806
:105340000010005C7FBB2200008400407FBB223045
:10535000000002580008025800ED00E02803002475
:105360002DE9F843374E984606EB8003D3F8DC402E
:10537000002C65D004F1D203FC360546B4F8D20205
:10538000A36104F5E97366601746E3614FF4807327
:10539000261DE160C4E904332368C4F8CC30A3635C
:1053A00000284AD194F8D10006F0D4FA18F0080F7A
:1053B00094F8D09034D1BA0723D4FB0711D4052137
:1053C00094F8D60270F040FC94F8D63201221E49BF
:1053D00003F01F005B09824041F823203046BDE8FE
:1053E000F8830135484606F0B5FAEDB218B140F23F
:1053F00006630572C38094F8D42202210BF09EF854
:10540000DDE76B1CDBB218B1037240F20653C380B8
:1054100094F8D52202210BF091F8FB07CFD5E0E7F5
:105420000135EDB218B140F206730572C38094F8ED
:10543000D52202210BF082F8C1E76FF099FEB1E7A7
:105440002646CBE7188C0C0800E100E00148FDF788
:10545000DDB900BF5C0300240148FDF7D7B900BFE8
:10546000340600240148FDF7D1B900BF0C0900241F
:105470000148FDF7CBB900BFE40B00240148FDF75C
:10548000C5B900BFBC0E00240148FDF7BFB900BF7D
:10549000941100240148FDF7B9B900BF6C14002431
:1054A00070B52422456B00238168C0F8BC200446F7
:1054B0002A6800F1340622F001022A602B606B603A
:1054C000AB608279C0F8C43080F8B830C0F8BC3026
:1054D000C364C0F8C0304365C0F8A030C0F8A43041
:1054E0009302816303F480534179C363130303F48C
:1054F00000530364130203F480634364C36D01F03B
:105500000200C90745D400287ED1A06412F0080229
:1055100054D0D4F8BC20002A00F08A802422C4F899
:10552000BC202A6822F001022A60002B7CD1304680
:10553000FCF74AFD012812D06B68304623F49043F3
:105540006B60AB6823F02203AB60AB6843F00803E9
:10555000AB602B6843F001032B6078F053FC627959
:10556000D6070DD5D4F8C830196841F48071196098
:10557000996841F001019960196841F020011960B2
:10558000950705D5D4F8C820136843F0800313604D
:1055900070BD0421A16470B30C21D007A164B5D5FE
:1055A0004FF4803143F00203616643F001034FF48E
:1055B0000031E365216612F00802AAD1D4F8BC10CC
:1055C00009B194F8B82084F8B8202422C4F8BC208B
:1055D0002A6822F001022A6013BB3046FCF7F4FC73
:1055E0000128BCD06B68304623F490436B60AB68F5
:1055F00023F02A03ACE7D10788D543F002034FF428
:105600008031E365616681E70821A164D1077FF5F8
:105610007DAF43F001034FF40031E3652166CAE733
:105620003046FBF753FCD8E73046FBF74FFC7EE7EC
:1056300084F8B82072E700BF816031E741712FE73D
:1056400081712DE72DE9F843434D3C20434C05F58E
:105650009872B5F83631C4F87C28A4F88838B5F8C3
:105660003A21B5F83E31A4F88A28A4F8803806F02B
:1056700071F90746422006F06DF90646382006F01B
:1056800069F981461FB10D23FB8000233B721EB1D7
:105690000D23F38000233372B9F1000F05D00D23E1
:1056A000A9F80630002389F80830B5F842313920CE
:1056B000A4F88238B5F84631A4F88438B5F84A31F0
:1056C000A4F8863806F046F980463A2006F042F9FA
:1056D00005463B2006F03EF90446B8F1000F05D020
:1056E0000D23A8F80630002388F808301DB10D23DB
:1056F000EB8000232B721CB10D23E3800023237267
:10570000484608F097FE0121484606F04BF940460E
:1057100008F090FE284608F08DFE204608F08AFE2C
:105720004046012106F03EF92846012106F03AF9EB
:105730000121204606F036F9384608F07BFE304657
:1057400008F078FE3846012106F02CF93046012198
:10575000BDE8F84306F026B9188C0C08802E00240A
:1057600038B5134D41F20D13124941F28832D5F884
:10577000D008D5F88C480004A060E06801402046BD
:105780000B430D21E360FDF777FB38B1D5F8C02856
:10579000034600201343C5F8C03838BD606900F4E3
:1057A000F050A0F50060B0FA80F0400938BD00BFAD
:1057B000802E0024C0E0FEFF2DE9F04FA74D7C2293
:1057C00000219BB005F68C0081F0F8FF4FF480318A
:1057D000D5F87C4895F8BC382268C5F890184FF485
:1057E0000031C5F88C28C5F89C180221C5F8A0180E
:1057F000002B00F088800422994B85F8BC28DA6CD5
:105800001B68D6030DD5180100F1D98001224FF095
:10581000006385F8BC28C5F8C03801201BB0BDE87E
:10582000F08F9C01F2D50AAB18460193FCF7CCFD32
:105830000B990029EAD0D5F88C480A0A894B66688A
:10584000A3FB0232884B894F33401009B94243EA27
:1058500012136360236843F00303236040F2F9806E
:105860004300834AB1FBF3F3B2FBF3F2296802323F
:105870002B685B1A9A42FBD800237E4A0493A360EC
:105880007D4BE16817680B4043F48053E3607B4B2A
:10589000A3FB073741F288337F0A03FB07F73B4638
:1058A000002B00F0CB80626B013B1106F8D5744BE6
:1058B000714AA3634FF4D573A360E3681A4041F2C1
:1058C00008131343E3604FB13B46626B12F0450F80
:1058D00002D0920440F1DC80013BF6D10023C5F8F0
:1058E000C838A360644BE268134043F48053E3601C
:1058F0003B46002B00F0A280626B013B1106F8D5FD
:105900005F4BA363E3E05F4B9A425FD05E4B9A42EA
:1059100000F00F8195F8880806F01CF8834695F88A
:105920008A0806F017F8824695F8800806F012F803
:10593000814695F8820806F00DF8804695F88408AF
:1059400006F008F8074695F8860806F003F895F87B
:10595000892806460E2158460AF0F0FD504695F873
:105960008B280E210AF0EAFD484695F881280E2181
:105970000AF0E4FD404695F883280E210AF0DEFD8A
:1059800095F8852838460E210AF0D8FD0E2195F8A5
:10599000872830460AF0D2FD0221B4F9040070F0E5
:1059A00053F9B4F90430002BFFF625AF03F01F00C4
:1059B00001225B093549824041F823201BE70AABED
:1059C00018460193FCF7CCF90C9932E7244BD3F835
:1059D000D42022F48032C3F8D420D3F8D42042F467
:1059E0008032C3F8D420D3F8D42002F4803203925A
:1059F000039ADA6F42F48032DA67DA6F22F4803287
:105A0000DA6787E72A684FEA134EA2EB090273466A
:105A1000824213D8002B40F03181C4F808E0E368DB
:105A200003EA0A030B43E3603B46626B12F0450F47
:105A300002D0920440F1F080013BF6D14FF00040DB
:105A4000012385F8BC38D5F8C0380343C5F8C03801
:105A5000E3E6074AB2FBF1F2296808E7802E00244A
:105A600000440258598B4F01002CC0FFFF340C003A
:105A70001021010000000024C0E0FEFFD34D6210A1
:105A8000C5002000007000520024024800E100E040
:105A9000636B5B0700F16F83636BDE0769D4636B35
:105AA000580601D54023A3630123704A37212046BD
:105AB000C5F8C8380023A360E3681A4041F23713E1
:105AC000134341F28832E360FDF7D6F970BB049AC4
:105AD0004FF6FE739A4200F23982DFF890A1DFF8A8
:105AE0009881634E002241F2371337212046A2608D
:105AF000E26802EA0A02134341F28832E360FDF7EA
:105B0000BBF900289CD1C4F8088041F22913E2684F
:105B100002EA0A021343E36047B13B46626B12F0AC
:105B2000450F01D0920427D5013BF7D14FF08050AB
:105B300086E7504BD3F8DC2022F40072C3F8DC2057
:105B4000D3F8DC2042F40072C3F8DC20D3F8DC2068
:105B500002F400720292029AD3F8842042F4007296
:105B6000C3F88420D3F8842022F40072C3F8842080
:105B7000D0E60123A36397E7636B5B0758D4A66362
:105B80006269049B002A03F101030493049B03DB75
:105B90004FF6FE718B42A5D904994FF6FE739942D8
:105BA00000F21782500040F1D4814FF00108D5F87F
:105BB0000090C5F8C4882368990700F0C4810023C9
:105BC000DFF8A8A02046A36041F20233E26802EAAF
:105BD0000A021343E360FBF7D7F900287FF430AFE4
:105BE000636941F20311C5F8F838A369C5F8FC38B8
:105BF000E369C5F80039236AC5F80439A060E36891
:105C000003EA0A030B43E360002F3FF417AFDFF80A
:105C100060C041F2873007E7636B5B0722D4636B98
:105C2000DE071CD42369DBB2032B06D0012007E773
:105C300004234FF08050A36302E7C4F838C06369BF
:105C400013F4604F3FF4DEAE590400F19D8213F46B
:105C5000004F0CBF4FF480304FF48050F0E601232A
:105C6000A363E3E704231846A363E9E6C0E0FEFF6D
:105C7000C500200000440258000010C14FEA0E4940
:105C8000C5F8D0E8D44A2046C4F80890E3681A4022
:105C900041F209331343E360FBF776F900287FF400
:105CA000CFAE6269C5F8E828A369C5F8EC38E769A2
:105CB000C5F8F078216AC5F8F418D4F818C04FEA8E
:105CC0001C5CC5F8CCC84FEA927C8DF828C0C2F3A2
:105CD000836C8DF829C0C2F3016C8DF82AC0C2F321
:105CE000074C8DF82BC0C2F3072CD2B28DF82CC014
:105CF0008DF82D201A0DADF82E20C3F303428DF838
:105D00003020C3F3C0328DF83120C3F380328DF8D8
:105D10003220C3F340328DF83320C3F300328DF8C4
:105D200034208DF83500B8F1000F00F01F811B04FE
:105D300003F47C1343EA17430E934FF40073C5F842
:105D4000D8380E9B01339B02C5F8D438C5F8DC382F
:105D5000C7F380334FF4007A20468DF84130C7F303
:105D6000C61307F07F07C5F8E0A88DF84230CB0FC7
:105D70008DF8437001278DF84430C1F341738DF8DD
:105D80004530C1F382638DF84630C1F383538DF8FB
:105D90004730C1F340538DF8483000238DF8493027
:105DA000C1F300438DF84A30C1F3C0338DF84B3056
:105DB000C1F380338DF84C30C1F340338DF84D3052
:105DC000C1F300338DF84E30C1F381238DF84F308D
:105DD000C1F30123C1F346018DF8503041F207139E
:105DE0008DF8511007218DF85270C4F80890DFF833
:105DF000E891E26802EA0902134341F28832E36063
:105E0000FDF73AF800287FF41BAEC4F808A041F271
:105E1000101BE36841F288321021204603EA09038F
:105E200043EA0B03E360FDF727F8002840F0948075
:105E300095F8BC38032B3FF4F0AC2F6863699A01E6
:105E40007ED44FF0400A41F2883210212046C4F837
:105E500008A0E36803EA090343EA0B03E360FDF7E4
:105E60000BF8002843D1D5F8D038372120461B0441
:105E7000A36041F23713E26802EA0902134341F2D8
:105E80008832E360FCF7F8FF88BB4FF0FF330D2149
:105E90006362C4F828A0E36A23F0FF0343F06303BE
:105EA000E36241F20D13A0602046E26802EA0902B3
:105EB000134341F28832E360FCF7DEFFB8B9019E7C
:105EC00004E02B68DB1B013300F08A80636B13F462
:105ED000957F636B40F087801B04F2D506F12002AA
:105EE000D4F8803046F8043BB242F9D1E9E7D5F85E
:105EF000C038C5F8C038394B0122A363D5F8C03883
:105F000018434FF40073C5F8C008204685F8BC2834
:105F1000A36041F21013E1682F4A0A401021134395
:105F200041F28832E360FCF7A7FF00283FF475AC2C
:105F30002A4A0123A263C5F8C00885F8BC386CE47E
:105F40004FF40060D7E74FF0806079E5049A9A42F9
:105F50003FD84FF000082AE6204BA363D5F8C0389D
:105F60000343C5F8C03885F8BC7856E440F6FC72A7
:105F700002EA830343EA97730E93C7F3C2638DF873
:105F80003C30C7F302638DF83D30C7F342538DF8C0
:105F90003E30C7F382438DF83F30C7F3C2338DF8EC
:105FA000403001230E9A9DF840001A4400F007008B
:105FB000023082409DF8300000F00F00C5F8D42870
:105FC0008340C5F8D8385B0A02FB03F3C5F8DC3818
:105FD000BEE64FF0807033E5C0E0FEFFFF0FE01F2C
:105FE0004FF0004087E7180700F1C880636B9907FE
:105FF00000F1C880636B9A0608D5C1E0D4F8802010
:106000002B6846F8042BDB1B0133E9D0636BDB0400
:10601000F4D40A9B5E4AA263C3F381128DF8142064
:10602000C3F340128DF815201A0A22F0FF0242EA4B
:106030001362DDE90B1392B209BAADF81620DAB299
:1060400006918DF81C20C3F307229DF83B108DF8B4
:106050001D20C3F303521B0C8DF81E200D9A23F054
:10606000FF03D0B203432046ADF82030C2F38523AE
:106070008DF82230C2F301238DF82330C2F30313CD
:1060800002F00F028DF824304FF400738DF82520B4
:106090008DF826101021A3603E4AE3681A4041F2B1
:1060A0001013134341F28832E360FCF7E5FE002849
:1060B0007FF43EAF9DF82430B8F1010F9DF8252004
:1060C000DBB2D2B205D1134314BF4FF400784FF4C2
:1060D0008078D5F89808C5F8E4886FF007FC0028A8
:1060E0007FF49BAB2C6803E02B681B1B013330D083
:1060F0006FF0DAFB0428F7D100230121D5F8D4286A
:10610000C5F8C038C5F8B83885F8BC18002A3FF47F
:1061100084AB4FF480406FF0E9FB00287FF47DAB47
:10612000D5F8C438F3B1012B7FF477AB02201A4CB9
:1061300085F80809A4F124030FCB84E80F00A4F12B
:10614000140310340FCB84E80F0000201BB0BDE80F
:10615000F08F4FF000420123C5F8C02885F8BC3805
:10616000FFF75BBBD5F8C838002BE0D0012B7FF4DC
:1061700054AB1846DBE70423A36395E40820BAE692
:106180002020B8E60220B6E64FF4005058E400BFE5
:106190003A0F0018C0E0FEFF8C370024C74BD3F83D
:1061A0000C19D3F8102970B58C0F93F80859100EFC
:1061B000C2F3072C83F83849C1F383640001012D31
:1061C00083F83949C1F3016483F83A49C1F30744BC
:1061D00083F83B49C1F30724C9B283F83C49C2F3B1
:1061E000035483F83D19A3F83E09C2F3C030B3F855
:1061F0003E1989B241EA0401C2F30344A3F83E19EF
:10620000C2F3403183F84049C2F3803483F8410936
:106210004FF0000083F8424983F84319C2F300317C
:1062200083F84419D3F8141983F8450940F2EF8034
:10623000022D00F0C3802A204FEA4C0C83F851490C
:10624000C1F3C01201F07F010CF07E0C83F852C93B
:106250004FF0010C93F852491443D3F8182983F8EE
:106260005249D40F83F85319910D83F85449C2F35E
:10627000417401F00C01C2F3815583F85549C2F312
:10628000826483F8564983F8571993F85719D3F85D
:106290001C49294383F85719C2F3405183F8581910
:1062A000002183F85919C2F3004183F85A19C2F347
:1062B000C03183F85B19C2F3803183F85C19C2F3F3
:1062C000403183F85D19C2F3003183F85E19C2F3DF
:1062D000812183F85F19C2F30121C2F3460283F8DA
:1062E0006019C4F3074183F86129220E090283F87B
:1062F00062C983F86429C4F30722A3F86619240647
:10630000B3F8661989B21143A3F86619D3F82019B6
:10631000C3F868490C0ED3F8682942EA0442C3F86E
:1063200068290A0AD3F8684902F47F422243C1F37C
:106330000724C9B2C3F86829D3F86859D3F82429C7
:106340002C43C3F8684983F86C19110E83F86D1952
:10635000110C0906C3F870191102D3F870490A46E6
:1063600001F47F01214392B2D3F82849C3F8701990
:10637000D3F870190A43C3F87029C4F30352D3F851
:10638000701941EA1461C3F8701993F87419114334
:10639000C4F3072283F87419210A01F47061A3F889
:1063A0007619B3F8761989B21143C4F34602A3F8FB
:1063B000761983F8782983F879C970BD1204C1F37E
:1063C000072C0D0E02F47C12C3F84829C1F30742D2
:1063D000D3F8484944EA0524C3F84849D3F8484962
:1063E00022434FF40074C3F84829D3F84829C3F86E
:1063F0008849013240F10004A40244EA9254920216
:10640000C3F88449C1F38034C3F8802914E74FEA04
:106410008C2CC1F3C26594000CF44062C1F3072CCC
:1064200004F47F74C3F84829D3F848291443CA0BED
:10643000C3F8484902F00602D3F8484944EA917487
:10644000C3F84849C1F3026483F84C59012583F825
:106450004D49C1F3425483F84E49C1F3824483F855
:106460004F49C1F3C03483F8502993F8502922438F
:1064700083F85029D3F8484993F8502993F8406994
:10648000023205FA02F2B540D617A2FB052EC3F878
:10649000885905FB06EE04FB0EEE0134A2FB042432
:1064A000A644520AC1F3803442EACE52C3F880298E
:1064B0004FEA5E22C3F88429BEE600BF802E002486
:1064C0006FF04EB86FF04CB810B51C2005F042FAD2
:1064D0000446112105F066FA1CB1A38822681B044A
:1064E0009361C8200DF0FEFE2046BDE8104007F085
:1064F000A1BF00BF1C48D0F80038D0F8082830B53C
:106500009B184FF01A040C8001D1184830BD174A6F
:106510000024D0F8040802F1100511464FEA137E5A
:10652000B3F1204FCC7001F102010EF1370C38BFEE
:106530000EF1300C8D424FEA031381F800C0EDD10B
:106540000B4D0024010FB0F1204FD47402F1020270
:1065500001F1370338BF01F1300395424FEA0010D3
:106560001374EFD1014830BD00E0F11F4017002443
:1065700048170024122301480B8070475400002460
:1065800000207047212808B524D0222816D02028C2
:1065900012D189B1072A0FD1154A164B0868B1F8F4
:1065A00004C012688979D861A3F820C083F822104A
:1065B00012B1014600209047002008BD0029FBD001
:1065C000022AF9D10A4B5B68002BF5D0098800201C
:1065D0009847F1E70029EFD0072AEDD1054BD8699C
:1065E0001A8C93F82230086000208A808B7108BDD5
:1065F000203800244017002400207047034B93F8F4
:106600002C00003818BF0120704700BF203800243C
:10661000034B93F82C00032894BF002001207047FF
:10662000203800240048704750380024164B0020C2
:1066300030B493F82A4014B1DD698D4205D00130A1
:1066400010330828F5D130BC7047104BB2B1996FA8
:1066500001EB40218A4201D1022C08D093F8182284
:1066600012B9012283F81822012283F8612003EB7A
:106670000013012283F88A2030BC704703EB00131B
:1066800083F88A20DFE700BF803800242038002408
:1066900030B40023194C04F1600084F8043103E0A5
:1066A00001331030082B1BD0C5698D42F8D190F80A
:1066B0002AC0BCF1030FF3D1A2B1A16F01EB4321BA
:1066C0008A4208D094F8182212B9012284F81822BC
:1066D000012284F8612004EB0314012384F88A303A
:1066E00030BC7047D4F8002104EB031304210132BD
:1066F00083F88A10C4F80021F2E700BF2038002494
:10670000C0B1836823B10F4B072283F86220704722
:106710000C4A042192F8600082F87430032882F851
:106720006210C2E91B3314BF4FF480738023C2E9A7
:1067300019337047034B012283F8182283F8612034
:10674000704700BF20380024244910B5CC8C91F844
:1067500024C0644531D963462431E646624603E0ED
:10676000944238D991F800E07144724491F801E004
:1067700092B2BEF1050FF3D191F802E0BEF1810FA4
:10678000EED1174A03E0A3421BD292F800C0624444
:10679000634492F801C09BB2BCF1050FF3D192F8AB
:1067A00002C0BCF1010FEED119B1002402230C711B
:1067B0004B7100210223117153712023038008487B
:1067C00010BD0029F9D0022300224B7120230A7149
:1067D0000380034810BD0021D3E700BF4017002409
:1067E00064170024244910B5CC8C91F824C064456A
:1067F00031D963462431E646624603E0944238D9F3
:1068000091F800E07144724491F801E092B2BEF157
:10681000050FF3D191F802E0BEF1810FEED1174AD6
:1068200003E0A3421BD292F800C06244634492F892
:1068300001C09BB2BCF1050FF3D192F802C0BCF1CC
:10684000010FEED119B1002440234C710B710021CE
:1068500040235171137120230380084810BD002983
:10686000F9D0402300220B7120234A710380034892
:1068700010BD0021D3E700BF401700246417002497
:10688000244910B5CC8C91F824C0644531D96346B5
:106890002431E646624603E0944238D991F800E09C
:1068A0007144724491F801E092B2BEF1050FF3D148
:1068B00091F802E0BEF1810FEED1174A03E0A34246
:1068C0001BD292F800C06244634492F801C09BB2AC
:1068D000BCF1050FF3D192F802C0BCF1010FEED16B
:1068E00019B1002440234C710B71002140235171D8
:1068F000137120230380084810BD0029F9D04023DC
:1069000000220B7120234A710380034810BD00212F
:10691000D3E700BF401700246417002403460A226F
:1069200001481A80704700BF8417002438B5D0F89A
:10693000D432B03350F823507DB195F81C32044660
:1069400023B9D5F818320BB16B7A8BB1812120466F
:1069500076F0F4FF6B7A022B00D038BD20468121FF
:1069600076F0ECFF20460121BDE8384076F0E6BF26
:10697000012176F0E3FF20468121BDE8384076F022
:10698000DDBF00BFD0F8D42200EB82022DE9F04138
:10699000D2F8C0420646002C4ED0B4F8643204F15E
:1069A0001007D4F870520846D2F8C422394603FBC7
:1069B00005F5D2F81080B5F5007FD4F86C2228BF19
:1069C0004FF40075B5FBF3F39BB2C04700281BDB07
:1069D0002B463A468121304677F036F9B4F86422E6
:1069E000B5FBF2F2D4E99B1311449B1AD4F8382278
:1069F000521BC4E99B13C4F8382213B10020BDE830
:106A0000F08103232372F9E7D6F8D432B03356F875
:106A100023208AB192F861320424112003F1480145
:106A20000133DBB202F8314002EBC101A34288809E
:106A300008BF002382F861324FF0FF30DFE700BF6C
:106A400038B5084BD3F8883253B1DB6914460D468C
:106A500098474FF40073026800202A60238038BDF5
:106A60001B68FFDE2038002408B5064BD3F88832B7
:106A700023B11B699847013840B208BD4FF0FF3081
:106A800008BD00BF20380024002070470020704758
:106A900008B520B904486EF03DFB044808BD044821
:106AA0006EF038FB014808BD24360D08AC3A0024CE
:106AB00048360D08024808B56EF02CFB014808BDA9
:106AC0006C360D08AC3A0024024808B56EF022FB83
:106AD000014808BD74360D08AC3A0024024808B5D8
:106AE0006EF018FB014808BD80360D08AC3A002452
:106AF00008B520B904486EF00DFB044808BD0448F1
:106B00006EF008FB014808BD90360D08AC3A002431
:106B1000B0360D08024808B56EF0FCFA014808BD11
:106B2000D0360D08AC3A0024024808B56EF0F2FAEF
:106B3000014808BDDC360D08AC3A0024D0F8D43248
:106B4000B03370B550F823402CB30026124B0546E5
:106B500084F83C12C4F8303204F50C7226720D230E
:106B6000812104F5047477F06FF8D5F8C8321F223C
:106B70000121C3F88C62A3F8781203F51E7118681E
:106B8000C3E9A1429A79012A08BFC3F89442BDE83B
:106B9000704076F049BF70BD55534253D0F8D422AF
:106BA00000EB82022DE9F041D2F8C0420646002CEB
:106BB00067D0B4F8643204F11007D4F87052084674
:106BC000D2F8C422394603FB05F5D2F81480B5F596
:106BD000007FD4F86C2228BF4FF40075B5FBF3F3A7
:106BE0009BB2C047002834DBD4F83802B4F86422E2
:106BF000401BB5FBF2F5D4E99B13C4F838022944D5
:106C00005B1BC4E99B13FBB1D6F8C80202FB03F37C
:106C100001220021B3F5007FC0F88472A0F8782229
:106C2000827928BF4FF40073C0F88C1200F51E71F2
:106C3000012AC0F8883208BFC0F89472006876F064
:106C4000F3FE0020BDE8F08119463046FFF776FFDD
:106C5000F7E7D6F8D432B03356F823208AB192F849
:106C600061320424032003F148010133DBB202F84E
:106C7000314002EBC101A342888008BF002382F8A3
:106C800061324FF0FF30DDE7D0F8D43200EB830300
:106C90002DE9F043D3F8C04283B0002C00F0B78058
:106CA0001646127805460F465A2A5FD85A2A00F22D
:106CB0009B80DFE812F04601990099005A01990083
:106CC00099009900990099009900990099009900FC
:106CD000990099009900990099008E0199009900F6
:106CE00099009900990099009900AC01CD01990093
:106CF00099003D01990099009900990010029900AE
:106D0000360299009900FA0099005E0299009900F4
:106D100099009900E1019900990099009900990062
:106D2000990099009900990099009900990099009B
:106D3000990099009900990099009900990099008B
:106D4000990099009900990099009900990099007B
:106D5000990099009900990099009900990099006B
:106D600099009900990099009900F001A82A53D040
:106D7000AA2A00F064829E2A36D1D3F8C43208468B
:106D800004F5197204F51A715B68984701460028EA
:106D900040F0098394F86232022B00F00483D6F8A5
:106DA0000A301ABAE2601BB104F1100080F006FD4F
:106DB000D4F868320022013B190E61F30702190C66
:106DC00061F30F22190A61F31742B4F8641263F3F6
:106DD0001F624BBA6383002362612383D6F80A30B3
:106DE0001BBAE360002014E094F8612205262025F8
:106DF0000221531C4832DBB204F8326004EBC200BB
:106E0000042B858008BF0023617284F861324FF043
:106E1000FF3003B0BDE8F08394F80880B8F1000FAC
:106E20007DD194F91C22002A80F2058394F8622215
:106E3000022A00F08083D3F8C43208469B68984742
:106E4000002840F0DE82D6F80230D5F8D4121BBA02
:106E5000B031C4F86C32D6F8062055F8211012BAB9
:106E6000C4F870220029D2D01344D1F868028342BA
:106E700000F24783B4F8643202FB03F3D4F818221B
:106E80009A424AD091F861320524202003F1480249
:106E90000133DBB201F8324001EBC202042B9080D7
:106EA00008BF002381F86132B1E794F80880B8F197
:106EB000000F34D194F91C22002A80F2BC8294F88D
:106EC0006222022A00F03783D3F8C43238469B6826
:106ED0009847002840F09582D6F80220D5F8D412C1
:106EE00012BAB031C4F86C22B6F8073055F8211048
:106EF0005BBA9BB2C4F87032002988D01A44D1F82A
:106F00006862B24200F27383B4F8642202FB03F3B6
:106F1000D4F818229A4240F0E182022323724FF4FF
:106F2000007339462846E36003B0BDE8F04329E525
:106F3000337900229B1AE26018BF012384F8623281
:106F400050E7D4F81822002A40F0398294F86212EF
:106F5000022900F04683D3F8C43238469B6898472C
:106F6000002840F0D382E0603CE7D4F81832002BD0
:106F700000F025827021002294F8603221740C21E7
:106F8000C4F81520E17594F86112C4F811209942F3
:106F9000C4F81920C4F81D2084F8212011D004EB76
:106FA000C30191F84012A17404EBC3010133B1F89D
:106FB0004412DBB2A183042B14BF84F8603284F83E
:106FC00060221223E36032799A4298BF1346E3604D
:106FD00008E7D4F81822002A00F0F1817278D2076D
:106FE00040F1B181B378002B00F0CF81802B40F0CD
:106FF000E0810821CC4A04F1180304F11000E1609B
:1070000012F8011D03F8011D8342F9D1EAE6D3F815
:10701000C4323846DB689847002840F074813279E2
:10702000042A134628BF0423E360002A3FF4DAAEA3
:10703000013BBD4A04F1100099B201F111030A4469
:10704000234412F8011903F8011D8342F9D1C9E65E
:1070500094F862223379012A03F0030300F06A8175
:10706000012B00F06C81022B00F06A81032B00F0F1
:1070700066810023E360B5E6737813F0020340F005
:107080009881D4E99B210A44D4F868128A4200F21C
:10709000E581E360A6E6D3F8C4323846DB6898475A
:1070A000002840F03881337A082B194628BF082180
:1070B000E160002B3FF496AE9C4A01F1100304F10D
:1070C00010000A4454FA83F312F8011D03F8011D5D
:1070D0009842F9D186E6D3F8C4320DF1020238465F
:1070E00001A95B689847002840F06F8194F86232EC
:1070F000022B00F06A81BDF802200821206152BAFB
:10710000019BA061013B62830C22E174E375190EBF
:10711000E2601A0C1B0A217562750222A3752276A1
:1071200077E6D3F8C43204F51972384604F51A71BB
:107130005B689847002840F0368194F86232022B51
:1071400000F03181D4F868320822A082013BE2606D
:10715000190E1A0C61F30700190A62F30F20B4F834
:10716000642261F3174052BA63F31F60E282206128
:1071700038E694F80890B9F1000F40F00081D4F897
:107180001822002A00F08A8194F91C22002AC0F2F9
:107190001582D3F8C43238469B6898478046002849
:1071A00040F0F181D5F8D432384605EB8303D3F8AB
:1071B000C432DB6898470146002840F08281D6F847
:1071C0000220D5F8D40212BAB030C4F86C22B6F856
:1071D000073055F820005BBA9BB2C4F87032002823
:1071E0003FF415AE1A44D0F86862B24200F2C6818C
:1071F000B4F8642202FB03F3D4F81822934240F05F
:10720000EC80B3F5007F4FF0010004F1100428BFBB
:107210004FF4007304F8080C1A46D5F8C832C3F8C6
:1072200088229A79C3F88C1203F51E718242C3F842
:107230008442A3F8780262D1C3F894425FE0227AD4
:10724000002A40F09C80D4F81812002900F08381B5
:1072500094F91C120029C0F22181D3F8C4323846B7
:107260009B689847D5F8D432002840F05A8105EB46
:1072700083033846D3F8C432DB689847002840F0CF
:10728000F280D6F80230D5F8D4121BBAB031C4F867
:107290006C32D6F8062055F8211012BAC4F87022C4
:1072A00000293FF4B4AD1344D1F86802834200F2E0
:1072B0002881B4F8643202FB03F3D4F81822934215
:1072C0007FF4E0ADB3F5007F4FF0010104F1100051
:1072D00028BF4FF40073217200241A46D5F8C83233
:1072E000C3F888229A79A3F8781203F51E71012A4F
:1072F000C3F88402C3F88C4208BFC3F8940218682C
:1073000076F092FB6EE50A4A92F8623063F07F03F2
:1073100082F8623083E6064A92F8673063F07F03B2
:1073200082F86730BFE600BFA0170024A41700242E
:1073300040170024022B3CD0012B7FF497AE002392
:1073400084F8623295E6D3F8C43207EBC70132798C
:10735000D86900EB810003790533934228BF1346B7
:10736000E360002B3FF43EAD03F1100203442244DE
:1073700013F8011D834202F8011DF9D132E53946A7
:10738000284603B0BDE8F04308E406219A4A04F118
:10739000160304F11000E16012F8011D03F8011D4D
:1073A0008342F9D11EE53A220221284675F0F0FF0A
:1073B0002DE524220521284675F0EAFF27E5202245
:1073C0000521284675F0E4FF21E528463A220221EE
:1073D00075F0DEFF4FF0FF301BE590F861320525B8
:1073E000202403F148020133DBB200F8325000EBF5
:1073F000C202042B948014BF80F8613280F86112BD
:1074000005E5D5F8D432B03355F82320002A3FF4EF
:10741000FEAC92F8613202243A2003F148010133B4
:10742000DBB202F8314002EBC101042B888075D039
:1074300082F86132EBE494F861320520202103F1F7
:1074400048020133DBB204F8320004EBC202042B21
:1074500091807FF4DAAC84F86182D8E4212205219E
:1074600075F096FFD3E4D5F8D432B03355F8232025
:107470008AB192F861320225272003F148010133D5
:10748000DBB202F8315002EBC101042B888008BF47
:10749000002382F8613205232372B8E494F8613244
:1074A0000525202003F148010133DBB204F83150F7
:1074B00004EBC101042B88807FF4A7AC84F861221F
:1074C000A5E4D5F8D432B03355F82320002A3FF490
:1074D0009EAC92F86132022427209EE791F8613237
:1074E0000525202403F148020133DBB201F83250B4
:1074F00001EBC202042B94807FF4D4AC81F86102CA
:1075000085E491F8613205242120BFE43A2202216A
:10751000284675F03DFF0523237278E482F86182E6
:1075200075E4B03355F82320002AB4D092F86132C4
:1075300002253A20A1E794F8613203F148010133B2
:10754000DBB204F8312004EBC1013A22042B8A801B
:107550007FF45BAC7FE794F861320525202003F1CE
:1075600048020133DBB204F8325004EBC202042BB0
:1075700090807FF44AAC84F8611248E490F861325C
:10758000052521242DE7D5F8D432B03355F8232032
:10759000002A3FF43CAC92F8613202243A2003F115
:1075A00048010133DBB202F8314002EBC101042B88
:1075B00088807FF43DAF82F8619228E494F86132CC
:1075C0000520202103F148020133DBB204F8320028
:1075D00004EBC202042B91807FF417AC84F8619213
:1075E00015E43A2275F0D4FE052323720FE491F8D6
:1075F00061320525212475E796170024D0F8D4328E
:10760000B03350F82330CBB110B51A7A022A07D024
:10761000033A012A02D80021FFF790FA002010BD9A
:1076200003F21F2293F81D120446FFF72DFB0028DA
:10763000F4DA01212046FFF781FAEFE700207047D6
:10764000D0F8D432B03370B550F8235025B12B7A2E
:10765000044683B1012B01D0002070BD05F21F222A
:1076600095F81D12FFF710FB0028F5DA01212046DE
:10767000FFF764FAF0E7D5E98523C5F83832D0F88A
:10768000C832C5F83422D3F88C321F2B04D12F4BCB
:10769000D5F810229A421AD095F861324FF0050CB5
:1076A0002021204603F148020133DBB205F832C045
:1076B00005EBC202042B91804FF0020208BF0023A9
:1076C0006A7285F86132FFF731F9002070BD95F8D4
:1076D0001D120129E0D895F81E32013B0F2BDBD893
:1076E00005F21F22FFF7D0FA00282B7A22DB013B9C
:1076F000022BB1D9EE681EB3D4F8D432B03354F8AB
:1077000023100029A8D02046D1F83842D1F81832E9
:1077100005F11002A41BB342C1F838424FF0000437
:1077200028BF334681F83C4204240C72812176F054
:107730008BFA91E7052B99D02046FFF7F7F88BE7F6
:1077400031462046FFF7FAF986E700BF555342431A
:10775000554B0021554A1B685548A2FB032330B501
:10776000DB0C544C83B0013BC4F89C13C4F8941355
:1077700042F20F7194F8C923C4F88C03C4F898132B
:10778000C4F89033002A00F08A8002254A4948480C
:1077900084F8C953FAF78EFF0123484A062137209F
:1077A00084F8D43384F8CA3384F8CB3384F8CC33E8
:1077B00084F8CD3384F8CE3384F8CF3384F8D033D3
:1077C00084F8D13384F8D23384F8D33384F8C933BE
:1077D000D2F8E83043F02003C2F8E830D2F8E830BD
:1077E00003F020030193019B6EF02EFA344B4FF40B
:1077F00000025A6094F8C933012B3BD1D4F88C2392
:10780000304B3148B2F1804F18BF9A4284F8C953C7
:10781000D1680CBF0123002341F00101824208BF5F
:1078200043F0010300F58060D160824208BF43F05D
:10783000010300F580602549824208BF43F001033F
:1078400000F57840824208BF43F001038A4208BF36
:1078500043F0010313B91E4B9A4207D191681D4BA7
:107860000B40062B06D0B3F5803F03D0136843F0DE
:1078700001031360184AD2F8D432B03352F82330DF
:1078800043B116480021164AC3F80802C3F8101283
:10789000C3F804220020C4E9000003B030BD02F0A8
:1078A000FF0084F8C80370E70000002483DE1B4358
:1078B0000014004020380024B03B0024004402584B
:1078C00000E100E00000014000040040001800401A
:1078D0000040014007000100882E00249456002437
:1078E0009446002410B50B68054A064C13602060CE
:1078F0000BB1002010BD6EF06DFD002010BD00BF6B
:10790000842E00246C310024F8B51F4FD7F8E426EC
:10791000B7F8E816D7F8883291614BB39B6998475E
:1079200030B30026D7F8883213B11B69984790B955
:10793000B6F57A7F24D00CF0A7FC013604460D463C
:107940000CF0A2FC001B61EB0501B0F57A7F71F130
:107950000001F5D3E6E7B6F57A7F4FF0FF3018BFA8
:107960000020B7F8E836D7F8E4261B049361F8BD89
:10797000064B03F16C02DB6EC7F888229847D0E70C
:107980004FF0FF30EDE700BF2038002440170024FF
:107990002DE9F84F344E90469A46B6F8F426D6F8BC
:1079A000F0461304A361BAF1000F50D0C8EBC853DE
:1079B000C24406F5F06901EB432B41F28937D6F852
:1079C00088225AB100235468494640461A46A047C7
:1079D000A8B9D6F888320BB11B699847013F3AD055
:1079E0000CF052FC04460D460CF04EFC001B61EB03
:1079F0000501B0F57A7F71F10001F5D3DFE741F2BF
:107A00008937D6F8883213B11B69984780B9013F8E
:107A100021D00CF039FC04460D460CF035FC001B5F
:107A200061EB0501B0F57A7F71F10001F5D3E8E76C
:107A30000BEB482008F101084FF4007249467DF035
:107A40003FFED045B9D1D6F8F046B6F8F42600206E
:107A5000A261BDE8F88FD6F8F0364FF0FF30B6F8E7
:107A6000F4269A61BDE8F88F203800242DE9F84FFC
:107A7000364E90469A46B6F8F426D6F8F0461304E9
:107A8000A361BAF1000F54D0C8EBC853C24406F545
:107A9000F06901EB432B4FF400720BEB4821484691
:107AA0007DF00EFED6F888220AB341F28937002312
:107AB000D468494640461A46A047D6F88832B8B13D
:107AC0000BB11B699847013F37D00CF0DDFB044632
:107AD0000D460CF0D9FB001B61EB0501B0F57A7F78
:107AE00071F10001F5D3D6F88822002ADFD10023F6
:107AF00041F2893713B11B69984790B9013F1CD0F7
:107B00000CF0C2FB04460D460CF0BEFB001B61EB03
:107B10000501B0F57A7F71F10001F5D3D6F888320E
:107B2000E8E708F10108D045B5D1D6F8F046B6F837
:107B3000F4260020A261BDE8F88FD6F8F0364FF0A9
:107B4000FF30B6F8F4269A61BDE8F88F203800249B
:107B500010B50F4CA36D23B119689A880B691A42AE
:107B60000AD0FDF729FE38B994F820300133DBB292
:107B7000072B84F8203003D9002384F82C3010BD63
:107B8000044A0123126884F82C30E26110BD00BF62
:107B9000203800247031002410B50B4CA36D23B1A4
:107BA00019689A880B691A420AD0FDF705FE38B9A0
:107BB000064B012220841B6884F82C20E36110BD51
:107BC000002384F82C3010BD2038002470310024AC
:107BD00070B5164D0021164E6B6C2C681B04B162FB
:107BE000144A0D21A3602046E3681A4041F20D13A8
:107BF000134341F28832E360FBF73EF950B16B6BFF
:107C000003436B630C4A09230020126886F82C306A
:107C1000F26170BD636903F4F053B3F5006FF1D105
:107C20000423022086F82C3070BD00BF0C370024DE
:107C300020380024C0E0FEFF7031002470B50C4DE8
:107C400004460E4695F82C30042B0AD0082B06D19A
:107C50006B6A83420AD0FFF7BBFF022801D00120E4
:107C600070BD0823C5E9094685F82C30022070BD97
:107C70002038002470B5804C94F82C506B1E082BD3
:107C80001BD8DFE803F06C60701A4705321A240035
:107C90007A4B5B6A002B60D1794B072265691B68C0
:107CA00084F82C20E361002D57D0A3690120D4E98A
:107CB0000221A84794F82C506B1EDBB2022B46D948
:107CC000042D18BF082D0CBF0120002070BDFDF74A
:107CD00047FD002840F0C480694AE3691268FA331E
:107CE0009342EDD2FFF734FFC6E7FDF739FD0028D8
:107CF000F2D0A36A0022012B84F8202040F2B48045
:107D0000626A013B08210132A36284F82C1062628E
:107D1000012070BD594B1E6A002E65D1FDF720FD74
:107D2000002868D00423656984F8206084F82C302A
:107D3000002DEDD0A3693046A268E168A84794F809
:107D40002C506B1EB9E76DF0AFFD04285FD04C4B93
:107D5000E2691B689B1AC82B77D8002070BD0223EC
:107D600084F82C3088E7FEF719FA0028EFD1454B4C
:107D70000421A06293F82C2084F82C10D88D196B64
:107D800084F83620090E1A6BA086120C84F837107E
:107D9000196B186B84F83820090A84F83A0093F8B4
:107DA000340093F8352084F83910120984F83B0028
:107DB00093F8350084F84020996B00F00F00DD8FB8
:107DC000DA8FE163D98FC2F30B1384F8410043EAE1
:107DD000152301F00F0203F00F0384F8442003F58C
:107DE000FA63A4F8423047E7254AE369126864332E
:107DF0009342BFF465AFFFF7ABFE6569002D3FF41A
:107E00003BAF0022A369E1681046A84734E7FEF7BC
:107E1000C5F900289BD11C4B1B78002BA3F1020352
:107E2000B3FA83F308BF01255B0984F8225084F874
:107E30002330FEF7B3F900287FF454AF114B03222F
:107E40009B6C84F82C20236316E7FFF781FE94F8DF
:107E50002C00042818BF08280CBF0120002070BD8A
:107E6000042384F82C3053E7FAD1FFF7B1FE94F8DD
:107E70002C506B1E21E700BF203800248C370024D3
:107E800070310024B8370024883700242DE9F041F0
:107E900006460D4690461F465F4C94F82C10042968
:107EA00005D0082900F08A800120BDE8F081062273
:107EB0000123C4F8148084F82C20584A2374536298
:107EC000EB06A761C4E9025662D1BFF34F8F544A53
:107ED00005F500712B46C2F8683220338B42FAD187
:107EE000BFF34F8FBFF36F8F002D00F08E80DFF850
:107EF0003C8198F83030012B4AD1731CD8F85010CF
:107F000000228B42C8F8342070D80323D8F80070C0
:107F1000C8F81C50182188F830304FF40073FA620A
:107F20003846C8F82030D8F838303E4A012B4FF098
:107F3000FF337B624FF4007318BF7602BB62FB6AAB
:107F400023F0FF0343F09003FB62FB6843F0400320
:107F5000FB609023BD6501253D65C8F82C30BE60EF
:107F6000FB681A4041F21813134341F28832FB6058
:107F7000FAF782FF002840D02B4B0022BB63D8F8D1
:107F800034300343C8F8343088F83050C8F82C2017
:107F900094F82130022B1BD8013384F821300CF0E7
:107FA00073F904460D460CF06FF9001B61EB0501F7
:107FB000B0F57A7F71F10001F5D375E7636AB342DA
:107FC0003FF475AFFFF704FE02283FF466AF6BE79E
:107FD000002684F82160FFF7BBFD656925B1A36920
:107FE0003246E1680120A84703205EE7D8F8343024
:107FF00043F00073C8F83430CAE7FB6B84F8210003
:1080000043F48D73FB63BDE8F081084A536B43F082
:1080100000635363BCE700BF203800248C37002482
:1080200000ED00E0C0E0FEFFFF0FE01F0C37002472
:108030002DE9F84F634F0C468046164697F82C10F2
:108040001D46042908D0082902D00020BDE8F88F79
:10805000FFF7BEFD0228F8D114F01F016AD10122FA
:10806000594B5A489A6002624FF40072C7F880492F
:108070005A60002C00F09880DFF860B19BF8303037
:10808000012B57D108F10100DBF85030CBF8341048
:10809000984200F28F800323DBF800A04FF0010923
:1080A0008BF830305046DBF83830CAF82C101121EC
:1080B000012B4FF0FF33CBE90942CAF824304FF4CB
:1080C000007314BF4FEA48224246CAF82830DAF853
:1080D0002C3023F0FF0343F09203CAF82C30DAF877
:1080E0000C3043F04003CAF80C308123CAF85840E2
:1080F000CAF85090CBF82C30CAF80820344ADAF885
:108100000C301A4041F21113134341F28832CAF87D
:108110000C30FAF7B1FE034688B32E4ACAF838206D
:10812000DBF8342013430022CBF834308BF8309046
:10813000CBF82C2097F82130022B11D8013387F887
:1081400021300CF0A1F804460D460CF09DF8001B00
:1081500061EB0501B0F57A7F71F10001F5D374E7A9
:10816000002587F82150FFF7F3FC7C69002C3FF4D1
:108170006CAFBB692A46F9682846A04765E7052227
:1081800087F82130DAF83C30484687F82C2043F451
:108190009573114A7E61CAF83C301368BD61FB617A
:1081A000C7E90248BDE8F88F0C4A536B43F00063FF
:1081B0005363BFE7DBF8343043F00073CBF834305F
:1081C000B8E700BF20380024A04100248C370024E9
:1081D000C0E0FEFFFF0FE01F703100240C370024C9
:1081E0002DE9F04104464FF41D707FF007FF05466E
:1081F00000285BD0D4F8D47204EB8707C7F8C0021C
:10820000237CC4F8BC02002B45D04023022201216C
:10821000204675F08BFA012240234FF001082046DA
:10822000A4F8782181210222002675F07FFAA4F8B3
:108230003880D7F8C43230462E81A5F8606285F8C0
:1082400062621B689847D4F8C84294F8943427684F
:10825000434508D03846FAF7D9FE41463846FAF782
:10826000ADFE84F8946405F504751F22002338469A
:1082700004F51E71C4F88C320123C4E9A152A2791D
:10828000A4F878329A4208BFC4F8945275F0CCFB37
:108290000020BDE8F0814FF4007302220121204646
:1082A00075F044FA01224FF40073B6E7D4F8D432E3
:1082B0000220B03344F82350EBE700BFF0B50023B1
:1082C00083B0ADF80630D0F8D43200EB8303D3F896
:1082D000C0524DB10A78044612F0600036D0202812
:1082E00005D0204675F066FB032003B0F0BD48784A
:1082F000FE2849D0FF28F4D14B88002BF1D1CE883D
:10830000002EEED11006ECD44FF4807381212B8126
:1083100005F50475D4F8C842204676F0BBFD20462A
:10832000012176F0B7FD1F22012304F51E7120689C
:10833000C4F88452A4F87832C4E9A226A2799A42F9
:1083400008BFC4F8945275F06FFB46E04B780B2BD6
:10835000C7D801A252F823F0DF8304084F84040831
:10836000E3820408E3820408E3820408E382040849
:10837000E3820408E3820408E3820408E382040839
:1083800017840408CF8304084E88002EA9D1CF8813
:10839000012FA6D11206A4D5D3F8C4329B69984701
:1083A000022328604FF48071C4F89432D4F8C832A4
:1083B000C4E906779A79998203F11401012A5F6270
:1083C0001D629E6241D0186875F02EFB05E094F89E
:1083D0009C32032B85D18B786B60002085E794F865
:1083E0009C32032B7FF47DAF0222D4F8C8320020E8
:1083F000C4F8942203F11401C4E906220DF1060425
:108400009862C3E908424FF480729A829A79012AED
:10841000D9D11C63D7E794F89C32032B7FF461AF6A
:10842000D4F8C8320122022104350020C4F8941285
:108430004FF48071C4E90622C3E908529A799982FF
:1084400003F11401012A9862BDD11D63BBE794F8C2
:108450009C32032BC1D14B88002BBED1D4F8C8620B
:108460008F8896F89434012B0AD00123390630689E
:1084700086F8943410D4FAF7C9FD002386F89434B2
:108480006B7A022B0DD03A06A7D5012BA5D001217E
:108490002046FEF753FBA0E707F00F01FAF78EFD29
:1084A000EBE72046812175F049FA0121204675F05D
:1084B00045FA92E7F8B5D0F8C852012604460022E2
:1084C00095F89434A5F87862B34227D031462868ED
:1084D00085F89464002775F037FC40F20113A4F886
:1084E000787132463146286885F894642B8775F098
:1084F0002BFC85F89474D4F8D4320025B03325874A
:1085000054F8230040B17FF081FDD4F8D432B03369
:1085100044F82350C4F8BC520020F8BD40F20113C7
:10852000A0F878212B87E6E72DE9F04FDFF8B4B308
:108530008BB0DBF88CA9DAF8143013F0010902D003
:108540000BB0BDE8F08FDAF81420DAF818301A42D0
:10855000F6D0DAF808280AF50061DAF81430C2F328
:108560000D220291CBF8602EDAF8182013409D07F7
:1085700005D5DAF8143003F00203CAF81430DAF83B
:108580001430DAF818201340DC061BD5DAF818305E
:1085900023F01003CAF81830DAF8203003F4F01290
:1085A00003F00F05B2F5802F00F04985B2F5402F9A
:1085B00000F02583CDF804A0019A936943F01003DD
:1085C000936101E0CDF804A0019A536992691340C8
:1085D000180300F19C82019A5369926913405F036A
:1085E00000F1D281019B5A699B691A4200F1EA802D
:1085F000019A5369926913401B0509D5029B9B6838
:10860000DF0700F16485019A536903F40063536145
:1086100001994B698A6913401E0116D54B6903F015
:1086200000634B619BF8583E002B00F0C282DBF8E0
:108630006C3E93F89C22042A04D093F89C22D2B278
:1086400083F89D22042283F89C22019A536992693F
:108650001340DD0400F14881019A53699269134087
:108660009C0400F1D780019A53699269134019075D
:1086700000F1C38001994B698A6913401A067DD4C1
:108680004B698A691340DB0228D59BF89089B8F1C1
:10869000010F1ED9924D0AF51267012604E001363A
:1086A00020372435464514D095F83C303A68012BE4
:1086B000F5D1002AF3DA66F07F0085F83B30C0B2CE
:1086C0006DF0CEFDEBE7019A536992691340DA022F
:1086D00004D5019A536903F480135361019A5369D5
:1086E000926913409F0231D59BF89079012F28D9C8
:1086F0000AF532627A4B012103E0B94203F1240307
:108700001FD093F87C020131146820320128F4D183
:10871000002CF2DADBF8605E85EA1445EE07ECD453
:1087200083F87B02DAF8180040F08000CAF81800DD
:10873000DAF814000506E0D4029A536843F4007393
:108740005360019A536903F400135361019A53690A
:10875000926913405C0000F1BD8001994B698A6900
:10876000134058077FF5ECAE4C68610700F1BF84F9
:10877000DBF88C395A6814435C60E1E6DAF81830AB
:108780009BF8908923F08003B8F1010FCAF81830E4
:1087900099D9534D01262F4603E00136243746452B
:1087A00007D097F87B32012BF7D1F0B26DF058FD6E
:1087B000F3E7019B5A699B691340DB028ED59BF856
:1087C000908968E7029A536823F0010353609BF88D
:1087D000583E012B00F00182DBF86C3E93F89C229E
:1087E000042A04D193F89D22D2B283F89C22019AE4
:1087F000536903F000435361FAE6DBF86C0E90F81E
:108800009C32032B00F0ED81019A536903F00803B9
:1088100053612FE7019AD2F800396FF30A03C2F8C7
:10882000003902F50063D2F8042842F480725A60DD
:108830009B68980700F1F78113F0060F0CBF002327
:108840000F238BF89339F9F74DFA9BF89369022EB1
:1088500000F06F844FF410530199003EDBF86C5E1A
:10886000CA6818BF012622F47052CA60CA6813434E
:10887000CB600123002185F89C32D5F8B8326960BD
:10888000C5F8A41285F8A012C5F894121BB15B6854
:108890000BB1284698470022402401274023114667
:1088A000284674F043FF2346002280212846C5F85D
:1088B0006041A5F8647174F039FFDBF86C3EDBF8B9
:1088C0008C29AF842C621E745369019203F4005307
:1088D0005361C8E6019A536903F0804353613CE752
:1088E000AC41002420380024029A102101985368DA
:1088F00023F001035360FAF761FB9BF89009E0B1A4
:108900000AF510634FF67F31996009F101091A6881
:108910002033814522F4001243F8202CC3F8E811DB
:10892000D3F8E02122F40012C3F8E021D3F8E021CB
:1089300042F00062C3F8E021E6D1029AD36943F025
:108940000113D3619BF89B39002B00F03B81029A05
:10895000D2F8843043F00B03C2F88430536C43F0F8
:108960000B035364DAF80038019C23F4FE63B44A25
:108970002046CAF800389BF8921974F059FF6369D1
:1089800003F48053636167E6019AD2F81878D2F84D
:108990001C381F40BFB2002F3FF424AE0AF510610F
:1089A0004FF00008CDF80CA01346A64D44468A4669
:1089B000CDF8109008E07F0804F1010405F12405CA
:1089C0000AF1200A00F03181FE07F4D5D3F810280F
:1089D00004F00F01D3F834684FEA4419CE40F60191
:1089E000F6B2164303F5106202EB44129268164089
:1089F000E2B2F007019221D50120029ADBF86C8ED9
:108A0000526B00FA01F122EA010202994A639BF8D3
:108A10009219CAF80800814200F078832B6A059306
:108A2000002C40F0FA82D8F89432022B00F0E88350
:108A300098F8A03213B1002388F8A032320702D58B
:108A40000823CAF80830F30602D51023CAF8083004
:108A5000700602D54023CAF80830B10700F1108132
:108A60003206DBF88C39A6D5D5E909068642A2D8AC
:108A7000811BEA6903F5106E8A42CE4428BF0A467C
:108A8000DEF81810033289B2B1EB920F31D39BF8A4
:108A9000928903F5805C019442460CEB043C9846B5
:108AA0001346B04240F29083811BEA69914228BF8D
:108AB00011462A6A01F103094FEA990973B98CB288
:108AC0000334A4080AD002EB840452F8040BA24237
:108AD000CCF80000F9D12A6AD5E909060A440E4407
:108AE0002A62DEF81820AE6292B29145D9D9019C73
:108AF0004346B0423FF65FAF04F00F0201219140C0
:108B0000D3F8342822EA0102C3F8342853E7019845
:108B1000D0F81838D0F81C2813405FEA13483FF407
:108B20005AAD484B0AF53066CDF80CA000279A469E
:108B3000CDF8149008E05FEA580807F1010706F144
:108B400020060AF1240A74D018F00109F3D0FBB210
:108B500000F530627D01019302EB47139C68D0F869
:108B600014180C40E1076FD4210700F19580E50649
:108B700001D51023B360A0070FD5039B5B691906CD
:108B800004D5029A536843F4806353609AF85732CD
:108B9000012B00F01C830223B360A20601D5202321
:108BA000B360A30402D54FF40053B360DBF88C0923
:108BB000C1E701238BF8583E4B6DC3F38303CBF819
:108BC0005C3E42E5029942F22B034A6913434B6132
:108BD0000B6943F00B030B61C4E600238BF8583E8E
:108BE00005E6D0F8B832002B3FF40EAEDB69002B5F
:108BF0003FF40AAE9847DBF88C39019304E605EBA5
:108C0000C5020AF58051C3F30A130BEB8202D2F8B6
:108C1000F40B03440868CBF8280E0968C2F8F43B4B
:108C2000CBF82C1EC6E402230BE6DDE903A9019371
:108C3000D8E4DDF80CA0DDF814900190CBE400BF7F
:108C400048460024AC4100240121B1609BF89219F0
:108C5000D0F840E00129D3F808C000F0A582B64959
:108C60008E4500F09B83DBF8F03B3B4300F04984EA
:108C7000DAF860220199DBF86C0E75F00BF873E7F7
:108C800021460398FAF79AF9EB7D012B00F09183C6
:108C90000223CAF80830E3E6DBF88C290823B36026
:108CA00002F53063126C2B4410460492A34A996873
:108CB000904204D90A0402D54FF400429A60DBF8CE
:108CC0006C5E01219BF8283E05F2AA2085F8AA32A5
:108CD0009BF829EE079085F8ABE2BBF82A2EA5F8A1
:108CE000AC22BBF82CCE0692A5F8AEC2BBF82E2E55
:108CF000C5F8941203F01F01A5F8B0220129C5F8A8
:108D0000982200F0A582022900F00783002940F094
:108D1000DE8203F06003202B00F0E983402B00F09B
:108D2000E683A3B9BEF1090F11D8DFE81EF0E80011
:108D3000C1001000D80010007D00640010003E004B
:108D40002300D5F8B4325B69002B40F0C285284679
:108D500074F030FE794B049A9A427FF608AF9BF884
:108D6000921901297FF403AF754ADBF88C0974F07E
:108D70005FFDFCE69DF81890B9F1010F8BF8709E2D
:108D8000E5D895F89C32DAB2022B069200F0038502
:108D9000032A00F0D784284674F00CFED5F8B832C8
:108DA000494628465B689847D4E7012ACFD195F811
:108DB0009C120229CBB200F2A684002BC7D0D5F8B2
:108DC000C832002128464FF0020C40F8081FC5F8B1
:108DD00094C2C5E90622C3E9092118624FF48072E2
:108DE00003F114019A829A79012A08BF186318685E
:108DF00074F01AFEAEE7069B00221B0AADF826208F
:108E0000013B062BA3D801A252F823F0ED8F0408F2
:108E1000D18F0408A78F04084F8D04084F8D0408D4
:108E2000458F0408FF8F040852EA0C0C8FD1069B73
:108E30007F2B8CD895F89C32032B88D00698D5F8D8
:108E4000C8325FFA80F985F89E9293F89424012A3B
:108E500012D01A684FF0000C83F81190D2F8001865
:108E600021F4FE61C2F80018D2F8001841EA00119E
:108E7000C2F8001883F894C40422002003F11401FE
:108E8000C5F894224FF48072A8619A829A79986208
:108E9000012AC3E9080008BF1863186874F0C4FD0C
:108EA000B9F1000F40F07284012385F89C3251E73C
:108EB00095F89C32013B022B3FF649AF069B012BF4
:108EC0007FF448AF0020D5F8C832C5F8A402A861E5
:108ED0000422C5F894229862C3E908007EE7069B45
:108EE000012B00F06F84069B022B7FF430AF4FEA1A
:108EF0001C2CD5F8C832002085F8A0C2E7E795F809
:108F00009C32013B022B3FF622AF022A7FF41FAFB7
:108F1000D5F8A4322846002B18BF4FF0030940F8BB
:108F20000C9FD5F8C832C5F89422C5E90622C3E9DA
:108F3000080200229A6251E70A31544F0A30544F16
:108F4000484600242B7C002B7FF401AFD5F8B832C3
:108F50000DF126005B6B98470346B5F8B002002878
:108F600000F03884BDF82620002A3FF4F0AE82429B
:108F70004FF0020128BF0246D5F8C802C5F8941286
:108F800000F11401C5E90622C0E90832002282621C
:108F90004FF4807282828279012A08BF03630068DD
:108FA00074F042FDD6E69DF8180005283FF6CFAED6
:108FB00001A353F820F000BF0B990408FD980408A2
:108FC000EF980408E1980408438D0408C798040842
:108FD0002A7CD5F8B832002A40F072849B6A0DF1E1
:108FE00026009847022203464270B6E7D5F8B4320D
:108FF0000DF12601287C1B6898470346ADE72B7CC2
:10900000002B7FF4A4AED5F8B8320DF126001B6B0F
:1090100098470722034642709FE798F89C32032B3B
:109020007FF40CADD8F8B8325B69002B3FF406AD85
:10903000002240460199C8F8D4229847FEE447F63A
:10904000F07213423FF4B6AA05EBC502C3F38814CD
:109050004FEA131CC3F301130BEB8202EE00D2F8AC
:10906000EC7B002C00F000830AF5805E002239467C
:109070000132DEF80000944241F8040BF8D107EB0E
:109080008404002B00F0BC810AF580522344106850
:10909000002220FA02F1083204F8011B9C42F8D1A8
:1090A00073190BEB8303D3F8EC7BDBF88C3901935A
:1090B0007319CCF30A0C0BEB83036744D3F8F42B3E
:1090C000C3F8EC7B6244C3F8F42BFFF775BADBF806
:1090D0006C3E93F89C22042A04D093F89C22D2B2CE
:1090E00083F89D22042283F89C22FFF78CBADBF8D8
:1090F0006C0E0122D0F8B83280F89C22002B3FF48D
:1091000037AB5B6801799847FFF732BBD5E90702B7
:1091100002442A62002C80D1DBF8AC09DBF8B029CC
:109120000590002A7FF47FAC1846B74A74F080FBA4
:1091300079E4B64BB64A0344934240F25281B54BB0
:10914000B54A0344934240F25781B44BB44A0344B6
:10915000934240F23582B34BB34A03449342C0F08A
:109160006B82B24BB24A0344934240F29182B14BBC
:10917000B14A03449342C0F08F82B04BB04A0344DB
:109180009342FFF467ABAF4BAF4A03449342C0F046
:10919000D582AE4BAE4A034493422CBF4FF4C0532A
:1091A0004FF4E053FFF758BB1CF0080F00F01D818F
:1091B000A84A96457FF6D8AC1CF4004F3FF4D4ACD7
:1091C0004FF400429A60CFE4019C434694E40023AC
:1091D0008AF85732DBF86C0ED0F8D432AE3350F840
:1091E0002330002B3FF4D7AC90F89C22032A7FF465
:1091F000D2AC5B6A002B3FF4CEAC01999847CAE42D
:10920000D8E90732934200F2278100F0988198F85C
:109210009C32032B00F0C8818021404674F08EFB05
:1092200005230020C8F89432D8F8C8329A7903F59B
:109230001571C3F86802012AA3F85402C3E9980023
:1092400008BFC3F87002186874F0EEFBFFF7F0BBBC
:1092500003F060025B0602D5402A7FF478AD95F8F2
:109260009C32013B022B3FF672AD5FFA8CFCBCF1E5
:10927000030F3FF66CADD5F8B8329B68002B3FF476
:1092800069AD4FF0000907992846C5F8D492984770
:10929000B5F8B022002A7FF45DAD00287FF45AAD06
:1092A0000422D5F8C832C5F81890C5F894224FF4B6
:1092B000807203F11401C3F828909A829A79012AE6
:1092C000C3E908997FF493ADC3F830908FE51B068E
:1092D000D5F8C85200F12D81002385F8553205F5E7
:1092E000157301224FF000099A7083F8009095F8E9
:1092F000941491423FF42EAD286885F894245A784E
:109300001978069074F0E0FA069805F29C42A97963
:1093100074F08EFA85F894941CE503F06003202B1A
:1093200000F07C81402B00F07981002B7FF40FADA1
:10933000BEF1010F5FFA8CF100F04681BEF1030F20
:1093400000F07E81BEF1000F7FF401AD95F89C32F4
:10935000022BDAB200F0A481032A7FF4F8AC01F00A
:109360000F0314221CF0800F02FB035340F0B28164
:10937000B3F86431002B3FF4EAAC02FB015202F572
:10938000AA70002940F02B8200230360D5F8C83270
:109390000222C5F89422C5E90622C8E51CF4004F54
:1093A0007FF40EAF1CF0200F3FF462AC20229A60D5
:1093B0005EE40023EB75DBF86C0ED0F8D432AE33EC
:1093C00050F82330002B3FF463AC90F89C22032A22
:1093D0007FF45EAC1B6A002B3FF45AAC01999847AE
:1093E00056E44FF47053FFF737BA1CF0200F60D0EB
:1093F00020229A60FFF7B8BB4FF46053FFF72CBAF6
:10940000CDF804A054E600BF48460024405327FF8F
:10941000FF340C00401E1BFF3F420F0000DC0BFF1F
:109420007F4F1200808CF9FE20D6130060B6E5FE57
:109430005FE3160000D3CEFE40771B00C05BB3FE97
:10944000C091210000CA91FE20753800E05459FEF9
:10945000E09C41000A30544F9A1AD8F8C832C8E943
:1094600006225A6203F11401059A1A6200229A62D6
:109470004FF480729A829A79012A01D10598186373
:109480001868CDE9050374F0CFFA069B00209A799D
:1094900003F51571C3F86802012AA3F85402C3E961
:1094A000980008BFC3F87002059874F0BDFAFFF782
:1094B000BFBAC64A964503D91CF4004F7FF480AE6C
:1094C0001A69DAF87432C2F312029B1ACAF86832C7
:1094D000002F7FF4CDABDBF8F02B002A00F0D28018
:1094E000DBF8EC2B1A44CBF8EC2BFFF7C1BBD5F81B
:1094F000D43228460799AE3355F823309B689847F5
:1095000028E4016CB14B994203D91368002BFFF694
:10951000AFAB00231361136943F400231361136994
:1095200043F018031361136943F0C0431361FFF75D
:109530009FBB4FF001036B7505F11403D1E6D8F81A
:10954000182093423FF663AED8F898329A42BFF49F
:109550005EAED8F8C83200204FF48072C8F8180008
:1095600003F114019A829A799862012AC3E90800EA
:1095700008BF18631868CDE9050374F055FA069B17
:109580004FF0000C059803F51571C8F898C29A7948
:10959000C3F868C2012AA3F854C2C3E998CC7FF487
:1095A00053AEC3F870C24FE6D8F8B832DB68002B70
:1095B0003FF432AE00224046C8F8D42298472BE64A
:1095C0004FF45053FFF748B995F89C32022BDAB2AA
:1095D0004CD0032A7FF4BBAB069B002B7FF4BAABC5
:1095E0004806D5F8C89240F006810422002309F10C
:1095F0001401D9F80000C5F894224FF48072AB61D1
:10960000A9F8142099F80620C9F82830012AC9E9D8
:10961000083308BFC9F8303074F006FAD5F8B8320C
:1096200000229B68C5F8D422002B3FF493AB079926
:1096300028469847FFF78EBB4FF44053FFF70CB90D
:1096400095F89C32022B5FFA83FC0FD0BCF1030F1C
:109650007FF47DAB480603D0069B134300F0C78020
:10966000D5F8C832002032E43C460AE54B062846CD
:109670003FF46EAB74F062F92846802174F05EF915
:10968000FFF768BB524A012174F0D2F8FFF7F0BA35
:109690004FF43053FFF7E0B84FF42053FFF7DCB836
:1096A0004A067FF454AB1CF0800FD5F8C8324FF057
:1096B00002024FF0000114BF05F1140005F5AA7075
:1096C0000160C5F89422C5E90622C3E909211862A0
:1096D000FFF784BB9B8C002B3FF439AB01F07F017B
:1096E000481C00EB800005EB800000293FF44CAEE5
:1096F0002422D5F8C83202FB01318A7D003A18BF16
:109700000122026044E6032B7FF421ABD5F8C83276
:109710000221C5E90622C5F8941204355A620022D6
:1097200003F114011D629A624FF480729A829A7951
:10973000012A7FF45CAB1D63FFF759BB4FF4005364
:10974000FFF78AB8B9F1000F00F0AE80696801290F
:1097500086D0D5F8B832C9B228465B6898479BF8DE
:10976000701ED5F8B8326960002B3FF479AF1B68E2
:109770002846984700283FF473AF284674F01AF93A
:10978000D5F8B832297928465B689847022385F8CE
:109790009C32FFF7DFBAB9F1000F3FF481AD012130
:1097A000D5F8B8326960002B5AD01B682846984714
:1097B000002855D0284674F0FDF8069B85F89C32A9
:1097C000FFF7C8BAC5F8A4324AE700BF0A30544FC1
:1097D00048460024D5F8C832A861FFF779BB242297
:1097E000D5F8C83202FB013191F8562286E72846A7
:1097F00074F0A4F834E701F00F0199F804308B42BB
:10980000FFF4F3AE01EBC1031CF0800F4FEA8303BA
:1098100041D103F51573002209EB030C242303FB4C
:10982000019383F855224FF000038CF800108CF858
:10983000023099F89434012B3FF4D7AE0123D9F8C4
:10984000000089F894349CF804309CF801209CF8BE
:10985000001074F013F84FF0000389F89434C4E654
:109860000422D5F8C8320020C5F894224FF4807243
:10987000A86103F114019A829A799862012AC3E9D6
:10988000080008BF1863186874F0CEF8032385F841
:109890009C32FFF75FBA1433012209EB030C242337
:1098A00003FB01935A75BEE7022349462846C5F8D3
:1098B000049085F89C32D5F8B8325B689847EFE49D
:1098C000DB6AFFF78CBBD5F8B4329B69002B3FF401
:1098D0003EAA0DF12601287C98470346FFF73DBBC1
:1098E000D5F8B4321B69002BF3D1FFF730BAD5F8A5
:1098F000B432DB68002BECD1FFF729BAD5F8B432CB
:109900009B68002BE5D1FFF722BAD5F8B4325B682B
:10991000002BDED1FFF71BBA2DE9F8434B4BD3F8F0
:109920008C53EE682C69A70701D5B00736D46107C0
:1099300001D572072AD4270701D530071ED4E106C6
:1099400001D5F20612D4E70701D5F0073BD414F491
:10995000025F2BD031066FD4600601D5710671D439
:10996000A20601D5B30629D4BDE8F8836FF0100232
:109970002A610022E96983F8A823E4E76FF008026E
:109980002A610022E96983F8A823D8E76FF004026E
:109990002A610022A96983F8A823CCE76FF00202AC
:1099A0002A610022A96983F8A823C0E7E305D3D57B
:1099B0003706D1D56FF480732B61CDE76FF02003AC
:1099C0002B61BDE8F883224B6FF001029D422A61B2
:1099D000BDD1DFF88C801F4BD8F800201F68BA4239
:1099E000B5D01D4888BFC2F580571C4B98BFBF1A21
:1099F0001A44D0F8D432B03350F82330002BA6D01C
:109A0000D3F81492C3F80822C3F81072B9F1000F0A
:109A10009DD10121C762C3F814123B46812174F025
:109A200013F9D8F800301F44B7F5805F14BF3B46E8
:109A30004B46C8F800308AE76FF40253E2052B6109
:109A40008AD5B7E76FF040032B6189E720380024FF
:109A50000014004068310024882E0024945600240D
:109A6000643100242DE9F84F234B81468A46D3F810
:109A7000BC32D3F81422002AFBD1BAF1000F37D040
:109A800009EB0A031D4E09F1FF39DFF8788003F175
:109A9000FF3B7027326819F8011F531C1848C3F3A5
:109AA0000B0381543360EFF3118287F31288D8F8E7
:109AB0000030D2B2316882F311888B42A3EB0103EC
:109AC0008CBF0022012203EB0233012B0ED10AF0DE
:109AD000DBFB04460D460AF0D7FB001B61EB0501DA
:109AE000B0F57A7F71F10001F5D3DCE7D945D1D12A
:109AF0005046BDE8F88F00BF882E0024683100244E
:109B0000945600246431002402784368022A0FD05E
:109B10000B490269D1F87C02023A184010B4400A9D
:109B2000D1E99C1404FB02005DF8044B0844704723
:109B3000034AD2E9992102EB410202EB532070471C
:109B4000203800242DE9F04F83B002F00207844D45
:109B5000019308B9002F6AD1D5F86C42002C53D17B
:109B60004FF0FF3E7F4C4FF0000CF146F046F246BE
:109B7000E36994F82A60984200F0A080002E3BD060
:109B8000012E05EB0C1B0AD19BF88B60F30706D462
:109B900016F07E0F03D1F60900F09380E0460CF139
:109BA000010C1034BCF1080FE2D1BEF1000F04DA51
:109BB000B8F1000FC0F29780C646D5F8FC400EF110
:109BC000020605EB0E18013405EB061CC5F8FC4037
:109BD0000CF1600CCCF80440C8E91F040024CCF858
:109BE000084005EB061494F86A40042C1FD8DFE8FF
:109BF00004F029441A444600E6460CF1010C1034E6
:109C0000BCF1080FB4D1D0E7D5E99C3606FB04348B
:109C1000A042A5D395F8183213B9012385F818325C
:109C2000012385F86130002003B0BDE8F08F95F87E
:109C30001832002B53D00123022085F8613003B085
:109C4000BDE8F08F12F00104D5F878C073D105EBB0
:109C50000610019B4FEAE20C90F86B80032B6CF32B
:109C6000C71880F86B8064D94FF6FF70834228BF15
:109C7000034605EB0610A0F86830002F45D15007C9
:109C800007D505EB061090F86B3043F0010380F820
:109C90006B30D3060AD505EB061696F86B30C3F386
:109CA0004502013262F3460386F86B30AB6F012048
:109CB00003EB4E230B6003B0BDE8F08FC6B9E64658
:109CC0007BE7666A1034B24588BFE1460CF1010CAF
:109CD00088BFB246BCF1080F7FF44AAF65E70123A5
:109CE00085F81832A7E7B9F1000F9CDBCE4664E790
:109CF000D5F8FC400CF10206E646013405EB061CE3
:109D0000C5F8FC40CCF864406BE7D5F80001D5F805
:109D1000FC3001300133C5F8000105EB0E10C5F829
:109D2000FC30C0F8803005EB0613042083F86A008D
:109D3000A5E723469DE7D5F88832002B3FF473AFA3
:109D40005C680CEB4E210023074AA04700283FF433
:109D50006AAF05EB0616022386F86A3063E700BF98
:109D600020380024803800242D66040870B5114D79
:109D700082B00E4695F86030022B16D1020AC4B2AA
:109D8000D5F86402002301A910440322FFF7DAFE8C
:109D9000012808D195F86030019A022B0CBF22F8F7
:109DA000146042F8246002B070BDC0F3D41200F019
:109DB0007F04E5E7203800242DE9F04F444E0D469E
:109DC00083B0174696F860102B6803293ED002290D
:109DD00061D14FEA13294FF4807A5FFA83F8421E6B
:109DE000012A23D84FF0010B9F421AD901288CBFBA
:109DF00000240124D6F8DC211AB1D6F8F8119942D2
:109E00004CD0D6F864020023092201A94844FFF788
:109E100099FE012823D0022814D020B12B689F423C
:109E2000E8D803202F6003B0BDE8F08FB8F1000F31
:109E300013D096F8183213B9012386F8183201238B
:109E400086F86130022003B0BDE8F08F4FF0800A41
:109E5000C3F3D41903F07F08C1E7D346C4E796F8EB
:109E60006010022913D00329ECD1019B53F828205C
:109E700022F07042B2FA82F22B685209A2421FD03D
:109E8000D8445B44D0452B601DD20229EDD1019B03
:109E900033F81820EEE74FF4807AD9E7D6F8741239
:109EA000013A02EB41224902B2FBF1F21344B3FB47
:109EB000FBF20BFB12320AB15B449B1A2B60AEE73C
:109EC0009F42B0D8ADE709F101094FF00008A6E7BD
:109ED000203800242DE9F04FDFF884918B4685B0BF
:109EE000174699F860C00968BCF1020FD9F86452AE
:109EF00040F08280CEB24FF4807305EB1125A6EBC3
:109F0000010890449844B94208F1FF38B8FBF3F8CF
:109F10004AD200F00103A8446FF0404A0193BCF11B
:109F2000030F07EB0604A8EB0503284614BF4FF404
:109F300080728022641A03A9944228BF1446944276
:109F400028BF002E14BF012200220A32FFF7FAFDBB
:109F500001282AD199F860C0DBF800E0BCF1020FBB
:109F60000EF1010324D0B44255D9039806EB0A023E
:109F7000011F00EB820201EB840142F8043F8A4298
:109F800003F10103F9D1DBF80030A11B19448F4222
:109F9000CBF8001002D1019B002B48D18F4205F174
:109FA00001054FF00006BAD8012005B0BDE8F08FDA
:109FB000B44246D903986FF00042811E324401EB4F
:109FC000440100EB420222F8023F914203F10103F7
:109FD000F9D1A11B71448F42CBF80010DED1019B57
:109FE000002BDBD086466FF000434FF6FF72012056
:109FF00023442EF81320D8E701F07F06C1F3D413D1
:10A00000BCF1030FA6EB01081D4414BF4FF480738D
:10A010008023904476E7AEEB060E0EEB04018F42F0
:10A02000CBF80010BAD1019B002BB7D003986FF08A
:10A0300040434FF0FF32234440F82320DBF8001068
:10A04000ACE7AEEB060E0EEB04018F42CBF800102E
:10A05000A4D1019B002BA1D0DDF80CE0C3E700BF29
:10A060002038002430B50446C06983B010B90120FF
:10A0700003B030BD0D460023032201A9FFF762FDA6
:10A080000128F5D1B4F92020002A19DB019B012D0C
:10A090004FEA421103EB421203D0022D1BD1E520FF
:10A0A0005854A368D3612378032B04D1002313777A
:10A0B00053779377D377636A190C53839182D6E7EA
:10A0C000064A92F8181209B982F8180201230220F0
:10A0D00082F86130CCE7E368E4E700BF2038002471
:10A0E0002DE9F041044682B00D4694F83C30042B33
:10A0F0007ED8DFE803F02B0369493A003D4E4FF666
:10A10000F777DFF8F48016E0BA425BD86AF0D6FF42
:10A1100001284FF0000134D1206BFFF727FE012802
:10A120002FD1019AD6F87812531E22638B4228BF92
:10A130000B46C6F8783296F8602001A9236B032AF3
:10A1400018469AB2E0D14345E0D93BE06900204689
:10A1500001F0FE01FFF786FF01283FD1636B002B62
:10A1600018BF022084F83C00BFE794F82830042B85
:10A1700002D1002384F82830A36B0BB12046984706
:10A18000012002B0BDE8F0811A4E0021E26AD6F843
:10A19000F83106F5EA70C6F8F8219B1AD6F8742251
:10A1A00002FB03F3D6F8DC2102EB4322C6F8DC21E4
:10A1B000D6F8E02102EB4322C6F8E021FFF752FF78
:10A1C00001280BD10420CDE7626B04F1300100209F
:10A1D000FFF780FE012801D10320C3E70228D0D178
:10A1E00094F82830042BCCD1002384F82830C8E719
:10A1F0000220F5E720380024F7FFFF0F38B50446AA
:10A2000094F83430052B60D8DFE803F031251D13B6
:10A210000D0394F82830082B3FD02D4B012202204B
:10A2200083F8192238BD94F82830082B30D001204B
:10A2300038BD00212046FFF715FF012845D1042035
:10A2400084F83400DCE7D4E90B01FFF78FFD012827
:10A250003BD10320F4E74FF0FF31206BFFF786FD81
:10A26000012832D1E36A002BF3D00220E8E7184D31
:10A2700004F130010120D5F86C220232FFF79CFD79
:10A28000012813D00238C0B201281ED80520D7E714
:10A290000023012084F82830CAE70023012202208D
:10A2A00084F828300A4B83F81922BBE7E368D5F815
:10A2B0007412226B03EB4123C5F87822C4E9033200
:10A2C000E36A002BBCD16262BAE7002038BD00BF50
:10A2D00020380024F8B5044694F83830032B4CD8C5
:10A2E000DFE803F021180B0200212046FFF7BAFE39
:10A2F000431EDBB2012B41D9F8BD0120626B04F192
:10A300003001FFF7E7FD01284FF00303F0D184F897
:10A310003830E1E700211E48FFF7A4FE01284FF086
:10A320000203F4D0E4E71B4BE66893F86020D3F80F
:10A330007412032AD3F8DC51D3F8F80114BF4FF498
:10A3400080728022206102FB01F1871A0244A5EB92
:10A35000412506EB4126E660C3F8DC51D3F8E05115
:10A36000C3F8F821A5EB4121C3F8E011E36AC4E981
:10A370000C025BB960620123C9E7022094F828301F
:10A38000062BB9D1002384F82830F8BD2763F2E703
:10A39000F4390024203800244368C3F308020A4437
:10A3A000B2F5007F2DE9F041054682B00C4605D29A
:10A3B00023446B60012002B0BDE8F08190F91A10CF
:10A3C000481C0AD0474A02EB011292F88B1021F088
:10A3D000010182F88B10FF22AA7695F91B20511CEF
:10A3E00016D0404E023206EB021191F86B10C1F309
:10A3F0004501012944D9013901F03F0106EB021260
:10A40000FF2692F86B0061F3460082F86B00EE764F
:10A410002A78022ACCD0334ED6F87422B4EB422FDD
:10A420004FEA42282EDCD6F87C721F407A42A242C4
:10A4300028DCE2192869424513D32A7E12072DD55C
:10A44000D6F8F821411C8A421ED300D10021434492
:10A45000A4EB080868610846DB1B08EB07042961C8
:10A460006B600028A6D096F86020032A35D080B211
:10A470004FF6F77290429DD81A4614446C6099E7E3
:10A480000021BBE7002096E796F818220ABB0123BB
:10A4900086F8183286F861306B68D8E701A96AF04F
:10A4A0000DFE0128EED16B68A4EB080428699844DE
:10A4B000297868613C44A8EB0703019802291A46F1
:10A4C0006B602861CDD1D6F88412B3EB412FD4D381
:10A4D00070E7012286F86120B9E7034A90423FF60F
:10A4E00069AFC9E720380024F7FFFF0F2DE9F047D7
:10A4F0004FF0010882B0044694F83830032B00F284
:10A50000A680DFE803F055170C020020236C84F8C6
:10A51000280003B19847022002B0BDE8F08700226E
:10A52000236C84F828200BB120469847012002B004
:10A53000BDE8F08723786768022B03D0454BD3F83A
:10A540007C321F40C7F34F272046FFF7DDFA414E0C
:10A550003F1A0546BFB207EB050C022201A90023F2
:10A5600028461FFA8CF9FFF7EDFA01284FF4007224
:10A570004FF00001D0D101987DF020F9E3694FF44C
:10A58000007120460BB16368EBB1D6F874325A1EE5
:10A59000914547D20135FFF7FFFE0028DBD196F841
:10A5A000183213B9012386F8183286F86180D2E791
:10A5B0002046FFF723FE012802D0022847D10320BE
:10A5C00084F8380098E7019B4FF020324FF0100ECE
:10A5D0004FF02E0C42F62E6AC3F80120C3F8052076
:10A5E000A3F8092083F800C0D4F824C0A3F820A061
:10A5F00083F80BE0C3F82220C3F8262083F82A2032
:10A60000E26BA3F81AC02CFA0EFC5A8722FA0EF25B
:10A61000A3F814C09A8683F82BE0D6F874325A1E39
:10A620009145B7D3C3EBC3532046590201F50071DE
:10A63000FFF7B2FE28B996F8183223B1012386F845
:10A6400061300220BCE7012386F81832F6E70020CB
:10A6500062E700BF20380024B1F904300F2B2DE948
:10A66000F0410D4682B00446164632D02046FFF730
:10A670004BFA94F91B80B8F1FF3F3BD05B4F07EBDF
:10A680000813DB6F984212D097F81832002B6ED067
:10A69000012387F861302378022B5ED02269002ADB
:10A6A00073D100230120336002B0BDE8F081B96F9F
:10A6B00001EB4821002966D0AB88204601331BB24C
:10A6C00001EB4311AB803160FFF71EFA28600120D7
:10A6D000EAE74FF40071FFF75FFE002843D04FF622
:10A6E000FF732046AB80FFF70FFA94F91B80B8F197
:10A6F000FF3FC3D12378022B3DD02269002AD0D05E
:10A700003A4F97F86030032B66D093B24FF6F7714B
:10A710008B4294BF00230123002BC0D130B997F89E
:10A720001832002B4BD0012387F86130002311220F
:10A7300001A9FFF707FA012825D10199BB6FCB1AB0
:10A7400048BF03F2FF13B3F5805F4FEA63222CD2B8
:10A750004FFA82F884F81B80ACE7D7F8842263684C
:10A76000B3EB422F9DD2002002B0BDE8F08101235F
:10A7700087F818328CE71D4F6368D7F88422B3EB53
:10A78000422FCBD38DE7237886E797F86030032BF1
:10A7900019D093B24FF6F772934294BF002301236E
:10A7A000002B7FF47EAF0020DEE797F8183213B954
:10A7B000012387F81832012387F86130CAE70123A3
:10A7C00087F81832AFE70A4B9A4294BF002301235F
:10A7D000002B7FF466AFE6E7054B9A4294BF002357
:10A7E0000123002B7FF45BAF98E700BF20380024E3
:10A7F000F7FFFF0F2DE9F047044688B094F830309A
:10A80000042B11D8DFE803F0501361035A00237EB4
:10A810009A0640F1F8800023112204A9E069FFF7AD
:10A8200091F9012800F0EF8008B0BDE8F087C44D31
:10A8300003AE04F11C0705F5077932463946484650
:10A84000FFF70AFF012800F0F9800228ECD195F902
:10A8500036325F1C0AD005EB0313FF2193F88B20DF
:10A8600085F8361222F0010283F88B2095F93732F1
:10A870005E1C17D0023305EB031292F86B20C2F373
:10A880004502012A40F25A81013A02F03F0205EBEB
:10A89000031393F86B1062F34601FF2283F86B10E9
:10A8A00085F83722042306E0A6486BF0AFFF4FF689
:10A8B000FF720123228484F830309FE70020E36A8E
:10A8C000207008B0BDE8F04718479D4D95F8443218
:10A8D000002BA9D104F11C0705F5077803AE324619
:10A8E00039464046FFF7B8FE012840F01581039B2A
:10A8F000002B00F0F0801A780AB1E52AEFD1AA6F98
:10A900009A1A48BF02F2FF12B2F5805F4FEA622145
:10A9100080F0498109018C4A0A44917B04290CD0BA
:10A92000D5F8FC100131C5F8FC1051600421917379
:10A93000D5F800210132C5F8002195F93622501CC6
:10A940000AD005EB021292F88B1021F0010182F877
:10A950008B10FF2285F8362295F93722511C17D02B
:10A96000023205EB021191F86B10C1F34501012988
:10A9700040F26181013901F03F0105EB0212FF2035
:10A9800085F8370292F86B0061F3460082F86B009D
:10A990002022002118467CF011FFD4F83110034624
:10A9A000D4F8352005A819605A6094F83B20B4F813
:10A9B00039109A721981627E0193DA7203F014F9E8
:10A9C000019B002800F0D8809DF816009DF8172004
:10A9D0009DF8191042EA4012BDF814004901A0F296
:10A9E000BC7042EA40229DF81A0041EA50019DF8ED
:10A9F000180092B241EAC02188B2D9811A821A8322
:10AA0000D882032357E720466BF000FF2369002B11
:10AA100000F08780237E03F0F70213F00403227610
:10AA200040F09480122A00F0AA800022E36A2046B7
:10AA300084F8282008B0BDE8F0471847DDF80C80FE
:10AA4000B8F1000F00F0BB8098F80030002B00F048
:10AA5000B68098F80BA01AF0080F7FF4EEAE0B2228
:10AA600004F1310140467CF0BBF900287FF4E5AEEB
:10AA7000637E8AEA0303DF0640F1E18095F936320E
:10AA80005E1C0AD005EB0313FF2193F88B2085F899
:10AA9000361260F3000283F88B2095F93722511C9F
:10AAA0003FF400AF023205EB021393F86B30C3F3AF
:10AAB0004503012B40F20681013B03F03F0305EB08
:10AAC000021292F86B1063F34601FF2382F86B10B9
:10AAD00085F83732E6E695F81C320922022B3FF45E
:10AAE000E1AE95F84432002B7FF4DCAE85F85432A9
:10AAF000404685F8503285F84422C5E99633D5F8AA
:10AB00003032C5F84832D5F87832C5F84C32FFF704
:10AB1000EDFC01283FF4E3AE02287FF485AE042368
:10AB2000C9E6237E1B0780D5054B93F8FC21002A3C
:10AB30007FF47AAE072283F8FC2176E70022A6E6AE
:10AB4000203800243C3A00249C3800240023A568C7
:10AB50002046E66A294684F82830FFF71DFC0028C5
:10AB600063D194F82830002B7FF45EAE0223C4E951
:10AB70000B6584F8283057E644F281723EE7E06ABC
:10AB80000421626AA063204684F83C3084F82810CF
:10AB900063636362C4E90B22C4E9023308B0BDE811
:10ABA000F0476BF033BE95F8182212B9012285F8F0
:10ABB000182201226FF00F0185F86120ABE695F9AC
:10ABC0003632591C0AD005EB0313FF2193F88B2072
:10ABD00085F8361222F0010283F88B2095F937327E
:10ABE0005A1C16D0023305EB031292F86B20C2F305
:10ABF0004502012A21D9013A02F03F0205EB031375
:10AC000093F86B1062F34601FF2283F86B1085F80E
:10AC10003722237EDB067FF545AE2C486BF0F6FD30
:10AC20004FF6FF720223228445E6002E3FF4FCAD6E
:10AC30002046334645E600219FE60022DEE7B8F8CD
:10AC40001420B8F81A3043EA0243D5F8742263623C
:10AC50005202D8F81C30B3FBF2F102FB1131A360B1
:10AC600009B113445B1AE36084F819A095F93632F0
:10AC70005A1C0AD005EB0313FF2193F88B2085F8AB
:10AC8000361222F0010283F88B2095F93722531CEB
:10AC90003FF4B7AE023205EB021393F86B30C3F307
:10ACA0004503012B10D9013B03F03F0305EB0212D2
:10ACB00092F86B1063F34601FF2382F86B1085F85E
:10ACC00037329EE60023FAE60023EFE73C3A002401
:10ACD00010B50378044690F818C0023B012B02D946
:10ACE0001CF0060F6ED11CF0200F44D194F91A20ED
:10ACF000511C0AD03A4BFF2103EB021393F88B202F
:10AD000022F0010283F88B20A17694F91B305A1CA3
:10AD100016D03349023301EB031292F86B20C2F3D1
:10AD20004502012A4BD9013A02F03F0201EB03131D
:10AD300093F86B1062F34601FF2283F86B10E27602
:10AD40001CF0080F0ED0264991F8FC31072B06D0D5
:10AD500091F81832002B3DD0012381F86130002397
:10AD600081F8FC310023E26A237084F8283042B372
:10AD7000BDE8104010471B4A0023E069D16910323A
:10AD8000884206D00133082BB0D0D16910328842F6
:10AD9000F8D11349023301EB031292F86B20C2F38E
:10ADA0004502012A1AD9013A02F03F0201EB0313CE
:10ADB00093F86B1062F3460183F86B1096E700225C
:10ADC000B4E710BD0121FFF74DF90128F9D194F83E
:10ADD00018C088E7012381F81832BDE70022E5E7B3
:10ADE000203800248038002438B51A4C94F84432B6
:10ADF0002BB970B190F828201AB1184638BD002040
:10AE000038BD0146442204F507707AF059FC012050
:10AE100038BD04F507750146442228467CF0CEFC77
:10AE200094F8603003224FF6FF71022B2846A4F8F5
:10AE3000361218BF1346D4F8801284F83422102238
:10AE400084F81C32C4F8401284F835226BF0DEFC22
:10AE5000DDE700BF20380024304A4FF0FF31F8B55D
:10AE6000A2F1600C00230C4603E001331032082BE2
:10AE700014D092F82A000428F7D10CEB031090F8B4
:10AE80008B00C607F1D4651C106A01D08142ECD951
:10AE90001C46013301461032082BEAD1002C01DA9E
:10AEA0000120F8BD1E4DA61C05EB0613D5F888221F
:10AEB000B3F86810D9B927012F44A96FD5F88832A3
:10AEC000F86F01EB4421D3B1DC680023154AA04799
:10AED000A8B1022809D1D5F8003105EB06160122E8
:10AEE000013B86F86A20C5F800310020F8BD05EB6B
:10AEF00004132701D86F12B193689847DCE7D5F89F
:10AF0000003105EB061603210122013B86F86A1089
:10AF100085F80421C5F80031E7E700BF8038002438
:10AF200020380024916604082DE9F04390F8283079
:10AF300083B00446013B082B0BD8DFE803F0383C14
:10AF40001F2305290A2E33000121FFF7C9F8012824
:10AF500002D003B0BDE8F08300222378216C84F88E
:10AF60002820002BF5D00322E162D4E9010384F804
:10AF70002820834238BF03462046A36003B0BDE8C3
:10AF8000F043A5E6002103B0BDE8F043FFF7A8B801
:10AF900003B0BDE8F043FFF79DB903B0BDE8F0434F
:10AFA000FFF72CB903B0BDE8F043FFF79FBA03B039
:10AFB000BDE8F0431EE4DFF834914368D9F87C62C1
:10AFC000026B19461E40D9F8740294F800C0B518F7
:10AFD0004702B5EB402F41D34FF6F778BCF1020F93
:10AFE00014D025692846002D5AD16168A368002035
:10AFF000E26A8B4284F8280038BF0B46A360002A1F
:10B00000A7D0204603B0BDE8F04310476168D9F8E7
:10B010008402B1EB402F5CD22069217E090732D532
:10B02000D9F8F811451CA9422AD299F8181200291A
:10B0300043D1012389F8183289F86130226B6368A3
:10B0400094F800C0D21B3B4432449B1B002697421D
:10B05000194663602263C4E90450BFD9BCF1020FF2
:10B0600037D02569002DC1D099F86030032B36D038
:10B07000ADB24FF6F7739D42B8D811446160B5E7A1
:10B08000E0D10025DEE701A96AF018F801287FF475
:10B0900060AF2069019D94F800C06368226BD1E71E
:10B0A00099F8601003290ED0A9B2414594BF002140
:10B0B00001210029B1D06168D4E7012189F861102C
:10B0C00094F800C0BEE708498D4294BF00210121D9
:10B0D000EFE7D9F88432B1EB432FCED386E7024BAA
:10B0E0009D4283D8C9E700BFF7FFFF0F2038002437
:10B0F000704700BF90F83C20034602F0FF0012B1F9
:10B10000002283F83C207047007970470079C0F333
:10B110004010704700794009704700BF704700BF7A
:10B12000704700BF03685A1C02601970704700BF67
:10B1300003685A1C02601970704700BF024B186800
:10B1400003681B68184700BFA06600242DE9F04182
:10B150003A4E33787E2B03D000273846BDE8F08185
:10B1600008214FF4FC4341F221041AB25B00002A8B
:10B1700084EA42009BB2B8BF83B20139F5D1B6F878
:10B180000140002C37D02E4A2E4DAA42E4D2052C85
:10B19000A2F106028CBF002701271444AC4228BF4D
:10B1A00047F00107002F46D141F2210EA24214D0F0
:10B1B000501E04F1FF3810F8011F082283EA012312
:10B1C00019B25B0000298EEA410C9BB2B8BF1FFA8E
:10B1D0008CF3013AF4D14045EDD1218861B1A21D33
:10B1E000AA42BAD2052904EB01002246B5D9A842E9
:10B1F000B3D20446DAE7144C671E41F22105BC467F
:10B2000017F8012F83EA0223082219B25B000029F4
:10B2100085EA41009BB2B8BF83B2013AF5D16445DB
:10B22000EDD16788094AFF1A231DB7FA87F79B1BE0
:10B230007F09938091E70F468FE700BF0000020867
:10B24000070002080000040801000208A0660024AC
:10B250004FF40063838170470120704701207047DD
:10B260002DE9F04F734D85B00F46A868AB89009269
:10B27000C3EB2014B5F910205B00B5F918E004FB0E
:10B2800004F4B5F81280C3EBE003CDF80CE024130E
:10B29000B5F91A60B5F91C1002FB04F4B5F90E20DB
:10B2A000029602FB03F3A413B5F9142004EBE32484
:10B2B000AB6AA4F5FA300193B5F9163080FB00EAC9
:10B2C0004FEAE37B82FB002C03FB0AF94FEA0C3CBC
:10B2D0006C620EFB0B99A3FB0E3B4CEA125C120353
:10B2E000CB441B0A43EA0B639B184CEB2B2BA3FBB1
:10B2F00008320BF5004B08FB0B2B4FEAEB734FEAC0
:10B300006B0953EA6B0B00F09280029E01FB0AFA74
:10B31000019A86FB0008039EC2F5801C4A464FEA4C
:10B3200048484FEAE17948EAD0380EFB09A94004C1
:10B33000A1FB0E1E4118F1444FF000000CF0004E2E
:10B3400049EB08094EEA5C0E41184FEACC7C09EB48
:10B35000C609BCEB010C6EEB090E1CEB0C084EEBA6
:10B360000E0118EB0C084EEB01014FEA88104FEA72
:10B37000811918EB000049EA986941EB090189003D
:10B3800041EA9071800010EB0C004EEB0101890046
:10B3900041EA9071800010EB0C004EEB010174F05B
:10B3A00021FEB5F922304FEA613884464FEA503E1B
:10B3B000B5F91E204FEAE37A03FB08F94EEAC14EC5
:10B3C000B5F920000EFB0A99A3FB0E35A94403FB37
:10B3D00008F50EFB0955A3FB0E3E75445B0E4FEAC4
:10B3E000E07E43EAC51313EB0C0341EB656500FBFC
:10B3F00001F10EFB0C11A0FB0C0C6144C00C40EAE7
:10B4000041301B1845EBE1451B0A43EA056303EB9A
:10B4100002130FB11B0A3B60009B23B104EB8404B1
:10B42000803424121C60012005B0BDE8F08F002399
:10B43000EFE700BFA066002431B10A4BD3ED127ACA
:10B44000FDEEE77AC1ED007A52B1064B9FED067A28
:10B45000D3ED137A67EE877AFDEEE77AC2ED007AD4
:10B4600001207047A06600240000C8422DE9F04F7B
:10B470005E4D934685B0B5F85E30286D1B02B5F879
:10B480005CE0B5F85A40C21AB5F85830019167EB44
:10B490000707AEFB020C1B04B5F856100EFB07CCD9
:10B4A000C009B5F86060C90340EA4C604FEAEC1C83
:10B4B000C018A4FB023E04FB07EE4FEA13234CF135
:10B4C000000C43EA0E634FEA2E2E5B18A6FB021413
:10B4D00006FB07444FEAD1514EF1000E41EA4421E8
:10B4E000E41511F5FA6844F10006B8F5FA6F029612
:10B4F00076F1000630DA01FB04F60394A1FB014A61
:10B500000AEB460AA6004FEA8A09361949EA9479F5
:10B51000374C4AEB09094FEA560AB6084AEAC97A93
:10B5200046EA8976B0EB0A0A6CEB690C9E1B504622
:10B530006EEBA90E3346A045029E4FF0FF34A641A4
:10B5400025DB02FB07F7A2FB022101EB4701D20F2B
:10B5500042EA4102B8EB0208019C7CB1696EA1FB92
:10B56000033201FB0E225B0D43EAC22352151B1A64
:10B5700062EB0C02DB0B43EA42432360BBF1000F9A
:10B5800001D0CBF80080012005B0BDE8F08F40F677
:10B59000AC56039C891944F1000401FB04F4A1FB9F
:10B5A000016101EB4401F4004FEAC109341B49EA8F
:10B5B000567961EB090924184CEB090C2046B419A3
:10B5C00041EB0109A41941EB09094FEA890949EA4C
:10B5D0009479A400A41B69EB0109610841EAC971CF
:10B5E000591A6EEB690E0B46ABE700BFA06600244C
:10B5F00024FAFFFF012070470E4B10B40E4C1B685D
:10B60000A06E1B1AFA2B09D809B1636F0B600AB13F
:10B61000A36F136001205DF8044B7047E36E0022B6
:10B6200023F00403104684F87020E3665DF8044BB1
:10B63000704700BF70310024A0660024054B002233
:10B6400000210120DA67C3F88020C3F88420C3F802
:10B6500088107047A0660024104B11491A680346F1
:10B66000D1F88800121AFA2A16D8D1ED1F6A0120E3
:10B6700091ED207AFDEEE66AD1ED217ABDEEC77A32
:10B68000FDEEE77A16EE902ADA8617EE102A1A8770
:10B6900017EE902A5A8770470020704770310024B7
:10B6A000A06600240F4B70B593F88C2082B00191F6
:10B6B000AAB9D3F8905095B12B681A687AB19B68F3
:10B6C0006BB104462846984748B1019922462E6836
:10B6D00028460B46316802B0BDE87040084702B00A
:10B6E00070BD00BFA06600240B4B70B5D3F894600A
:10B6F0008EB133681A6872B19B6863B105463046F3
:10B700000C46984738B131682A46234630460968C6
:10B71000BDE87040084770BDA06600242DE9F041E7
:10B720004FF0B046D6F88050D6F888301D4012D081
:10B73000DFF828800127B5FA85F4C4F11F0408EB6F
:10B74000840307FA04F4D3F8980003689847A543E4
:10B75000C6F88840EFD1BDE8F08100BFA0660024A4
:10B760002DE9F8430D46D0E9003113448B4220D82F
:10B770000446AE18076BCAB14FF0000900F10C087F
:10B7800001E0AE4212D0E36A5A1C2344E262202A4E
:10B7900015F8011B1973F4D14146204617B9F7F784
:10B7A00081FC0746AE42C4E90B97ECD13846BDE8B0
:10B7B000F8834FF0FF37F9E738B51446002944D035
:10B7C000344B0D469FED344A93ED367AD3ED396A0A
:10B7D000B8EEC76AB3F9F420B8EEE60AD3ED377ACB
:10B7E00004EE902AB3F9F020C6EE046A93ED3A7A9B
:10B7F00005EE902AB3F9F22005EE102AB3F9EE20F7
:10B80000B3F9EC30F8EEE44A06EE102AF8EEE55A09
:10B81000F8EEE77AB8EEC55AB8EEC77AC7EE843AC2
:10B8200007EE903AB8EEC66AE6EEA45AF8EEE77A6A
:10B83000A6EE856AA6EEA57AE6EE867AA6EE870AD9
:10B84000A3EEA70A77F0A6FA28600CB3114BF6EE28
:10B85000005A9FED115AD3ED376AB3F9E220F8EEA2
:10B86000E66AB3F9E03007EE102A9FED0C6A07EEA6
:10B87000903A86EE850AB8EEC77AF8EEE77A20EEBF
:10B88000070AA7EEA50A20EE060A77F083FA2060E1
:10B89000012038BDA06600240000F04A0000C84224
:10B8A000174B70B5D3F8F86026B1164A032130461D
:10B8B000F9F708F800213046F8F730FD72680023E8
:10B8C000114915695A0101EB431401338A586A4042
:10B8D00012F47C5F07D0102BF4D100220B4BF260E6
:10B8E0007361002070BD0949F4607161237F002BF2
:10B8F000F7D1304640F62B42BDE870406AF0D0B92F
:10B90000A0660024009F2400A80000244803003003
:10B9100038B50E4DD5F8F84024B10D4A64212046C3
:10B92000F8F7D0FF00212046F8F7F8FC2046F8F79A
:10B93000B9FE2368586890F83D30012B01D172F0B0
:10B94000E1FB012385F8FC3038BD00BFA066002470
:10B95000009F240038B50409013C042C19D80F4D70
:10B9600000F00F0335F8140040FA03F212F0010260
:10B9700011D00122254402FA03F3013B18407CF068
:10B98000ABFF2B7B064A184400EB400002EB800023
:10B9900038BD002038BD104638BD00BFCC8D0C0826
:10B9A000F83B0024E0B10F4B0F4A70B506680D4616
:10B9B00082B0044633449B0A02EB4303988A69F041
:10B9C000D7FBC5F381030022A1883046CDE90032C0
:10B9D000C5F3411305F0130273F0B6FA02B070BD5F
:10B9E000704700BF0000FEA7CC8D0C082DE9F04F7A
:10B9F0005422044600218BB0AB487BF0DFFEAB4AFB
:10BA0000611EE01C144611F8013F5D1E052D88BF24
:10BA10000023884244F8043BF5D102F1100311469B
:10BA200051F8040B012800F030818B42F8D1114607
:10BA300051F8040B022800F01E818B42F8D1114608
:10BA400051F8040B032800F00C818B42F8D1114609
:10BA500051F8040B042800F0FA808B42F8D111460B
:10BA600051F8040B052800F0E8808B42F8D152F819
:10BA7000041B062900F0D7809342F8D18C4F1A2678
:10BA80004FF0000ADFF8208207F12805DFF838922E
:10BA900098F80C404CB32046FFF75CFF20B105231B
:10BAA000C6718371002303720321FFF77BFF00231C
:10BAB00002E001331C2B37D015F83320A242F8D115
:10BAC00007EBC303DC6A0123D9F8F0200621C8F88C
:10BAD0001040D0189A4488F81420C9F8F00088F86B
:10BAE000161088F8153089F8EC30013608F10C088A
:10BAF000F6B2202ECCD1BAF1000F12D0DFF8C8A1D7
:10BB00004FF0000BDFF8C481D14699F8EC306BB9E7
:10BB10000BF1010B09F1F40908F58C78BBF1030F67
:10BB2000F3D10BB0BDE8F08F0024CCE7B9F80600E4
:10BB300069F01EFBB9F8040069F01AFBD9F8F0307F
:10BB40004FF4403CF421012BC9F8283001FB0BA134
:10BB5000D9F80020D4BF002301234FF0030EC9F809
:10BB60001020C9F81C300023C9F8383089F82C306F
:10BB7000C9F83030C9F8203089F8483004930823D8
:10BB8000C9E905C34FF48063C9F834304FF48073BA
:10BB9000A9F824304FF48053C9E90FE34B6E002B12
:10BBA0007DD093689F0003D59168424B0B40936012
:10BBB0009368DE0014D4404B40491B689068B3FB87
:10BBC000F1F33F490133014041F08051916004930A
:10BBD000049B2BB1049B013B0493049B002BF9D1E4
:10BBE0009368DD001CD4F423012103FB0BA3019116
:10BBF000596E41F010015966996E41F00101996644
:10BC0000F423916803FB0BA301F00401586E00F0CC
:10BC1000100001435CD05A6E42F010025A6677E77A
:10BC200000230193ECE7274B172193F8642183F855
:10BC30004811013283F8642120E72249142491F845
:10BC4000640181F83C41013081F864010FE71D492E
:10BC5000342491F8640181F83041013081F86401A5
:10BC6000FDE61849352491F8640181F8244101303A
:10BC700081F86401EBE61349312491F8640181F8FD
:10BC80001841013081F86401D9E60E49302491F859
:10BC9000640181F80C41013081F86401C7E68B66CC
:10BCA00089F860307DE700BFA0670024F4670024B6
:10BCB000CC8D0C08C0FFFF5F00000024400D030086
:10BCC000C0FFFF6FA0660024D017002400000030E2
:10BCD000596E21F4817141F0020159669368DC07C5
:10BCE00013D4784B9A4200F0178303F580739A427D
:10BCF00000F01283744B9B68D90706D473498B6894
:10BD000023F47C1343F440338B60714B71491B68FF
:10BD1000D368194043F208030B43D36091689368DA
:10BD200001F0040103F00803194300F06182D9F81F
:10BD30001000D9F81C30012B00F05583036B23F061
:10BD40000F030363F42303FB0BA35A6E22F00302D9
:10BD500042F001025A66019A002A7FF4D9AE019A94
:10BD6000059299F86020012A3FF4D2AE8268012141
:10BD7000940789F86010816802D4CA0700F18882AC
:10BD8000F421554A554B01FB0BA14C6E224042F069
:10BD900002024A668268134043F00043836083686E
:10BDA0004F4A002BC0F2E581F4214E4B4E4C4FF42C
:10BDB000806C01FB0BA14D4803274D4D4A6E22F0CC
:10BDC000030242F001024A66D9F80820D9F80C6053
:10BDD000A24218BF9A424FF40054C9F878600CBFD1
:10BDE00001230023C9F89C70824208BF43F001037D
:10BDF0001830824208BF43F001031830824208BF66
:10BE000043F001031830824208BF43F001031830A9
:10BE1000824208BF43F001031830824208BF43F05A
:10BE2000010300F55670824208BF43F00103183049
:10BE3000824208BF43F001031830824208BF43F03A
:10BE400001031830824208BF43F0010318308242D8
:10BE500008BF43F001031830824208BF43F00103DA
:10BE60001830824208BF43F00103002089F86000C7
:10BE7000C9F89800C9E91F00C9E928004FF400601B
:10BE8000C9E921C04FF48070C9E923404FF4003064
:10BE90004C46C9F89400286844F8742F1BB9154B18
:10BEA0009A4240F0BE84F423022103FB0BA383F8E3
:10BEB000A9100021136889F8A81023F0010313606A
:10BEC0001FE000BF002002400060025800630258DB
:10BED0000010005C03C0F0FFFDEEFFFFC0FFFE3F5F
:10BEE00000F8C32510000240280002404000024034
:10BEF000802E0024B80402402B681B1A052B00F288
:10BF0000BD811368DF07F7D4A44913680868A44902
:10BF10006FF30F001940A34BB0F1005F43EA010338
:10BF20000BD32E2E40F21F833F3E132E05D89E4882
:10BF3000F040C00701D59D4B0B4313602046536969
:10BF400023F007035361F5F765FDD9F8D02002F01F
:10BF50001F013F228A408260D9F87420944B954992
:10BF6000954E8A4218BF9A4201F11801A2EB0600D1
:10BF70000CBF012300238A4208BF43F0010318319C
:10BF80008A4208BF43F0010318318A4208BF43F0D8
:10BF9000010318318A4208BF43F0010318318A4275
:10BFA00008BF43F0010318318A4208BF43F0010380
:10BFB00001F556718A4208BF43F0010318318A42E5
:10BFC00008BF43F0010318318A4208BF43F0010360
:10BFD00018318A4208BF43F0010318318A4208BF72
:10BFE00043F0010318318A4208BF43F001031831BE
:10BFF0008A4208BF43F001037049511AD1F1000C85
:10C000004CEB010C6E498A4208BF43F001036D49B5
:10C010004642A2EB010701F1140146414CEA030339
:10C02000D7F1000EA2EB010043EA06034EEB070E28
:10C0300041424EEA0303414163480B430291634985
:10C04000571A794279410B430391111A48424841EA
:10C050005F49571A0343794279415E4FBA4214BF90
:10C06000002701270B4301D1002F3BD046EA0C06E5
:10C07000029B4EEA060E039E43EA0E031E43D3B212
:10C0800030430143394300F05D831422083B01260D
:10C09000514FB3FBF2F3514A9E401A449200D9F833
:10C0A0007C30C9F8DC60802BC9E9352700F00881B5
:10C0B000D9F87830D8B2013B072B10607E6000F2CF
:10C0C0000481461E002900F06285454B4549034422
:10C0D0009B0001220020B240C9E93831C9F8E820AC
:10C0E00018604A60F423012100204FFA8BFE03FB05
:10C0F0000BA30A460295C3F8C80083F8A91009F1FA
:10C100001003C9F85C40C9F8AC30374B04E0013289
:10C110000C33072A00F00A81597D0029F7D093F9E2
:10C120000D107145F3D1002101989D7D06912F4995
:10C13000039501EB80011869D1F8084199F8601066
:10C1400001293FF4E5AC4FF0010189F86010D9F8FE
:10C1500010108D686F0740F10F81F42303FB0BA3D0
:10C160005A6E42F020025A664FF0000389F86030A0
:10C17000CEE4059B01330593059B9342FFF40FAE7C
:10C18000F422002102FB0BA2536E23F0120343F0B2
:10C190001003536689F86010BAE400BF0010005C19
:10C1A0003F8010FE002D02000F030F00002D120033
:10C1B00010000240280002401C5402580854025843
:10C1C000B8040240305402586C5402585854025873
:10C1D0008054025894540258805802580096001611
:10C1E0003F96001640590258A0670024CC8D0C08D9
:10C1F000D068AA4B0340D9F8440043F00303D3604E
:10C20000136923F001031361136923F0704303439F
:10C210001361A34B9A4277D003F580739A4273D08F
:10C22000A04B9B6813F4403F14BF01230023002B55
:10C2300000F0EA80F5F756FDD9F814300146B3F561
:10C24000003F00F01E82B3F5403F00F01E82B3F5C0
:10C25000803F00F01682944BD9F810001A6841F222
:10C260000303B3EB124FC0F0C780904B9942836831
:10C2700000F20F8123F4807383605AE5F4232022B7
:10C2800003FB0BA3C3F8C820032283F8A9203FE4D3
:10C29000826802F00D02012A1DD05A6E002142F080
:10C2A00010025A669A6E42F001029A66F42303FB6A
:10C2B0000BA35A6E42F010025A6689F8601027E408
:10C2C0000023C9F8783013607E600023C9E9383351
:10C2D000C9F8E83006E78268754B764D134043F0A5
:10C2E00002038360032303602A688368DE077FF507
:10C2F00047AD2B689B1A022BF7D98368DF07F4D56B
:10C30000F42303FB0BA3C8E76B4B9B6813F4403F7C
:10C3100014BF012300238AE7614B68499B68896841
:10C320000B43D8073FF5F1AC6349E8E4D9F81010A6
:10C330005B4B029D9942D9F8F07052D003F580739F
:10C3400099424ED0574882688B685E073FF5E0AB54
:10C3500099F86030012B3FF4DBAB02F01F0240F292
:10C3600021230124D34089F86040234040F0FF801E
:10C3700089F86030FFF7CCBB00284FEA906709DBF3
:10C38000C0F31305002D40F0E6800125BD40CE69C5
:10C390002E43CE61A50901F1300604F01F0407F019
:10C3A0001F0705F00C054FF01F0CA7400CFA04FC0A
:10C3B000745924EA0C043C4374518D688C6805F070
:10C3C000040504F008042C4300F082808C68E60722
:10C3D00032D501990131C9B20191002189F860106B
:10C3E00095E63548AFE7026BD9F8283022F00F0206
:10C3F000013B13430363A5E4314B994242D8836860
:10C4000023F44073836094E42E4B9A6D02F440321F
:10C41000B2F5803F00F08881B2F5003F00F06981FD
:10C42000002A7FF418AF1B681A017FF514AF07A824
:10C43000F5F796FC07990EE7D1F8C040C0F3130555
:10C44000002824EA0504C1F8C040C2DA144CA14215
:10C4500000F01D8104F58074A14200F01881114C98
:10C46000194EA568B668F60740F11B81F423002138
:10C4700003FB0BA35A6E42F020025A6689F8601043
:10C48000FFF746BB114B994200F22881836823F4E1
:10C49000407343F4807383604BE400BFFCBFFFFF35
:10C4A00000200240006302580010005C002D3101A2
:10C4B000C0FFFF7F802E00240023024000210240A5
:10C4C00021BCBE00004402580060025841787D0142
:10C4D000C0F30454039FC50D01F1140607FA04FCD0
:10C4E000072705F00405A740745924EA070444EA25
:10C4F0000C0474519F4C246804F07044B4F1805FC4
:10C50000CC6800D0CC680C6E850604F0F844B4EB1F
:10C51000806F03D10C6E24F000440C664C6E04F066
:10C52000F844A54203D14C6E24F000444C668C6E56
:10C5300004F0F844A54203D18C6E24F000448C66CC
:10C54000CC6E04F0F844A5427FF440AFCC6E24F0EA
:10C550000044CC663AE790FAA0F50126B5FA85F5D5
:10C5600006FA05F513E7282E7FF6E7ACE3E48B68BF
:10C57000DC0733D48C68804B1C421FD18C687F4B06
:10C58000234043F001038B602C688368DB0602D0F4
:10C590007B4B994222D079480B68DE071ED48B680A
:10C5A000DE0704D48B68034043F001038B602B68E3
:10C5B0001B1B022BF0D90B68DB07EDD4F42303FB24
:10C5C0000BA35A6E42F010025A669A6E42F00102B4
:10C5D0009A66002389F86030FFF79ABAF420694B15
:10C5E00000FB0BA0446E234043F48073436612B1FA
:10C5F000634B994206D0F42303FB0BA35A6E22F43B
:10C6000080125A66F42303FB0BA35A6E12F4805275
:10C6100000F0A8809A6E22F006029A66D9F85C00B3
:10C620000024594BD9F83C20C363584B0364584B42
:10C63000C3641C230B604B6889F8604043F010030F
:10C640004B60CB6823F003031343CB6090F8343086
:10C65000012B0CD0012380F8343090F83530012BB9
:10C6600000F02C814FF4006380F834404365D9F822
:10C670001020424B91680B4043F004039360FFF796
:10C6800047BA1B0CB1FBF3F1E5E58108E3E5414C4A
:10C69000414E3B4FA568B668BF683E43F7073FF57C
:10C6A000E5AE3E4F05F0E076B84200F08D803C4F9D
:10C6B000B84200F0A7803B4FB8427FF48AAE6F02C9
:10C6C0003FF587AE384881427FF483AEA16821F000
:10C6D000E071314341F48001A1607AE6334B994225
:10C6E00083682AD823F4407343F400738360FFF710
:10C6F00020BBDA6C186802F04052470701D5002AC7
:10C7000032D02B4B1B68DE0503D5B2F1805F00F001
:10C71000D380274B1B689D037FF59DAD254BB2F160
:10C72000005F08BF194696E51B689B007FF593AD37
:10C7300007A8F5F7AFFB09998DE543F440738360D3
:10C74000FFF7F7BA1C48103B10441822A828B3FB87
:10C75000F2F300D80833194A0126194F1A449E40B3
:10C7600092009CE49A6659E71B681649C3F3C1031B
:10C77000D94070E50010005C3F000080C0FFFF7FE3
:10C7800000210240FEF0FFFF0100040855000408EC
:10C79000590004080023024000200240000084CB1E
:10C7A000000052C70000B8CF0060025881F0FA02C2
:10C7B0000044025800127A00F0FBFDBF0082001016
:10C7C000800802400090D0032D023FF502AE85485C
:10C7D00081427FF4FEAD844984480968B1FBF0F1E1
:10C7E000A068013120F0E0704900304340F40000BF
:10C7F000A060069102E00699013906910699002988
:10C80000F9D1E6E5E8013FF5E4AD764881427FF4F1
:10C81000E0ADA16821F0E071314341F08071A16089
:10C82000D7E5734B7348824218BF9A4200F1140057
:10C830000CBF01230023824208BF43F001031430E0
:10C84000824208BF43F001031430824208BF43F024
:10C8500001031430824208BF43F0010314308242C6
:10C8600008BF43F001031BB9634B9A4240F0958126
:10C87000F4210220614B01FB0BA1134481F8A900B4
:10C880001421B3FBF1F38340106842F2A0516FF31F
:10C8900010100143002089F8A80020461160C9F853
:10C8A000D030F5F7B7F8D9F8D02002F01F010122F7
:10C8B0008A404260FFF750BB5149CCE403684031E5
:10C8C000504A514D866DAB4218BF934205F1300579
:10C8D00001960CBF01220022AB4208BF42F00102C8
:10C8E0001835AB4208BF42F001021835AB4208BF11
:10C8F00042F001021835AB4208BF42F0010205F5D3
:10C900005675AB4208BF42F001021835AB4208BF72
:10C9100042F001021835AB4208BF42F0010218355F
:10C92000AB4208BF42F001021835AB4208BF42F0EB
:10C9300001021835AB4208BF42F001021835AB4284
:10C9400008BF42F00102142505FB07F7022580F815
:10C95000355044652D4C2E4DA34208BF42F00102D4
:10C96000A4F59564AB4218BFA3420CBF0124002478
:10C9700001D0002A4ED01D6825F001051D60002C55
:10C9800079D0D0F86CC0D0E919566E60BCF1000FB8
:10C9900004D0D0E91C566E60002C74D0C56D019E89
:10C9A00005F01F0E3F2505FA0EF5B5601D6825F44C
:10C9B00080251D6085685F60402D00F0F5809960DE
:10C9C000C3F80C8014B9002A00F09980196821F08E
:10C9D0001E0141F016011960196841F00801196043
:10C9E000BFE000BF0060025800000024400D0300BB
:10C9F000085402581C54025894540258F8ABFDA72E
:10CA000000093D005800024040000240B8040240C6
:10CA100028000240684DDFF8A8C1634518BFAB424B
:10CA20000CF1280C0CBF01250025634508BF45F01B
:10CA300001050CF1140C634508BF45F001050CF12C
:10CA4000140C634508BF45F001050CF1140C634557
:10CA500008BF45F00105D3F800C02CF0010CC3F865
:10CA600000C0DFF864C1634508BF45F0010515B992
:10CA7000524DAB4243D1D0F86CC0D0E919566E602C
:10CA8000BCF1000F85D1002A88D14D4DDFF828C1B7
:10CA9000634518BFAB420CF1140C0CBF01250025F7
:10CAA000634508BF45F001050CF1140C634508BF50
:10CAB00045F001050CF1140C634508BF45F0010574
:10CAC0000CF1140C634508BF45F001050CF1140C82
:10CAD000634508BF45F0010515B9384DAB420ED18D
:10CAE000C56D019E05F01F0C012505FA0CF575605A
:10CAF00085685F60402D5BD09960C3F80C802E493B
:10CB00002F4DAB4218BF8B4205F128050CBF012108
:10CB10000021AB4208BF41F001011D6825F00E0560
:10CB200045F00A051D60274DAB4208BF41F00101E9
:10CB30001435AB4208BF41F001011435AB4208BFC8
:10CB400041F001011D6845F004051D601E4DAB421A
:10CB500008BF41F0010111B918498B4212D1D0F838
:10CB60006CC0016E0868C20303D5086840F4807089
:10CB70000860BCF1000F05D0DCF8001041F48071B2
:10CB8000CCF800101A6842F001021A606FE50F4BF2
:10CB90000F4903449B00FFF79CBA4023C1F8C830FB
:10CBA00081F8A970FEF7B4BFC3F80880D96009E71F
:10CBB000C3F80880D960A2E71C5402589454025864
:10CBC0000854025844540258805402583F820010BE
:10CBD0004009024010B54FEA511E024400EB8E0C92
:10CBE000624529D901F01F034FF0FF3450F82E1091
:10CBF00004FA03F30B4093FAA3F3B3FA83F3DBB223
:10CC0000202B16D10CF104018A4202D817E08A4287
:10CC100012D98C460431DCF8003093FAA3F3B3FA4E
:10CC200083F3DBB2202BF2D0ACEB000C03EBCC0097
:10CC300010BD03EB4E1010BD4FF0FF3010BD20466D
:10CC400010BD00BF0369416853EA0102F0B43B4ED6
:10CC50005DD0C56A013390ED067A6A1C876830EEB4
:10CC6000077A0361012AC26280ED067A42D090ED14
:10CC7000075A07EE902AD0ED096A70EE455A3468DB
:10CC8000B8EEE76A611AC5EE867AB94277EE857A20
:10CC900030EE670AC0ED087AC0ED077AF0EE667AEA
:10CCA000E5EE807AC0ED0A7AC0ED097A01D8F0BCD1
:10CCB0007047012A28DD06EE905AF8EEE66A87EE04
:10CCC000A66AB5EEC06AF1EE10FA1DDBF1EEC67A87
:10CCD000F4EE677AF1EE10FA16D6D0ED056AF4EEAE
:10CCE000E76AF1EE10FA15D5037BFBB10323F0BC24
:10CCF00003707047326880ED080A521A002180EDF7
:10CD0000070ABA424162D2D9DFED0D7AE5E7316810
:10CD100041609EE707EE903A0223F8EE677A0370CF
:10CD2000F0BCC7EE276AC0ED066A70473168002282
:10CD30000361C36241608261B9E700BF70310024C2
:10CD40000000000010B5DFED4F4A844600F1480EA8
:10CD50000346DA6AB1EC017AD3ED067A013277EE56
:10CD6000877A012ADA62C3ED067A71D093ED075A09
:10CD700007EE902A93ED096A77EE455AF8EEE77AC6
:10CD8000C5EEA76A76EE857AF0EE466A37EE677AE8
:10CD9000C3ED087AE5EE876AC3ED0A6AC3ED077A48
:10CDA0001833C3ED036A7345D3D1374C4168226809
:10CDB0000369521A816801338A42036147D990EDB1
:10CDC000056A0022DFED2F5ADCF82C10F0EE657AB0
:10CDD000DCED0A6A012901F1FF3E11DD07EE90EA60
:10CDE000F8EEE77A86EEA77AB5EEC07AF1EE10FAA1
:10CDF00045DBF1EEC77AF4EE677AF1EE10FA3ED633
:10CE0000B4EEE76A01320CF1180CF1EE10FA26D4F8
:10CE1000022AD9DDB4EEE76AF1EE10FA1FD407EE6C
:10CE2000903AD0ED066A90ED0C7A0223F8EE677A1C
:10CE3000D0ED125A037086EEA76AC7EE276A85EE18
:10CE4000A77A80ED066AC0ED0C6A80ED127A10BDFB
:10CE5000F0EE477A83ED087AF0EE646A9EE7037B92
:10CE600013B10323037010BD002221680361C36264
:10CE700041608261026343648264C36510BDDFED7B
:10CE8000017ABDE70000000070310024B0EEC06AF6
:10CE9000F0EEE05AF0EE407AF4EEC65AF1EE10FAF7
:10CEA0000EDCB5EE400AF1EE10FA4AD0F4EEC65AA6
:10CEB000F0EE466AF1EE10FA4FD5B0EE655A03E097
:10CEC000F0EE656AB0EE465A85EE267A9FED242A8A
:10CED0009FED243A9FED244ADFED244ADFED242A1A
:10CEE000DFED243AB7EE005ADFED236AF4EEC65ABE
:10CEF000F1EE10FAA7EE023AE7EE223AA7EE034A65
:10CF0000A7EE235AE7EE044AE7EE246AB1EE667A0A
:10CF100087EE050A10D4F5EEC00AF1EE10FA03D53B
:10CF20009FED167A37EE400AF5EEC07AF1EE10FA70
:10CF300048BFB1EE400A70479FED117A37EE400AC4
:10CF4000E9E7F5EEC00ADFED0F7A9FED0F0AF1EE8B
:10CF500010FA58BFB0EE670A7047B0EE465AB3E712
:10CF600039094E3DE3B59EBE88FA16BE45FE7FBF29
:10CF700099FB243F69A2163EA7DFA8B4DB0F494006
:10CF8000DB0FC93FA7DFA834DA0F4940D1ED007AA3
:10CF9000F7EE002AD0ED043A90ED054AE7EEA73A05
:10CFA000D0ED064A90ED075AD0ED085A90ED096A87
:10CFB000D0ED0A6A90ED0B7AC0ED043A91ED003A9B
:10CFC000D1ED013AD0ED0C7AA3EE234A80ED054A6B
:10CFD000D1ED003A91ED024AE3EE844AC0ED064AF3
:10CFE000D1ED004A35EE245A80ED075AD1ED014AC1
:10CFF00091ED005AE4EE855AC0ED085AD1ED015A80
:10D00000A5EEA56A80ED096AD1ED015A91ED026A9B
:10D01000E5EE866AC0ED0A6AD1ED016A37EE267A3E
:10D0200080ED0B7AD1ED026A91ED007AE6EE877A17
:10D03000C0ED0C7A91ED027AD1ED017A90ED0D3AC6
:10D04000D0ED0E3AA7EE273A90ED0F4AD0ED104AF8
:10D0500090ED115AD0ED127AD0ED135A90ED006A8E
:10D0600080ED0D3A75EEA25A91ED023AD0ED016ACB
:10D07000E3EE033A90ED027AC0ED0E3AD1ED023ABA
:10D0800034EE234A80ED0F4A91ED004A74EE844A53
:10D09000C0ED104AD1ED014A35EE245A80ED115A07
:10D0A00091ED025AC0ED135A77EE857AC0ED127AEF
:10D0B000D1ED017AD1ED005A67EEA77A91ED025ACF
:10D0C000E5EEA57AE5EE057AA5EEA76A80ED006AA1
:10D0D00091ED016AE6EE276AC0ED016AD1ED026AC0
:10D0E000A6EEA77A80ED027A90ED037A77EE277AA2
:10D0F000C0ED037A704700BF2DE9F04F4FF00009F3
:10D10000864600F110050646034689B000F1300856
:10D11000074648462C468B469C46B246CDF80CE066
:10D1200000283CD10CF1040CA445FBD1032800F1EC
:10D13000010151D09C46AA46029398B1DCED047AD5
:10D14000AAEB0903B64601927246F3EC016A0EF1AE
:10D15000100E92ED007A5345E6EEC77ACCED047AD4
:10D16000F2D1019ADCED046A0CF1100C15ED047A91
:10D170000AF1100AC445C6EE877ACCED007ADCD1FC
:10D18000029B0436084608F10408143314351034A1
:10D19000103709F104099C46B2460028C2D0DCEDE4
:10D1A000007AD646394601927246F1EC016A0EF1D8
:10D1B000100E92ED007A9942E6EEC77ACCED007A35
:10D1C000F2D10CF1040C019A0AF1040AA445E6D14B
:10D1D000032800F10101ADD1DDF80CE00023594630
:10D1E00004AD764677460020049305930693079393
:10D1F000F2EC017AE5EC017AB0B104AC3B46B4EC58
:10D20000017AF3EC016AE6EEC77AB34245ED017AA2
:10D21000F5D1013004280BD0F2EC017A1037143626
:10D22000E5EC017A0028E8D1103714360120DFE759
:10D2300008AD10310EF1400E042875ED017AA1F110
:10D240000402744641ED017A1ED07346F3EC016A84
:10D25000B1EC017AA342E6EEC77AC2ED007AF5D1CD
:10D260005EED016A013887EEA67A82ED007A17D06A
:10D27000AEF1140E103C114675ED017A0428A1F1AF
:10D28000040241ED017AE0D15EED016A103CAEF19D
:10D29000140E032087EEA67A01ED017A1146EBE722
:10D2A00009B0BDE8F08F00BF60EEA00AE0EE000A12
:10D2B000F5EEC00AF1EE10FA07DBB1EEE00AB4EECB
:10D2C000400AF1EE10FA00D670479FED010AFBE725
:10D2D0000000000060EEA00AE0EE000AE1EE010AA4
:10D2E000F5EEC00AF1EE10FA07DBB1EEE00AB4EE9B
:10D2F000400AF1EE10FA00D670479FED010AFBE7F5
:10D3000000000000DFED297AB4EEE70AF1EE10FA32
:10D3100028DD9FED277A30EE470AB4EEE70AF1EEFA
:10D3200010FAF8DCDFED237AB4EEE70AF1EE10FA3A
:10D330002FDD30EE670A37EEC00A60EE007ADFEDCF
:10D340001E5A9FED1E6ADFED1E6AA7EEA56A9FEDCD
:10D350001D7A60EE275AE7EE866AA7EEA67AA5EE5A
:10D36000870A7047DFED187AB4EEE70AF1EE10FA9B
:10D37000D8D59FED0F7A30EE070AB4EEE70AF1EE4A
:10D3800010FAF8D4DFED0B7AB4EEE70AF1EE10FAFA
:10D39000CFDC9FED0E7AB4EEC70AF1EE10FACCD5D1
:10D3A00030EE270A37EE400AC7E700BFDB0F4940DF
:10D3B000DB0FC940DB0FC93F9A7C2E36FAAF4FB95D
:10D3C0003587083CA4AA2ABEDB0F49C0DB0FC9BFC2
:10D3D00010B5404CB4FBF2F4A14219D3DFED3E7A14
:10D3E000F7EE005AB0EE677AB0EE676AF0EE676A61
:10D3F0000023C0ED005AC0ED017A80ED027A80ED85
:10D40000036AC0ED046A836143610362C36110BDB6
:10D4100007EE902ADFED315AB7EE006ADFED306A91
:10D42000B8EE677A07EE901AB0EE405AF8EE677AD7
:10D4300027EE257A67EEA67AC6EE076AC7EEA64AF9
:10D44000FDEEE47A17EE902A2032402A3FD8B0EE63
:10D45000640AFFF757FFB0EE404ADFED227A34EE60
:10D46000A70AFDEEC07A17EE902A2032402A29D86A
:10D47000FFF748FFF8EE006A60EE266A012B1CD029
:10D48000B7EE006AF6EE004A36EE406A66EE244ACF
:10D4900035EE055AF7EE007A84EE057A77EE275AD4
:10D4A00037EEC75A84EEA57AC6EE257A86EEA56ACF
:10D4B000C5EE256AF0EE475A9AE7F7EE004AB0EE5D
:10D4C000666AE5E7DFED086A9FED030AD6E79FEDA0
:10D4D000024AC2E720A1070000000000BD378635E0
:10D4E000DB0FC940DB0FC93F00000080DFED077A8A
:10D4F00030EE270AFDEEC07A17EE903A2033402B2B
:10D5000000D8FFE69FED020A704700BFDB0FC93F5E
:10D51000000000002DE9F84F9DF828408946DDF80D
:10D520002CB00546002C17461BF8011B0CBF4FF012
:10D5300020084FF030081C1E08463ADB00295CD05A
:10D54000002C53D04FF0000A5B4600E064B313F8A0
:10D55000016B013C002EF9D1BAF1000F2FD1264604
:10D5600044B14D454146284600D2B847013CF8D168
:10D570000B9B18780146A0B14FF0FF344FF0000A22
:10D5800000E09B464D45284600D2B8475B4613F85D
:10D59000011B0029F5D10B9BF61A5E44BAF1000F6E
:10D5A00010D13046BDE8F88FBAF1000F1BD15646B6
:10D5B000E0E7634229B31C464FF0010AC4E70028A4
:10D5C000E0D10646002C04F1FF3AEADD54464D4511
:10D5D0004146284600D2B847013CF8D201365644AD
:10D5E0003046BDE8F88F30B12646CBE726464FF0EF
:10D5F000FF34B246C6E70646D3E72646002CB0D134
:10D60000CFE76FEA040A0E46E0E700BF0FB430B57B
:10D6100083B00B4C06AB53F8042BD4E95A010193A9
:10D620006AF078FF0546206803685B699847002820
:10D63000F9D0284603B0BDE8304004B0704700BFC1
:10D64000A06600240EB410B583B00446084905ABAB
:10D6500001A853F8042BCDE900346AF05BFF0022E7
:10D66000019B1A7003B0BDE8104003B0704700BFC3
:10D6700031B104080CB4F0B53C4CADF5277DD4F8BD
:10D680007031002B6DD094F8783199420BD9012379
:10D69000D4F87C218340134205D10DF5277DBDE8E8
:10D6A000F04002B07047324B4FF47A71314A1B6838
:10D6B000A2FB030206A8920901FB12332E49FFF7D1
:10D6C000C1FF06ABAC9A064603442C4901A801935E
:10D6D000ADAB00936AF01EFF019B0A2100225D1C86
:10D6E00001951970019BD4F87051591C01911A7061
:10D6F000ADB12B685B6A1BB128469847D4F87051CE
:10D700009DF818100029C8D00DF119042B6828467F
:10D710001B68984714F8011B0029F7D1BDE7D4F81E
:10D720007471002FB9D0304426ABFD2206A9841CA9
:10D730001846ADF810202246CDF81250ADF816501C
:10D7400077F0BEFF02220346044402A93846CDE921
:10D75000023430F009FB0DF5277DBDE8F04002B042
:10D760007047D4F87431002B8DD196E7A066002461
:10D7700070310024D34D6210EC360D0825B1040839
:10D7800038B5184C0330D4F8802102EB9003B3F580
:10D79000007F18D804EB810104F5C27520F0030066
:10D7A000C4F8803105EB8205D1F88429C3F50073F4
:10D7B00010440D4A9B00C1F8840904210020FFF7A2
:10D7C00059FF284638BD0021084A00250846FFF7C2
:10D7D00051FFD4F80C3A284643F00073C4F80C3AD1
:10D7E00038BD00BFA0660024F8360D081C370D08B0
:10D7F0004B1EDBB2062B70B586B03DD8204A02EB3B
:10D800004303B3F848511F4BA3F15804002808BF45
:10D810001C46A44620893CF8082B4FFA82FE90B1A2
:10D82000A5EB0E022B1A002AB8BF5242002BB8BF3C
:10D830005B429A4202DD64464FFA80FE3CF8080FD4
:10D840000028EDD12288104B93F8100AA379059394
:10D85000A38804930D4BA67800910D4903960028E8
:10D8600018BF0B4603210120CDE90152094AFFF7F9
:10D8700001FF204606B070BD4FF48075C3E700BFBE
:10D88000CC8D0C08041B0024A06600242C370D0846
:10D89000704E0D0830370D0803685A1C0260187866
:10D8A000704700BF03681A46591C016012F8021B3A
:10D8B0000260587841EA0020704700BF02681346B2
:10D8C000511C016013F802CB0360D31C5178036034
:10D8D00093781B0443EA0123111D43EA0C03016002
:10D8E000D07843EA0060704712B370B504468646AC
:10D8F00004E0981B17D114EB0C0C15D01EF8013B5B
:10D90000A3F14100A2EB0E0C192811F8010BA0F1B4
:10D91000410598BF203300F12006192DE9D91B1AC3
:10D9200004D10028E7D170BD604670BD184670BDB7
:10D9300010467047038800211A4A30B503F0030EE1
:10D9400090F802C0184CA3F5FA630EEB4E0E0CF1E2
:10D95000FF3C40F2B5550CEB8E0C04EB4C044FEA47
:10D96000930CB4F85831847905FB0C3390F803C05C
:10D9700022444FF47A740CF1FF3C634490F804C0E5
:10D9800003EB43030CEBC30C43790089CCEB0C1C79
:10D9900003EB8C03C3EB031302EB8302C2FB040112
:10D9A00030BD00BF80436D38CC8D0C08F8B51646ED
:10D9B0001F46404D0446394630464FF47A720023E4
:10D9C00072F010FB3C4B05443C4F3D4E83FB051071
:10D9D000E9172844C1EB601183FB0103C8170B440E
:10D9E000C0EB631087FB003CC317C3EBAC0386FBA3
:10D9F00003764FEAE37ECEEBE61EC1EB0116A5EB04
:10DA0000860CC0EB00154FEA8E0684F806C0A1EB29
:10DA10008501617103EB4301A0EBC10040F2B551F8
:10DA200001FB1E332071B3F5896F37DA40F2DA213A
:10DA30008B4239DCB3F5B77F2249B4BF4FF0000EFB
:10DA40004FF0010E0EEB4E0075464FEA4E0701EB0C
:10DA5000C001B1F86E011C4907EB0E0C01EBCC0CB8
:10DA60000B210CF1160C01E03CF8020D984212DD7E
:10DA70000139F9D17744134901EBC701B1F85801D5
:10DA8000012106F5FA6E0133A17075441B1A22813B
:10DA90002580E370F8BD0131C9B2F2E7032540F2F9
:10DAA00096500627AE46D6E7022540F229400427C5
:10DAB000AE46D0E780BC92C789888888ABAAAA2ADC
:10DAC00073B06D16CC8D0C08248F0C0830B5304C1B
:10DAD0008DB086460D46EC461EF0030F0FCCACE829
:10DAE0000F000FCCACE80F0094E80F008CE80F009B
:10DAF0000FD1284B284A03FB0EF3B2EBB30F44D3EC
:10DB0000264AB2EB331F34BF01220022C2F11D02AC
:10DB100000E01C220EF1FF33019240F26D1220480A
:10DB2000002B194602FB0EF21E4CB8BF0EF102018B
:10DB3000EE4602EBA10280FB0310DB17ADF10401FE
:10DB400001EB8501A3EB6015C3EBE0132A441A44F3
:10DB5000253284FB0230D3171044C3EBA003C3EB80
:10DB6000C303D31A5EF8040FC218714584FB023C4C
:10DB70004FEAE2739444C3EBAC03C3EBC303A2EBE1
:10DB80000303EFD1C01A0DB030BD1D22C2E700BFA4
:10DB9000848F0C08295C8FC2285C8F020AD7A300EF
:10DBA0001F85EB51932449920D4B10B553E9024365
:10DBB00054EA03020AD10146002340F2011218463A
:10DBC0000B80C1F802208B710B8110BD054A1268D1
:10DBD000121943F10003FFF7E9FE012010BD00BF59
:10DBE000C07000247031002430B5144D83B0044659
:10DBF000D5F8181AD5F81C3A51EA03020AD10023C5
:10DC000040F2011218462380C4F80220A371238138
:10DC100003B030BD0A4A1268521843F10003FFF7FF
:10DC2000C5FEB5F8203A20460DF106022146ADF8B2
:10DC3000063067F0A3F9012003B030BDA0660024D0
:10DC40007031002488422DE9F04198464FF00104DC
:10DC500039D301FB04F4B0FBF4FC8C45F9D264B376
:10DC60000025BCF1000F04FB1C00B4FBF1F7D4BF8E
:10DC7000002601266DB966B9A142354619D9C646B6
:10DC80000CF1300C0EF801CB00238EF80030BDE80B
:10DC9000F081BCF1090F18DD002A0CBF5723372390
:10DCA000C6466344A14205F101050EF8013BF0466A
:10DCB000EAD83C46B0FBF7FCD3E7C64600238EF813
:10DCC0000030BDE8F0818446CAE73023E8E700BFB2
:10DCD0002DE9F0410446154608469442B4FBF2F69D
:10DCE00007D205FB1644134B1B5D00F8013BBDE852
:10DCF000F0819642B6FBF2F70CD20E4B05FB17678C
:10DD000005FB1644DA5D1B5D00F8012B00F8013BB2
:10DD1000BDE8F081BA42B7FBF2F807D905FB1878E5
:10DD2000044B13F8082000F8012BE7E74046FFF703
:10DD3000CFFFF3E77C370D08B5EEC00ADFED357A8B
:10DD40000023F1EE10FA30B5C8BF30EE270A87B0D5
:10DD5000D8BF30EE670ADFED307A054603A902939B
:10DD600020EE270ACDE90033FDEEC07A17EE904A87
:10DD700084EAE470A0EBE47068F0CAFA002C03A80F
:10DD8000B4BF2D2320238DF8003071F011FB012842
:10DD90002AD0022834D003281ED003A968467AF07E
:10DDA00087FC684671F004FB044669462846033C3C
:10DDB000E4B2224677F084FC002328462B5571F00C
:10DDC000F7FA2E22431C0DEB04012A54E8187AF0CE
:10DDD00067FC284607B030BD302303A968468DF89C
:10DDE00001307AF065FCDCE743F23002302303A90E
:10DDF0006846ADF801208DF803307AF059FCD0E781
:10DE000043F2300303A96846ADF801307AF050FCC4
:10DE1000C7E700BF6F12033A00007A440378202B53
:10DE200003D110F8013F202BFBD0092BF9D02D2B6B
:10DE300063D02B2BB7EE000A08BF01300278A2F1A5
:10DE40003003D9B2092961D8F2EE046ADFED4D7AC8
:10DE500007EE103A10F8012FB8EEC77AA2F130039E
:10DE6000D9B2A7EEA67A0929F0EE477AF0D92E2A80
:10DE700050D0037803F0DF03452B3BD110B4427838
:10DE80002D2A73D02B2A62D0A2F130030130092B46
:10DE900063D80024002303EB830302EB430310F851
:10DEA000012FA2F13001303B0929F4D9B3F59A7F53
:10DEB0001A46B7EE007A28BF4FF49A72072B09D999
:10DEC0001346DFED316A083B27EE267A072BFAD896
:10DED00002F007022AB1F2EE046A013A27EE267A2E
:10DEE000FBD1002C3BD0C7EE877A5DF8044B20EEC7
:10DEF000270A704720EE270A704742780130BFEEAC
:10DF0000000AA2F13003D9B209299DD92E2ADFEDEA
:10DF10001D7AAED143780130A3F13002D1B2092984
:10DF2000A8D8B2EE047AF0EE475A06EE902A10F81E
:10DF3000013FB8EEE66AA3F13002D1B2C6EE076A3D
:10DF4000092927EE257A77EEA67AEED992E782782C
:10DF50000230A2F13003092B9BD9B7EE007A67EEAD
:10DF6000877A5DF8044B20EE270A704782780230EA
:10DF7000A2F13003092B01D801248BE7B7EE007A18
:10DF8000B1E700BF0000000020BCBE4C0378092BA5
:10DF900001D0202B05D110F8013F202BFBD0092BFD
:10DFA000F9D02D2B09D001784FF0010CA1F13002EE
:10DFB000D3B2092B0AD900207047417801304FF0C5
:10DFC000FF3CA1F13002D3B2092BF4D8002310F8A2
:10DFD000011F03EB830302EB4303A1F13002D1B233
:10DFE0000929F4D90CFB03F0704700BFAB4BAC4AD6
:10DFF0002DE9F04F4FF0000A97B09E1A41F221052B
:10E000001F462C2200210DEB020079F0D7FBA44A19
:10E01000A44B0892CDE90976DA68D10707D5A24A60
:10E020005A6002F188325A60DB68DC070DD49D4BE0
:10E03000D3F80C21D20708D59B4AC3F8042102F17A
:10E040008832C3F80421D3F80C31002101227E2349
:10E0500008A8149105A98DF854208DF81430FDF707
:10E060007FFB0028C0F2298108214FF4FC4303E024
:10E070005B0001399BB207D01AB2002AF8DA85EAB0
:10E080004202013993B2F7D1884AADF81630884B75
:10E09000934280F0518198460DF11809CDE902A70D
:10E0A000B8F802204FF0000CB8F80030C2F30B0BA8
:10E0B00010048DF81DC00BF10601ADF81810C3F364
:10E0C0000B014FEA1333ADF81A108DF81C3000F134
:10E0D00091800622494608A8FDF742FB0028C0F2BD
:10E0E000FD80BDF8164049460DF11E0011F8013BB8
:10E0F000082284EA032403E06400013AA4B207D0B2
:10E1000023B2002BF8DA85EA4303013A9CB2F7D137
:10E110008842EBD15A46D8F8041008A8FDF720FB36
:10E120000028C0F2DB80D8F8041001EB0B0081421C
:10E1300015D00139013811F8013F082284EA03247F
:10E1400003E06400013AA4B207D023B2002BF8DA4E
:10E1500085EA4303013A9CB2F7D18142EBD1ADF895
:10E16000164008F11408514B984599D3DDE902A7F0
:10E1700000230222494608A8ADF81830FDF7F0FA4E
:10E180000028C0F29A80BDF816300DF11A0041F255
:10E19000210119F8012B082483EA022303E05B0024
:10E1A000013C9BB207D01AB2002AF8DA81EA420297
:10E1B000013C93B2F7D14845EBD102220DF1160193
:10E1C00008A8ADF81630FDF7CBFA002875DB1398D8
:10E1D000002840F08980149800286EDB9DF85420B8
:10E1E000002A40F0978000280DBF01220022012361
:10E1F000002364E0E246674601960137062249465D
:10E2000008A8FFB28DF81D70FDF7AAFA002851DBAF
:10E21000BDF8164049460DF11E0011F8013B0822D9
:10E2200084EA032403E06400013AA4B207D023B2D5
:10E23000002BF8DA85EA4303013A9CB2F7D1884211
:10E24000EBD1D8F804105A4608A801EB0A0631466B
:10E25000FDF786FA00282DDB06EB0B00864215D071
:10E26000711E013811F8013F082284EA032403E0FB
:10E270006400013AA4B207D023B2002BF8DA85EA91
:10E280004303013A9CB2F7D18142EBD1032FDA4428
:10E29000ADF81640B1D1019E63E700BF000004084D
:10E2A000000002080020005223016745BCF30D085E
:10E2B00008EE0D08DDE9016A039F012300220AF13F
:10E2C000010ABAF1020F02DC002B7FF49AAE12B100
:10E2D000FCF73CFF28B9052006F032F8DDE902A77B
:10E2E000EBE717B0BDE8F08F089B099A034493420F
:10E2F000E3D80BABC0F120022146184479F05EFA56
:10E30000149818B90BA908A8F4F7CCFE00221490B1
:10E31000139261E70A4AD16841F00101D160D168E6
:10E32000C9077FF560AFD2F80C1141F00101C2F8C6
:10E330000C11D2F80C2156E70DF1180918E700BFAF
:10E340000020005270B545880B4604460021C5F3F5
:10E350000B0518462A4679F031FA0A4A2169034624
:10E36000914206D3084A914206D31846BDE8704050
:10E3700008470029F9D170BD2A46BDE8704077F002
:10E380009FB900BFBCF30D08EBF80D08184B03EB69
:10E390008000D0F8540138B300EB400003EB80025A
:10E3A00092F901C1BCF1FF3F1FD092F80901D8B129
:10E3B00003EB0C00002310B590F864E18C2092F878
:10E3C0000811142200FB0CFC0A4C0CEB0100013A72
:10E3D000714434F8100013FA80F3F6D1064AA2FB18
:10E3E0000320C0F30F1010BD70470020704700BF1E
:10E3F000A066002400000030CDCCCCCC036810B562
:10E400001A790446022A03D000232360237110BD29
:10E41000987AFDF79FFA0028F6D040F61A6100229C
:10E42000C18020210272FDF7BDFA00232360237111
:10E4300010BD00BF10B1036882889A61704700BFA9
:10E440000379022B00D0704790F9102008311C4846
:10E4500002EB420210B41B4C83B050F832200094FF
:10E460006944194C11F808CCA24224D017498A42B9
:10E4700023D001F580618A4205D0154B9A420CBF2A
:10E4800003234FF0FF33116803EB430321F0010135
:10E4900000EBC30011600169936851F82C1023F060
:10E4A000E0430B439360136843F00103136003B030
:10E4B0005DF8044B70470023E5E70123E3E700BF65
:10E4C000A80200240001020300300140003800408F
:10E4D0000034014010B50446C06900B110BD0921E7
:10E4E0001420FFF74DF9E06110BD00BF90F9103026
:10E4F000F0B503EB4303294E154683B056F833605D
:10E50000044683689A0719D501230DF106028DF898
:10E51000061030460DF10701F5F7FEFD01230DF160
:10E5200006020DF1070130468DF80650F5F7F4FDAF
:10E53000A3689B0717D5012003B0F0BD43691BB149
:10E540009A88186812048261154B164AD3F8240A77
:10E55000154BC0005768A3FB003080095368DB1BD4
:10E560009842FBD2D0E70E4A4FF4FA700E4BD2F825
:10E57000242A0C4900FB02F24868A3FB02329209EC
:10E580004B681B1A9A42FBD26369002BD3D01A68DE
:10E5900001209B88936103B0F0BD00BFA802002456
:10E5A000A0660024001000E0D34D621010B503797E
:10E5B00084B084468E46012B0DD0022B02D0002061
:10E5C00004B010BD8368DB0758BF01F07F0104B0C1
:10E5D000BDE810408AE781680DF10F0014467246CD
:10E5E00001F001018DF80F40CDE900019CF81110F8
:10E5F0009CF91000F5F784F804B010BDF8B50526B5
:10E6000007220A2107460068FFF7D0FF05F03CFE0D
:10E6100004460D4605F038FE001B61EB0501B0F520
:10E620007A7F71F10001F5D3013EEFD10526242256
:10E6300041213868FFF7BAFF05F026FE04460D4673
:10E6400005F022FE001B61EB0501B0F57A7F71F148
:10E650000001F5D3013EEFD10526C02242213868E2
:10E66000FFF7A4FF05F010FE04460D4605F00CFE72
:10E67000001B61EB0501B0F57A7F71F10001F5D364
:10E68000013EEFD10120F8BD10B5044694220B21C4
:10E690000068FFF78BFF712201212068FFF786FFDA
:10E6A000002204212068FFF781FFC822052120688D
:10E6B000FFF77CFF002206212068FFF777FFC822C2
:10E6C00007212068FFF772FF002208212068FFF76A
:10E6D0006DFFC82209212068FFF768FF012010BDE7
:10E6E00000680379012B09D0022B01D0002070476C
:10E6F0008368F022DB0717D5FF21F7E6826890F9DF
:10E7000010C002F00102417C60464FF0F00C10B5E1
:10E7100084B00DF10F040192FF228DF80FC0009418
:10E72000F4F7EEFF04B010BD7F21DFE60068CA43B6
:10E73000037941EA0211012BCAB208D0022B01D0A1
:10E74000002070478368DB0715D5D221CEE610B5CF
:10E7500084B0846890F910C08DF80F200DF10F027D
:10E7600004F00104417C0092D22260460194F4F747
:10E77000C7FF04B010BD5221B8E600BF006803799E
:10E78000012B09D0022B01D0002070478368B422EE
:10E79000DB0717D5FF21A9E6826890F910C002F0C7
:10E7A0000102417C60464FF0B40C10B584B00DF10D
:10E7B0000F040192FF228DF80FC00094F4F7A0FF20
:10E7C00004B010BD7F2191E600680379012B09D0C8
:10E7D000022B01D00020704783680A46DB0715D55D
:10E7E000A52183E610B584B0846890F910C00DF1BE
:10E7F0000F0204F001048DF80F10417C6046009276
:10E80000A5220194F4F77CFF04B010BD25216DE62C
:10E8100000680379012B09D0022B01D0002070473A
:10E8200083689622DB0717D5FF215FE6826890F99F
:10E8300010C002F00102417C60464FF0960C10B50A
:10E8400084B00DF10F040192FF228DF80FC00094E7
:10E85000F4F756FF04B010BD7F2147E60068037946
:10E86000012B09D0022B01D00020704783680A4693
:10E87000DB0715D5872139E610B584B0846890F997
:10E8800010C00DF10F0204F001048DF80F10417C4F
:10E890006046009287220194F4F732FF04B010BD65
:10E8A000072123E60068C9010379CAB2012B05D00C
:10E8B000022B01D000207047782117E610B584B0F4
:10E8C000846890F910C08DF80F200DF10F0204F04C
:10E8D0000104417C0092782260460194F4F710FF15
:10E8E00004B010BD00680379012B09D0022B01D0C0
:10E8F0000020704783685522DB0717D5A521F5E571
:10E90000826890F910C002F00102417C60464FF02D
:10E91000550C10B584B00DF10F040192A5228DF8AD
:10E920000FC00094F4F7ECFE04B010BD2521DDE526
:10E93000006810B5037984B0012B0FD0022B02D0F0
:10E94000012004B010BD83683122DB074CBFF421E5
:10E950007421FFF7CBFD012004B010BD82680DF1DA
:10E960000F0490F910C002F00102417C60464FF0A4
:10E97000310C0192F42200948DF80FC0F4F7C0FE20
:10E98000012004B010BD00BF00680379012B06D040
:10E99000022B01D00020704701225821A6E5826891
:10E9A000417C02F0010210B590F9104084B020467D
:10E9B0000DF10F040192582200948DF80F30F4F7F6
:10E9C0009FFE04B010BD00BF00680379012B06D084
:10E9D000022B01D0002070470122482186E5826881
:10E9E000417C02F0010210B590F9104084B020463D
:10E9F0000DF10F040192482200948DF80F30F4F7C6
:10EA00007FFE04B010BD00BF00680379012B06D063
:10EA1000022B01D0002070471A46082166E5826863
:10EA200090F910C002F00102417C60464FF0020CE8
:10EA300010B584B00DF10F04019208228DF80FC0BB
:10EA40000094F4F75DFE04B010BD00BF00680379C8
:10EA5000012B06D0022B01D0002070470122082193
:10EA600044E58268417C02F0010210B590F9104043
:10EA700084B020460DF10F040192082200948DF815
:10EA80000F30F4F73DFE04B010BD00BF144B30B59D
:10EA9000D3F8284A85B07CB12379012B0FD0022B03
:10EAA0000AD1A1680246204611F0010118BF802159
:10EAB00005B0BDE8304019E5002005B030BDA268C2
:10EAC0000DF10F05617C8DF80F0094F9100002F034
:10EAD0000104802200950194F4F712FE05B030BDC8
:10EAE000A06600242DE9F04105461F462948164638
:10EAF00095F9103082B003EB430350F83380AB68D4
:10EB00009A0716D501230DF106028DF8061040462E
:10EB10000DF10701F5F700FB3B4632460021404668
:10EB2000F5F7FAFAAB689B0719D5012002B0BDE8EA
:10EB3000F0816B691BB19A88186812048261164BC8
:10EB4000D3F8240A154BC000A3FB0030144B8009F6
:10EB50005A685C68A4EB020C6045FAD2D2E70E4A10
:10EB60004FF4FA700D4BD2F8242A0D4900FB02F243
:10EB70004868A3FB023292094B681B1A9A42FBD2E7
:10EB80006B69002BD1D01A6801209B88936102B079
:10EB9000BDE8F081A8020024A0660024D34D6210D5
:10EBA000001000E030B5057983B084468E46012D13
:10EBB0000DD0022D02D0002003B030BD8468E407E0
:10EBC00058BF41F0800103B0BDE830408AE780685B
:10EBD00014460A46009400F001049CF811109CF9B8
:10EBE00010000194F4F78CFD03B030BD2DE9F04125
:10EBF00005461F462948164695F9103082B003EBAA
:10EC0000430350F83380AB689A0716D501230DF102
:10EC100006028DF8061040460DF10701F5F77CFA63
:10EC20003B46002231464046F5F776FAAB689B0733
:10EC300019D5012002B0BDE8F0816B691BB19A883B
:10EC4000186812048261164BD3F8240A154BC000D1
:10EC5000A3FB0030144B80095A685C68A4EB020CDB
:10EC60006045FAD2D2E70E4A4FF4FA700D4BD2F853
:10EC7000242A0D4900FB02F24868A3FB02329209E4
:10EC80004B681B1A9A42FBD26B69002BD1D01A68D1
:10EC900001209B88936102B0BDE8F081A8020024A6
:10ECA000A0660024D34D6210001000E030B5057955
:10ECB00083B084468E46012D0DD0022D02D0002057
:10ECC00003B030BD8468E40758BF41F0800103B051
:10ECD000BDE830408AE7806814460A46009400F098
:10ECE00001049CF811109CF910000194F4F724FF22
:10ECF00003B030BD10B50446006884B00379012B21
:10ED00002DD0022B01D0002027E0836802AA13F047
:10ED1000010F4FF0060314BF1F219F21FFF766FF6D
:10ED20000028F0D0BDF80810BDF80A20C9BABDF817
:10ED30000C30D2BA07EE901ADBBAF8EEE76A07EEAB
:10ED4000902AB8EEE77A07EE903AC4ED046AF8EE3E
:10ED5000E77A84ED057AC4ED067A04B010BD8368C5
:10ED600002AA417C03F0010390F9100000921F22D7
:10ED700001930623F4F7E0FED2E700BF10B5044686
:10ED8000006884B00379012B2DD0022B01D0002024
:10ED900027E0836802AA13F0010F4FF0060314BFA7
:10EDA0002521A521FFF722FF0028F0D0BDF808108B
:10EDB000BDF80A20C9BABDF80C30D2BA07EE901AD5
:10EDC000DBBAF8EEE76A07EE902AB8EEE77A07EECC
:10EDD000903AC4ED076AF8EEE77A84ED087AC4ED5C
:10EDE000097A04B010BD836802AA417C03F00103D4
:10EDF00090F910000092252201930623F4F79CFE5F
:10EE0000D2E700BF006810B5037984B00C46012B2F
:10EE100024D0022B01D000201EE0826812F0010FE6
:10EE200003AA14BF1D219D21FFF7E0FE0028F2D0A8
:10EE3000BDF80C309FED106ADBBADFED106A07EE0B
:10EE4000903AB8EEE77AC7EE067A77EEA67AFDEE4C
:10EE5000E77A17EE903A238004B010BD836803AAC6
:10EE6000417C03F0010390F9100000921D220193F0
:10EE70000223F4F761FED9E7CFF7534100007A434C
:10EE8000006810B5037984B0012B31D0022B09D072
:10EE90001E490020D1F82C3AD1F8302A8B628A60C2
:10EEA00004B010BD062302AAF721FFF79FFE002839
:10EEB000EED09DF809309DF80C209DF808C01B018C
:10EEC0009DF80BE012019DF80A1043EA0C3342EA68
:10EED0000E329DF80DC043EA11130C4942EA1C1290
:10EEE000C1F82C3AC1F8302A8A608B6204B010BD98
:10EEF000826802AC417C062302F0010290F9100006
:10EF0000CDE90042F722F4F717FED0E7A06600240F
:10EF1000006810B5037984B0012B1CD0022B0ED0F1
:10EF20009DF80D3001209DF80CC01B029DF80E10BD
:10EF3000104A43EA0C430B43136504B010BD8368C9
:10EF400003AA13F0010F4FF0030314BF0021802127
:10EF5000FFF74CFEE4E7826803AC417C032302F038
:10EF6000010290F91000CDE900420022F4F7E4FD1F
:10EF7000D6E700BFA0660024006810B5037984B00E
:10EF8000012B1CD0022B0ED09DF80D3001209DF8D6
:10EF90000CC01B029DF80E10104A43EA0C430B43B1
:10EFA000536604B010BD836803AA13F0010F4FF03D
:10EFB000030314BF00218021FFF718FEE4E78268F5
:10EFC00003AC417C032302F0010290F91000CDE96B
:10EFD00000420022F4F7B0FDD6E700BFA06600248F
:10EFE000006810B5037984B0012B28D0022B01D022
:10EFF000002022E0836803AA13F0010F4FF00303FF
:10F000000CBF83211946FFF7F1FD0028F0D09DF8D1
:10F010000C309DF90C109DF80D201B0400299DF863
:10F020000EC043EA02230D4AACBF00214FF07F41DE
:10F0300043EA0C030B43C2F8DC3004B010BD826815
:10F0400003AC0323417C02F0010290F91000CDE9EA
:10F0500000421A46F4F770FDD7E700BFA06600240F
:10F06000006810B5037984B0012B28D0022B01D0A1
:10F07000002022E0836803AA13F0010F4FF003037E
:10F0800014BF00218021FFF7B1FD0028F0D09DF8CA
:10F090000C309DF90C109DF80D201B0400299DF8E3
:10F0A0000EC043EA02230D4AACBF00214FF07F415E
:10F0B00043EA0C030B43C2F8D83004B010BD826899
:10F0C00003AC417C032302F0010290F91000CDE96A
:10F0D00000420022F4F730FDD7E700BFA06600240D
:10F0E00010B500230446006884B0C4F83630638746
:10F0F0000379012B22D0022B01D000201CE0836871
:10F1000002AA13F0010F4FF0060314BF032183215D
:10F11000FFF76CFD0028F0D0BDF90A30BDF80810EB
:10F12000BDF80C205B4201EB410102EB420203EB14
:10F130004303E1866287238704B010BD836802AA77
:10F14000417C03F0010390F9100000920322019327
:10F150000623F4F7F1FCDDE790F91030F0B503EB8E
:10F160004303274E154683B056F833600446836840
:10F170009A0715D501230DF106028DF806103046C9
:10F180000DF10701F4F7C8FF01230022294630469C
:10F19000F4F7C2FFA3689B0717D5012003B0F0BDA9
:10F1A00043691BB19A88186812048261154B164A8C
:10F1B000D3F8240A154BC0005768A3FB0030800920
:10F1C0005368DB1B9842FBD2D4E70E4A4FF4FA7027
:10F1D0000E4BD2F8242A0C4900FB02F24868A3FB2C
:10F1E000023292094B681B1A9A42FBD26369002BC8
:10F1F000D3D01A6801209B88936103B0F0BD00BF93
:10F20000A8020024A0660024001000E0D34D621084
:10F2100010B5037982B08E46012B0DD0022B02D09F
:10F22000002002B010BD8368DB0758BF41F08001A9
:10F2300002B0BDE810408FE7816814467246009422
:10F2400001F00104417C90F910000194F4F774FC82
:10F2500002B010BD2DE9F0478046C549C54A88B0C7
:10F26000D8F8383001F1180E0846D8F800708946F1
:10F270000025B2FBF3FC98F835305A1B867906302E
:10F280009C1B002AB8BF5242002CB8BF6442944273
:10F2900001DA814675B28645EFD11FFA8CFCB9F8C8
:10F2A000020001F11E0E02E006318E4517D00A78E9
:10F2B0000646AA42F8D1ACEB0002B1F802A0002A3F
:10F2C000ACEB0A04B8BF5242002CB8BF6442A24261
:10F2D000EADD89460631504656468E45E7D1CDF8DF
:10F2E00000C0012002960F2699F80510A24A049149
:10F2F00099F80410039199F8001001910321FEF789
:10F30000B9F9B9F802209B4B00213846B3FBF2F360
:10F31000C8F84030FFF794F8002276213846FFF70E
:10F3200045F90F224E213846FFF740F904F0ACFFB3
:10F3300004460D4604F0A8FF001B61EB0501B0F583
:10F340007A7F71F10001F5D3013EEFD199F80520E4
:10F350000F264F21384602F00F02FFF727F904F07D
:10F3600093FF04460D4604F08FFF001B61EB05017F
:10F37000B0F57A7F71F10001F5D3013EEFD199F834
:10F3800005200F265021384602F00F02FFF70EF934
:10F3900004F07AFF04460D4604F076FF001B61EB93
:10F3A0000501B0F57A7F71F10001F5D3013EEFD18F
:10F3B0000F26FF2252213846FFF7F8F804F064FFC9
:10F3C00004460D4604F060FF001B61EB0501B0F53B
:10F3D0007A7F71F10001F5D3013EEFD198F8351035
:10F3E000072941D0654D95F8100AFEF701FA044649
:10F3F000012276213846FFF7D9F8A2780C21384649
:10F40000FFF7D4F822790D213846FFF7CFF8A2791B
:10F41000A3880E211201384642EA1322D2B2FFF726
:10F42000C5F84FF4807195F8100AFEF7E1F904462B
:10F43000022276213846FFF7B9F8A2780321384630
:10F44000520002F0FE02FFF7B1F80421227938469B
:10F45000FFF7ACF8A279A38805211201384642EAE9
:10F460001322D2B2FFF7A2F80022762138460F26E7
:10F47000FFF79CF8032214213846FFF797F804F0B1
:10F4800003FF04460D4604F0FFFE001B61EB05017F
:10F49000B0F57A7F71F10001F5D3013EEFD132462C
:10F4A000642663213846FFF781F804F0EDFE044638
:10F4B0000D4604F0E9FE001B61EB0501B0F57A7F13
:10F4C00071F10001F5D3013EEFD1082265213846E4
:10F4D0000F26FFF76BF864210DF11F023846FFF786
:10F4E00097FE9DF81F206421384622F0100242F05A
:10F4F00060028DF81F20FFF759F804F0C5FE04469E
:10F500000D4604F0C1FE001B61EB0501B0F57A7FEA
:10F5100071F10001F5D3013EEFD10DF11E024D2135
:10F5200038460F26FFF774FE9DF81E204D21384601
:10F5300002F03F0242F040028DF81E20FFF736F83D
:10F5400004F0A2FE04460D4604F09EFE001B61EB93
:10F550000501B0F57A7F71F10001F5D3013EEFD1DD
:10F5600003213846FEF76CFF08B0BDE8F08700BF06
:10F57000B48F0C0840420F00A4370D08A066002489
:10F5800070B5056884B004460E462B79012B15D062
:10F59000022B02D0002004B070BDAB68E122DB0773
:10F5A0001CD528461146FEF7A1FF0028F2D03246AE
:10F5B000FF21206804B0BDE8704029E6AA68697C94
:10F5C00002F0010295F910000DF10F050192E12200
:10F5D00000958DF80F20F4F793F8E6E761212846AF
:10F5E000FEF784FFE1E700BF70B5056884B004460C
:10F5F0000E462B79012B16D0022B02D0002004B02E
:10F6000070BDAB68C3222846DB074CBFE1216121F6
:10F61000FEF76CFF0028F1D03246FF21206804B0CD
:10F62000BDE87040F4E5AA6895F9100002F0010207
:10F63000697C01920DF10F020092C3228DF80F2018
:10F64000E122F4F75DF8E5E770B5056884B004469B
:10F650000E462B79012B1BD0022B02D0002004B0C8
:10F6600070BDAB68F0222846DB074CBFE121612169
:10F67000FEF73CFF0028F1D02246FF2152F8040B90
:10F68000FFF7C6FD0028E9D02379337004B070BDC0
:10F69000AA6895F9100002F00102697C01920DF14F
:10F6A0000F020092F0228DF80F20E122F4F728F8E3
:10F6B000E0E700BFF0B583B015461C4606460DF1E5
:10F6C00007020F46FFF7A4FD9DF8072005EA020395
:10F6D000A34201D103B0F0BD22EA0502394630460B
:10F6E000224303B0BDE8F040FEF760BF10B582B022
:10F6F0000821044600686A46FFF78AFD9DF800303D
:10F70000DB0602D4002002B010BD06236A460021A9
:10F710002068FFF7CBFA0028F4D09DF801209DF86F
:10F72000001012029DF80230DFED496A02EB01423F
:10F730009DF8041014024FEA01219DF80340134480
:10F740009DF8052001EB044148BF03F17F430A44C3
:10F75000090207EE903A3F4B48BF02F17F42F8EEB4
:10F76000E77A93ED0D6A07EE102AB3F93820F8EE28
:10F77000C65AB3F93E10B8EEC77A93F8344A04EE8D
:10F78000901AB3F94210112CC7EE263A87EEA67AEA
:10F7900006EE902AB3F93A20D3ED0C7A06EE102A41
:10F7A000B3F93C2005EE102AB3F94020F8EEE66AE2
:10F7B00004EE102AF8EEE77AB8EEC66AB3F94420F0
:10F7C000B8EEC55AF8EEE44AB8EEC44A66EEA36A4B
:10F7D00027EE232A23D0A7EE045AA7EE246AE5EEEB
:10F7E000075AE5EE877A77EEA67AE6EE027AB3F963
:10F7F0002E20F6EE006AC3ED127A07EE902AB3F9D6
:10F800002C10F8EEE77A07EE101AB8EEC77A67EE1A
:10F81000A37AE7EE267AC3ED137A02B010BD03EEA9
:10F82000102AF8EEC32A03EE101AB8EEC33AA7EE78
:10F83000224AE7EE034AA4EE075AA4EE876AE5EEF1
:10F84000075AE5EE877A77EEA67AE6EE027ACEE7F9
:10F8500000007848A0660024F0B5044683B00D4649
:10F860001746061D20680379012B19D0022B02D000
:10F87000002003B0F0BD83683246FF21DB075CBF88
:10F880003246FF21FFF768FC0028F1D015B123793B
:10F89000DB07E7D4002FECD023793B7003B0F0BD39
:10F8A0008268417C02F0010C90F91000FF22CDE942
:10F8B000006CF4F741F9E7E770B50446051D82B026
:10F8C00020680379012B16D0022B02D0002002B051
:10F8D00070BD83682A46FF21DE075CBF2A46FF21F0
:10F8E000FFF73AFC0028F1D02379DB07EFD5206839
:10F8F0000379012BE8D18668FF22417C06F00106DE
:10F9000090F91000CDE90056F4F716F9EAE700BFC8
:10F91000024630B5044652F8040B83B00379012B3C
:10F920000ED0022B01D0002008E0FF21FFF714FCCD
:10F930000028F8D02079C04300F0010003B030BDAA
:10F940008568417C05F0010590F910000092FF22C6
:10F950000195F4F7F1F8EBE770B5B42282B00446F4
:10F96000FF210068FEF722FE10B9002002B070BD32
:10F970002068251D0379012B13D0022BF5D1836854
:10F980002A46FF21DE075CBF2A46FF21FFF7E4FB82
:10F990000028EAD02379DB07E8D520680379012B1A
:10F9A000EBD18668FF22417C06F0010690F9100039
:10F9B000CDE90056F4F7C0F8EAE700BF70B50A4693
:10F9C00082B00446A5210068FEF7F0FD10B90020C2
:10F9D00002B070BD2068251D0379012B13D0022BC6
:10F9E000F5D183682A46FF21DE075CBF2A46FF2146
:10F9F000FFF7B2FB0028EAD02379DB07E8D52068BF
:10FA00000379012BEBD18668FF22417C06F00106C9
:10FA100090F91000CDE90056F4F78EF8EAE700BF40
:10FA200070B582B00446CDE90023FFF795FF10B909
:10FA3000002002B070BD5522A5212068FEF7B6FD5A
:10FA40000028F5D0251D2A46FF212068FFF7E0FB9E
:10FA50000028EDD02379DB07F5D40DF1FF350DF14A
:10FA6000070615F8011F2046FFF7A8FF0028DFD082
:10FA7000B542F6D1DDE700BF002A34D0F0B5044628
:10FA800083B00E46051D8F1816F8012BA52120689E
:10FA9000FEF78CFD90B9002003B0F0BD8268417C78
:10FAA00002F0010C90F91000FF22CDE9005CF4F7A0
:10FAB00043F80028EFD02379DB070FD520680379BE
:10FAC000012BEBD0022BE6D183682A46FF21DB070E
:10FAD0005CBF2A46FF21FFF73FFBEAE7B742D3D1DD
:10FAE000012003B0F0BD0120704700BFF0B59622A1
:10FAF00083B00E460446FF210068FEF757FD10B99B
:10FB0000002003B0F0BD251D20680379012B1ED015
:10FB1000022BF5D183682A46FF21DF075CBF2A4606
:10FB2000FF21FFF719FB0028EAD02379DB07EBD48C
:10FB3000E12220681146FEF739FD0028E0D0324668
:10FB4000FF21206803B0BDE8F040FFF761BB876884
:10FB5000FF22417C07F0010790F91000CDE9005722
:10FB6000F3F7EAFFDFE700BF002A42D0F0B5044612
:10FB700083B00E46051D8F189622FF212068FEF7E0
:10FB800015FD90B9002003B0F0BD8268417C02F001
:10FB9000010C90F91000FF22CDE9005CF3F7CCFFD7
:10FBA0000028EFD02379DB070FD520680379012BDC
:10FBB000EBD0022BE6D183682A46FF21DB075CBF2E
:10FBC0002A46FF21FFF7C8FAEAE7E122206811463A
:10FBD000FEF7ECFC0028D5D03246FF212068FFF765
:10FBE00017FB0028CED00136B742C5D1012003B0A3
:10FBF000F0BD0120704700BFF0B50B460546164624
:10FC0000044683B087211A4655F8040BFEF7CEFC54
:10FC100020680379012B19D0022B02D0002003B0F9
:10FC2000F0BD83682A46FF21DF075CBF2A46FF211B
:10FC3000FFF792FA0028F1D02379DA07E8D4002EF2
:10FC4000EDD0C3F34013337003B0F0BD8768FF22DB
:10FC5000417C07F0010790F91000CDE90057F3F758
:10FC60006BFFE7E7F0B5782183B016460446002223
:10FC70000068FEF79BFC10B9002003B0F0BD251D05
:10FC800020680379012B13D0022BF5D183682A4613
:10FC9000FF21DF075CBF2A46FF21FFF75DFA00283E
:10FCA000EAD02379DA07EBD45B09337003B0F0BDF7
:10FCB0008768FF22417C07F0010790F91000CDE929
:10FCC0000057F3F739FFEAE770B5CC2282B004465B
:10FCD000A5210068FEF76AFC10B9002002B070BDD3
:10FCE0002068251D0379012B13D0022BF5D18368E1
:10FCF0002A46FF21DE075CBF2A46FF21FFF72CFAC8
:10FD00000028EAD02379DB07E8D520680379012BA6
:10FD1000EBD18668FF22417C06F0010690F91000C5
:10FD2000CDE90056F3F708FFEAE700BF70B5B4224B
:10FD300082B00446FF210068FEF738FC10B90020AD
:10FD400002B070BD251D20680379012B21D0022B44
:10FD5000F5D183682A46FF21DE075CBF2A46FF21D2
:10FD6000FFF7FAF90028EAD02379DA07EBD4CC219F
:10FD70002046FFF723FE0028E1D002E02379DB07CD
:10FD8000DED52A46FF212068FFF742FA0028F5D188
:10FD9000D5E78668FF22417C06F0010690F9100045
:10FDA000CDE90056F3F7C8FEDCE700BF2DE9F04FC0
:10FDB00082468DB0002090460AF104070891069013
:10FDC0000A930790069B5046DC0008EBC30305939B
:10FDD000FFF7C2FD28B941E09AF8043013F00102A0
:10FDE00008D03A46FF21DAF80000FFF711FA0028A0
:10FDF000F2D133E003929A070B9040F1CC80F021CE
:10FE00005046FFF7DBFD48B3083CDDF80C9008EBEB
:10FE10000403012409932546089B003B18BF0123D6
:10FE20000493049B082D8CBF002303F001039B4621
:10FE3000002B5DD06E1E089B43FA06F606F0010605
:10FE4000F2017821DAF80000FEF7B0FB30B1DAF801
:10FE500000000379012B3FD0022B07D000220A9B20
:10FE60001046069919700DB0BDE8F08F83683A46C8
:10FE7000FF21DB075CBF3A46FF21FFF76DF9002841
:10FE8000ECD09AF8043013F00102E0D199094FEA5E
:10FE9000531E4FEAD31C01EA5313DB074BD46645CC
:10FEA00002D0BBF1000F73D1BCF1000F2DD005992A
:10FEB00011F80930234301F809306400013514F0CA
:10FEC000FF04EDB2ADD109F101095FFA89F9B9F189
:10FED000080F30D00124A4E78268417C02F0010CB5
:10FEE00090F91000FF22CDE9007CF3F725FEC6E76C
:10FEF000069BD3B1079BAB4217D9099B13F8093076
:10FF00001C4214BF012600269AE74EEA0101039B1A
:10FF100011F0010F059908BF2B46039311F8093022
:10FF200023EA040301F80930C7E7079B5E1BB6FA12
:10FF300086F6760984E7402D07D80A9B069A1B7837
:10FF400093423FF63FAF024689E7059BDD795C1E91
:10FF50009E1D14F801CF082182EA0C0301394FEAF3
:10FF60005C0C43F3000311F0FF0123F0730383EAF9
:10FF70005202D2B2F0D1A642EBD19542DDD1069B1E
:10FF80000133DBB20693039B002BDCD00793D4E74D
:10FF90000B9E324663E70646324660E710B5002303
:10FFA0000446006886B0C4F8363063870379012BB5
:10FFB00012D0022B0DD183680DF10B02DB074CBF71
:10FFC0003421B421FFF7C8F818B19DF90B30002B8C
:10FFD00011DB002006B010BD8268417C02F00102F6
:10FFE00090F910C001920DF10B026046009234228C
:10FFF000F3F7A2FDE8E7092303AA24212068FEF70E
:020000040805ED
:1000000055FE0028E5D09DF810209DF80F109DF8B2
:10001000133012041B0442EA01629DF8121043EAF5
:1000200001639DF80C10C2F30F42C3F30F43228704
:1000300063879DF80D301B0443EA0163C3F30F434C
:10004000E38606B010BD00BF0368DA6B10B5044646
:1000500082B012B1904740B123685B6B1BB121465F
:1000600001A8984718B9FF23E38202B010BDBDF87C
:100070000630013B9BB2F7E738B58B680446016058
:100080000D46984700230B4A237522612B6B13B151
:10009000204698472075084B93F8383A1BB1237DCA
:1000A00023F00103237500232046E382BDE8384096
:1000B000CAE700BF0001FF00A0660024F0B50D46AE
:1000C00083B00446184616461F466FF071F928445F
:1000D000E6732946A0732046256800243B46324635
:1000E00000946C69A04703B0F0BD00BF294BF0B588
:1000F000D3F8285A85B09DB1B02280212846FEF75A
:1001000055FA402280212846FEF750FA002280212D
:100110002846FEF74BFA102280212846FEF746FAC1
:100120004FF480642DB9013CA4B2002CFBD105B082
:10013000F0BD00270DF10F062B79012B08D0022B03
:1001400004F1FF3217D094B2002CF0D0012BF6D17D
:10015000AA68013C95F9100002F0010CA4B2697C78
:1001600040228DF80F70CDE9006CF3F7C9FA002C2E
:10017000E2D105B0F0BDAA68013C4021284612F04A
:100180000102A4B218BF0022FEF7B0F9002CD3D1AF
:1001900005B0F0BDA06600240C4B10B5D3F8284A7A
:1001A00094B1A0F1500280212046D2B2FEF7FEF9B0
:1001B000002280212046FEF7F9F9204610228021F6
:1001C000BDE81040FEF7F2B910BD00BFA0660024E4
:1001D000F0B5254B2038254C85B000EB8000D3F8D6
:1001E000285A661D0444064425B90134A642FCD1B0
:1001F00005B0F0BD0DF10F072B79012B22781AD035
:10020000022B0AD00134A642F7D100224021284611
:1002100005B0BDE8F040FEF7C9B9AB6840212846FB
:10022000DB0719D50134FEF761F9A642E4D1002DB0
:10023000EBD105B0F0BD8DF80F200134AA6895F917
:10024000100002F00102697CCDE900724022F3F750
:1002500057FAB442D0D1D8E70134FEF747F9B44297
:10026000CAD1002DE5D0D0E7A0660024D48F0C08B9
:10027000754BF0B5D3F8285A85B0002D00F0968064
:10028000D42280212846FEF791F980222846114683
:10029000FEF78CF9A82280212846FEF787F93F2235
:1002A00080212846FEF782F9D32280212846FEF7D6
:1002B0007DF9002280212846FEF778F9402280212E
:1002C0002846FEF773F98D2280212846FEF76EF945
:1002D000142280212846FEF769F9A12280212846B0
:1002E000FEF764F9C82280212846FEF75FF9DA227A
:1002F00080212846FEF75AF9122280212846FEF76F
:1003000055F9812280212846FEF750F9CF2280211D
:100310002846FEF74BF9D92280212846FEF746F9F8
:10032000F12280212846FEF741F9DB228021284670
:10033000FEF73CF9402280212846FEF737F9A42237
:1003400080212846FEF732F9A62280212846FEF7B2
:100350002DF9AF2280212846FEF728F9A622802118
:100360002846FEF723F9AE2280212846FEF71EF923
:10037000202280212846FEF719F9002280212846F4
:10038000FEF714F9B02280212846FEF70FF940222B
:1003900080212846FEF70AF9002280212846FEF730
:1003A00005F9102280212846FEF700F94FF48064F9
:1003B00035B9013CA4B2002CFBD1012005B0F0BD41
:1003C00000270DF10F062B79012B2AD0022B04F107
:1003D000FF3214D094B2002CF6D18122802128461D
:1003E000FEF7E4F8C82280212846FEF7DFF8AF22A6
:1003F00080212846FEF7DAF8012005B0F0BDAA6892
:10040000013C4021284612F00102A4B218BF00228C
:10041000FEF76CF8002CD6D1002DDED1012005B0FE
:10042000F0BDAA68013C95F9100002F0010CA4B2DD
:10043000697C40228DF80F70CDE9006CF3F760F90C
:10044000002CC0D1C9E700BFA0660024FBF766B945
:10045000FBF764B9FBF762B9FBF760B9FBF75EB96C
:10046000FBF75CB9FBF75AB901207047034620B18E
:10047000026812B1D26902B1104793ED017AF6EE2B
:10048000007A074BB8EEC77AD3ED016AE7EE267A19
:10049000FDEEE77A17EE900A00F30B00704700BFFD
:1004A000DC700024034620B1026812B1126A02B166
:1004B000104793ED027AF6EE007A074BB8EEC77A52
:1004C000D3ED026AE7EE267AFDEEE77A17EE900AA0
:1004D00000F30B00704700BFDC700024034628B116
:1004E00002681AB1516A09B19369184793ED037A0A
:1004F000F6EE007A064BB8EEC77AD3ED036AE7EE64
:10050000267AFDEEE77A17EE900A00F30B007047AB
:10051000DC70002410B5044630B1036823B1DB68F9
:1005200013B1BDE81040184703F0AEFED4E9042330
:100530009042994134BF0120002010BDD8B10E4B2C
:10054000F0B5076816460D4A0D463B4483B0044695
:100550009B0A02EB4303988A64F00AFEC5F3810309
:10056000A188384605F01302CDE900366B096EF01C
:10057000EBFC03B0F0BD70470000FEA7CC8D0C086B
:100580002DE9F04FBA4E85B0BA4CA64256D21D4660
:1005900002E00C36A64251D273798B42F9D13379FD
:1005A000834201D00028F4D1F3799342F1D1346829
:1005B000002C43D0002326606360A360E3602361C6
:1005C0006361A361E36133792371012B96F806B06F
:1005D000C4F808B0317AE16032D0022B2ED1F07A23
:1005E000FBF7B8F996F90970A061B07A2774FBF7A8
:1005F000B1F906466061F0B1DFF8948207EB47017C
:100600007B0058F8319008EBC1010193B9F1000F5C
:1006100011D0887DE8B10E2200230D213046F27101
:100620003372B571FBF7BEF93368B2889A61204620
:1006300005B0BDE8F08F2046FDF7E0FE0024F6E7A8
:10064000F07AFBF787F9727AB37AA0612274637447
:10065000EDE7B1F808A0504664F08AFD01214FEAA9
:100660005A100AF01F0A023801FA0AF1092812D8B2
:10067000DFE810F0F6001100EE0018011001E600AE
:10068000E000D800D0000A007B4BD3F89C0020EAA1
:100690000101C3F89C107B00D91908EBC10148790E
:1006A000FBF758F9791CCBB20146019318B10372DC
:1006B00040F60A30C8807B000291D81908EBC000D0
:1006C000C079FBF747F902990346039020B1019ADC
:1006D000027240F60A50D8807B000291D81908EBCC
:1006E000C0008079FBF736F90299824628B1019B58
:1006F000037240F60A40AAF806007B00D8191BF0E6
:10070000040308EBC0000293807A0246084614BF37
:100710004E212E21FFF712FF03987B002E2103EBC1
:10072000070B08EBCB0B9BF80B20FFF707FF50469E
:100730009BF80C200E21FFF701FF9BF804A0BAF1F3
:10074000000F40F0ED80D9F8002022F00102C9F836
:1007500000204A4A914500F0C180494A914540F045
:10076000AC80454AD2F8901041F48041C2F8901014
:10077000D2F8901021F48041C2F89010029B002B17
:1007800040F098804FF000714FF08072D9F80C0063
:1007900040F00040C9F80C00D9F8080020F4F070CF
:1007A000C9F80800D9F80000C00727D4D9F8080014
:1007B000344B034034481843C9F80800D9F80C00FA
:1007C000C30005D4D9F8000040F48050C9F80000F7
:1007D000D9F80C0011432D4A02400A4342F08862C6
:1007E000C9F80C20D9F8002022F40062C9F80020D2
:1007F000D9F8502022F00102C9F85020BAF1000FB8
:1008000040F09B807B003B4408EBC308012388F841
:10081000163000E7184BD3F8880020EA0101C3F82E
:10082000881038E7144BD3F88C0020EA0101C3F894
:100830008C1030E7104BD86F20EA0101D9672AE706
:100840000D4BD3F8940020EA0101C3F8941022E77D
:10085000094BD3F8800020EA0101C3F880101AE7A1
:10086000054BD3F8980020EA0101C3F8981012E76D
:10087000A0020008FC0300080044025800300140B8
:1008800000380040E0FFBF8F07000020FFFF39D88D
:10089000A80200243E4BD3F8900020EA0101C3F8DF
:1008A0009010F8E63A4BD3F8840020EA0101C3F82F
:1008B0008410F0E600210A4668E7364A91451BD1CC
:1008C000334AD2F8901041F40041C2F89010D2F8A7
:1008D000901021F40041C2F890104FE72C4AD2F852
:1008E000981041F48051C2F89810D2F8981021F471
:1008F0008051C2F8981041E7274A914527D0274AEE
:10090000914532D1224AD2F8981041F48011C2F8B0
:100910009810D2F8981021F48011C2F898102DE7A1
:100920005046FBF717F820B1019B40F60A620372AC
:10093000C2800D21FBF736F805E75046FBF70AF8B1
:1009400000283FF45FAF0268838893615AE7104A3A
:10095000D2F8981041F40051C2F89810D2F89810CB
:1009600021F40051C2F8981008E70D4A91457FF430
:1009700005AF02F50C32D2F89C1041F02001C2F80C
:100980009C10D2F89C1021F02001C2F89C10F5E6D2
:1009900000440258003C0040003401400050014037
:1009A00000140058084B53F8203029B153B19A88ED
:1009B000196812048A617047002BFCD01A689B8862
:1009C00093617047704700BFC08D0C082DE9F04F50
:1009D000DFF84C9283B099F8FCA0BAF1000F02D076
:1009E00003B0BDE8F08FD9F8F840237C002BF7D195
:1009F00099F84DBAD44699F84C7A09F5256099F8DA
:100A00004EEA01228349CDE900A4DA468378C5780D
:100A1000C3F1FF032C469BB293B1B0F80080C3F141
:100A2000FF037D4E05FB03F3A6FB08B61B127609F8
:100A3000052E00F2EA80DFE806F0D5BAA1856B4EFC
:100A4000AE46AB462B46A2460125274600951E0220
:100A500046EA0446172446EA0B060CEB040802FAA1
:100A600004F5A8EB0403013C35429BB208BF012505
:100A700003F12A0318BF022541F82350631CEED16D
:100A80000430664B0CF1180C98421FFA8CFCBDD157
:100A90004FF44063D346DDF800A0A9F8503C802312
:100AA000019CA9F8523CBAF1000F05D089F84EEA32
:100AB00089F84DBA89F84C7A99F8543C002B8FD0BC
:100AC000204640F62B41F3F7FFFD204603B0BDE87A
:100AD000F04FF3F771BE504EEF1A5FFA83FA1C46DF
:100AE0002B46A6FB08E56D09C5EB0515A8EB8505AA
:100AF000ADB2C5F13C0507FB05F51F46A6FB056534
:100B00000AEB55155FFA85FE0125F34600959EE731
:100B1000414FEE1AAB465FFA83FA1C46A7FB085317
:100B2000DE465B09C3EB0313A8EB83039BB203FB15
:100B300006F6A7FB063701230AEB57170093FFB20F
:100B40003B4684E7344EA5EB030EAB46DFB2A6FB73
:100B500008546409C4EB0414A8EB8404A4B2C4F1DF
:100B60003C040EFB04F4DE46A6FB046407EB5414BD
:100B70005FFA84FA01240094544668E7DFF898E0AD
:100B8000EE1AAA46DFB2AEFB08B56D09C5EB051536
:100B9000A8EB8505ADB205FB06F6AEFB065E0125AA
:100BA00007EB5E1E00955FFA8EFEF3464FE71A4E86
:100BB000EF1A5FFA83FEAA469B46A6FB08535B0921
:100BC000C3EB0313A8EB83039BB2C3F13C0303FB0A
:100BD00007F70123A6FB076700930EEB5717FFB239
:100BE0003B4634E7EC1A0C4E5FFA83FE9B4608FB4B
:100BF00004F42B462F46A6FB04640EEB54145FFA54
:100C000084FA01240094544621E754463B46F346B7
:100C10001DE700BF4803003089888888F0720024EF
:100C2000A0660024F8B5354DD5F8F84074B195F8B4
:100C3000FC3006465BB162685379032B5BD8DFE872
:100C400003F04B4E5102136840331E60F8BD6368D9
:100C50002B4A1B69C3F3032352F82300E3685F6840
:100C6000EFF31183102282F31288DFF89CC06268D0
:100C70001CF80000234992F805C031F81C10D2F886
:100C800000C001F4F051DCF80C2022EA0102E16816
:100C9000CCF80C203A5822F001023A500A691F2A77
:100CA00023D94868203A202101FA02F2C260DBB25F
:100CB00083F31188002223682274586890F83D302D
:100CC000012B01D16DF01EFAD5F8F8400022E3683F
:100CD0001A77FAF71DFEAEE713683433B5E71368E9
:100CE0003833B2E713683C33AFE74868202101FA94
:100CF00002F28260DBE700231B60FFDEA0660024B7
:100D0000188C0C08388C0C08888D0C0810B5234CF6
:100D1000D4F8F8308BB194F8FC2072B1204A92F8E4
:100D20000421032A0AD0022A10D0002384F8FC30C0
:100D3000FAF7B6FD08B984F8540C10BD5A68537917
:100D4000032B27D8DFE803F023201D185A685379B6
:100D5000032B1FD8DFE803F00D0A070213684033A6
:100D600000221A6010BD13683C33F9E7136838336A
:100D7000F6E713683433F3E71368403364221A60EC
:100D800010BD13683C33F9E713683833F6E713688E
:100D90003433F3E700231B60FFDE00BFA0660024AE
:100DA00080AA002470B5424D82B0D5F844458CB37A
:100DB00095F84835012B41D0022B2DD1082294F90A
:100DC0001030002185F84B258DF8052040F20442B3
:100DD00003EB43038DF80410ADF80620354A52F8B2
:100DE0003300A3689A0743D5042300210DEB0302C7
:100DF000F3F792F9A3689B0722D53C22FF212E48E6
:100E000076F0DCFC95F8493523B901F0C5FA0123E9
:100E100085F8493502B070BD0DF10302A0212046CE
:100E2000FEF7F6F99DF8033003F00503012B3AD0E5
:100E3000002B32D1D5F844450822C0E74822BEE74E
:100E40001E4A4FF4FA701E4BD2F8242A1D4900FBAB
:100E500002F24868A3FB023292094B681B1A9A42BD
:100E6000FBD26369002BC8D01A689B889361C4E7E2
:100E700063691BB11A689B881B0493610F4B11496E
:100E8000D3F8242A0E4BD2004E68A3FB02329209FB
:100E90004B689B1B9A42FBD2A6E70B4A40F2DC53FD
:100EA00012689A42B6D9D5F84445482287E700BF70
:100EB00090880024A802002484C20024A066002494
:100EC000D34D6210001000E07031002400212DE9A4
:100ED000F04F4FF00A0AA7B09E4E0C469E4D89E097
:100EE000B9F1000F18D142F04002BEF18C0F85F825
:100EF0004C2500F2E18004F1010C98340CF1980CBF
:100F00000DEB040974464FF0040EEC4409F88CEC28
:100F100004F1020E0CF88C2CBEF18C0F40F0020C88
:100F200000F2CA8004F198024FF005096A4402F801
:100F30008BCC04F1040C02F88C9CBCF18C0F00F2F9
:100F4000BB800EF1980E4FF0060B9B00EE44DBB217
:100F50000EF88CBC04F1060E02F8897CBEF18C0FF1
:100F600000F2AA8004F19C0C4FF0070BEC440CF843
:100F70008CBC02F8873C04F108038C2B00F29C80A7
:100F800004F19E0C0DEB0C0E0EF88C9C02F8850CF7
:100F900004F10A008C2800F28F8004F1A0034FF0C6
:100FA000060C6B4403F88CCC02F8837C04F10C0231
:100FB0008C2A00F2818004F10B0304F1A200144694
:100FC000983368446B4400F88CBC03F88C8C480957
:100FD00001F01F070122BAF1010A56F8203002FA87
:100FE00007F223EA020346F820306FD00131B1F551
:100FF000F07F6BD23C223046FBF7ECFD011E5EDB3E
:1010000005EB410395F84C25C1F30720CFB2B3F8A7
:1010100050C502F0400904F1020E01951CF0040FC6
:101020005FFA8CF34FEA1C287FF45AAFB9F1000F36
:1010300003D102F0380C9C4516D002F08702BEF1B5
:101040008C0F42EA030285F84C2535D8631C98348E
:101050004FF0040C6C44983304F88CCC6B44744609
:101060000EF1020E03F88C2CBEF18C0F24D804F183
:1010700098030DEB0302052302F88C3C231D02F8B4
:101080008B0C8C2B18D80EF198000DEB000E06205F
:101090000EF88C0C201802F8897C8C280CD8621D64
:1010A00004F19C030727044698326B446A4403F812
:1010B0008C7C02F88C8C8AE76FF0004487E71CB9BF
:1010C000204627B0BDE8F08F234B0193019B2349B5
:1010D000D3F8445595F91030AA6803EB43039207FF
:1010E00051F8330021D5234603AA0021F3F714F861
:1010F000AB689B0701D50120E3E7194A4FF4FA706A
:10110000184BD2F8242A184900FB02F24868A3FBC6
:10111000023292094B681B1A9A42FBD26B69002B70
:10112000E9D01A689B889361E5E76B691BB11A687F
:101130009B881B0493610A4B0B49D3F8242A094B63
:10114000D2004E68A3FB023292094B689B1B9A4265
:10115000FBD2C8E784C2002490880024A80200249F
:10116000A0660024D34D6210001000E0437913F014
:10117000010306D0C268D0E90731581A531E18403F
:1011800070471846704700BF437913F0020307D039
:101190000269D0E90913581E531E401A18407047BF
:1011A000184670474379024613F0010017D0106AC1
:1011B000D168D36901F1FF3C1B1A13EA0C030CD070
:1011C00000F1010C536900B5BCFBF1FE1B5C01FB97
:1011D0001EC1D8B211625DF804FB18467047704713
:1011E00043799B070AD5436A8269D154436A0269ED
:1011F0000133B3FBF2F102FB11334362704700BFCE
:101200004171704781717047D0E90920101AB0FA16
:1012100080F04009704700BF014B1B685B681847AE
:10122000E0DF0024024B08301B689B68184700BFB2
:10123000E0DF002401207047012070470120704743
:10124000012070470120704731B10B4BD3ED017A7B
:10125000F8EEE77AC1ED007A6AB10749074B896871
:10126000DFED076A0B4407EE903AF8EEE77A87EE77
:10127000A67A82ED007A7047E0DF00244D95FFFFEB
:101280000000C84201207047012070478C4A014687
:1012900000239446104610B590F904400C30012C00
:1012A00049D00133092BF7D1854C002394F9040070
:1012B0000C34022852D00133092BF7D1804C002383
:1012C00094F904000C34032863D00133092BF7D1BF
:1012D0007B4C002394F904000C3405286DD00133B5
:1012E000092BF7D1764C002394F904000C3406281E
:1012F00076D00133092BF7D1002392F904000C3288
:10130000072800F086800133092BF6D16D4B1C684D
:10131000630640F19F806C4A00239646104690F881
:1013200004C01430BCF1360F00F0B28001330F2B33
:10133000F5D10023B0E003EB43035CF8233003B3A3
:1013400062480B7990F8D04090F8D100984218BFCD
:101350009C420CBF01200020A6D110BD03EB43032B
:101360005CF823307BB15A480B7990F8D14090F863
:10137000D000984218BF9C420CBF012000209DD194
:1013800010BD4F4C92E74E4C94F904000C340328E6
:101390009BD103EB43035CF82330002B35D04D4841
:1013A0000B7990F8D04090F8D100984218BF9C4239
:1013B0000CBF012000208BD110BD03EB43035CF870
:1013C000233023B344480B7990F8D04090F8D100F3
:1013D000984218BF9C420CBF0120002082D110BD52
:1013E00003EB43035CF82330002B86D03B480B799A
:1013F00090F8D04090F8D100984218BF9C420CBFA2
:1014000001200020A9D0034677E72D4C62E72C4C41
:101410006AE703EB43035CF82330002B3FF476AF1D
:101420002F4A0B7992F8D00092F8D1209A4218BF37
:1014300098420CBF012000207FF468AF10BD0A68FD
:1014400013B11B68934215D000EB80005EF820308A
:1014500093420FD0E0030FD51B4B086803F5967439
:1014600002E014339C4207D01A689042F9D1DA683E
:10147000D201F6D5012010BD0B79142BFAD0173B01
:10148000DAB21E2A19D8174BD34003F0010010BD61
:1014900003EB83030EEB8303002092F804C01432A5
:1014A000BCF1360FCBD001300F28F6D1002BD1D0B4
:1014B0001A680B689A42CDD1DCE7002010BD00BF4E
:1014C000C0910024C0730024CC1B002430060024EB
:1014D00008090024E00B0024B80E00249011002419
:1014E00068140024010000660B4B8446002010B5F0
:1014F00003F5967E02E014339E450BD01A686245D0
:10150000F9D1DA68441C8A42F5D0D9601433E0B2CC
:101510009E45F3D110BD00BFCC1B0024704700BF17
:1015200040F2FF72034B914203EBC003A8BF114688
:1015300019827047E0DF0024112806D8044B03EB22
:101540008003DB6E0BB19B68196026F0D1BA00BF37
:10155000E0DF0024112806D8034B03EB8003DB6E89
:101560000BB19B6819607047E0DF00240C4A1378C8
:101570007BB10C4B93F8B41059B193F8B51059B135
:1015800050680022FA2883F8B520A8BF4FF0FF303A
:1015900070476FF0010070476FF00200704700BFA6
:1015A000E41E0024E0DF00242DE9F041104C00256A
:1015B0001746022304F1B80884F8B910FF21064643
:1015C000424684F8B850FDF7EDFA68B1424630461D
:1015D0000223FF21FDF76AFB30B1B4F8B83028468A
:1015E0005BBA3B80BDE8F0816FF00C00FAE700BF0A
:1015F000E0DF00240B4B93F8B82182B193F8B921B6
:1016000052B109490022886883F8B921B0F5967F64
:10161000A8BF4FF0FF3070476FF0020070476FF0C7
:1016200001007047E0DF0024E41E0024024BD3F8E1
:10163000BC315B68184700BFE0DF0024024BD3F8E1
:10164000BC319B68184700BFE0DF0024024BD3F891
:10165000BC31DB68184700BFE0DF0024014BD868CD
:10166000704700BFE41E0024044B93F8C03113B14F
:10167000034B186970476FF001007047E0DF0024EA
:10168000E41E0024F0B5484D83B095F8B4303BB16A
:1016900095F8C1610446012E38D0022E54D00EB107
:1016A00003B0F0BD012280210068FCF77FFF01221A
:1016B000FF212068FCF77AFF324631462068FCF7AC
:1016C00075FF95F8C22191212068FCF76FFF314624
:1016D00001222068FCF76AFF3246FF212068FCF7F0
:1016E00065FF324680212068FCF760FF3146012209
:1016F0002068FCF75BFF2D4B2D4901221B68087009
:1017000085F8C121C5F8C43103B0F0BD01AA00219C
:101710000068FDF77DFD9DF80430254FDA0738702D
:1017200039D5D5F8C831002BBAD0204AD5F8C41124
:10173000126892B2521A9342B2D24FF0FF32002393
:101740007A6085F8C131ABE701AA13210068FDF783
:101750005FFD9DF80430164F5B073870E1D03346CB
:1017600001AA1E212068FDF7A1FABDF80430206807
:1017700001225CBA0B21FCF719FF0E4BA4B2012227
:101780003870A3FB0434002385F8B520E40885F8FD
:10179000C1317C6084E7054B02221B6885F8C121BA
:1017A000C5F8C4317CE700BFE0DF002470310024BD
:1017B000E41E0024CDCCCCCC38B52D4D04460323FB
:1017C000002105F118020068FDF770FA48B96FF0C2
:1017D0000103002220686B611146BDE83840FCF728
:1017E000E5BE95F81AC008212B7E58B25B00420076
:1017F0000028DBB282F00702B8BFD3B20139F4D1BE
